:100000004BC0000042C2000040C200003EC20000DF
:100010003CC200000C94596938C2000036C200008E
:1000200034C2000032C200000C944F690C94456940
:100030002CC200002AC2000028C2000026C2000014
:1000400024C2000022C2000020C200001EC2000024
:100050001CC200000C94056A18C2000016C2000001
:1000600014C2000012C2000010C200000EC2000044
:100070000CC200000AC2000008C2000006C2000054
:1000800004C2000002C2000000C20000FEC1000065
:10009000FCC10000FAC1000011241FBECFEFD0E266
:1000A000DEBFCDBF0E9400F0D7C10000076342361B
:1000B000B79BD8A71A39685618AEBAAB558C1D3CF9
:1000C000B7CC5763BD6DEDFD753EF6177231BF00BD
:1000D0000000803F05A84CCDB2D44EB93836A902F5
:1000E0000C50B9918688083CA6AAAA2ABE00000036
:1000F000803F08000000BE922449123EABAAAA2A03
:10010000BECDCCCC4C3E00000080BEABAAAAAA3E1D
:1001100000000000BF000000803F00000000000859
:100120004178D3BB4387D1133D190E3CC3BD4282F6
:10013000AD2B3E68EC8276BED98FE1A93E4C80EFB4
:10014000FFBE01C4FF7F3F0000000000FF004C8A9B
:1001500097509545406BA6D8E4B2282EAE90BF26A6
:10016000B14EE86FD0FBE0709A51862C379845323B
:10017000539D06840D971A8CE61E2E0DB41D401655
:100180009AC591F9F786A142660620AFAE19EE270F
:10019000C2BB0EBAB90AAA95CA45040444C1796A19
:1001A00091EE7D3E2E4C960BA96E5A6A9FF56D0519
:1001B000BB8F808DB4F54FC14AE99E674536394FF4
:1001C00075ADF44CB227A939D78036F7C49C7E6A46
:1001D000605F677992B4DD0E4786CD1A6DC6258AB9
:1001E000F464D953D154DB67F78B22BD5CFEA44D78
:1001F000F9A7590EC57E3BF9BA7D430AD39F6C3BE4
:100200000BDEB2875E3710ECC8A6856546290CF177
:10021000D6BCA38C755E4934200DFAE9D7C7B6A7C2
:10022000988A7C6E6155493D32271D1209FFF6EE12
:10023000E5DDD5CEC6BFB9B2ACA6A09A958F8A85AA
:10024000817C78736F6B6864605D5A56FF59E97DF5
:1002500015B150F39942EE9D4F04BC7632F1B2765F
:100260003B03CC98653405D8AC8259320CE7C4A264
:100270008161432509EDD3B9A089725C46321E0B1A
:10028000F8E6D5C4B4A596887A6D6053473C30260D
:100290001B1108FEF5EDE4DCD4CDC6BFB8B1ABA5AB
:1002A0009F99948F8A85807C77736F6B6763605D9D
:1002B000595653504D4A484543403E3C3A383634EF
:1002C00032302E2D2B2A282725242321201F1E1DC6
:1002D0001C1B1A19181716161514131312111110C6
:1002E0000F0F0E0E0D0D0C0C0B0B0B0A0A09090952
:1002F0000808080807070706060606060505050597
:1003000005040404040404030303030303030302B6
:1003100002020202020202020202010101010101C3
:1003200001010101010101010101010101000000C0
:1003300000000000000000000000000000000000BD
:10034000000000000000000000000000FF0C0B0B8C
:100350000B0A0A090909080808080707070606061C
:100360000606050505050504040404040403030347
:100370000303030303020202020202020202020258
:10038000010101010101010101010101010101015D
:10039000010101000000000000000000000000005A
:1003A000000000000000000000000000000000004D
:1003B000000000000000000000000000000000003D
:1003C000000000000000000000000000000000002D
:1003D000000000000000000000000000000000001D
:1003E000000000000000000000000000000000000D
:1003F00000000000000000000000000000000000FD
:1004000000000000000000000000000000000000EC
:1004100000000000000000000000000000000000DC
:1004200000000000000000000000000000000000CC
:1004300000000000000000000000000000000000BC
:1004400000000000000000000000000011241FBE9A
:10045000CFEFD0E2DEBFCDBF1AE1A4EAB9E001C020
:100460001D92AF37B107E1F719E0A0E0B1E0EAE192
:10047000FFEE00E00BBF02C007900D92A43AB10757
:10048000D9F70E943E6A0C948B77BACD2F923F9297
:100490004F925F926F927F928F929F92AF92BF9294
:1004A000CF92DF92EF92FF920F931F93CF93DF9340
:1004B00000D000D0CDB7DEB78AE090E10E942431B1
:1004C00040903B1050903C102091C81020FF15C068
:1004D00025FD02C00C94030E420124FD0FC0809143
:1004E00020109091211095958795480E591E21FD59
:1004F00007C0C12CD12C76010BC0420121FFF9CFDE
:10050000C0902010D0902110EE24D7FCE094FE2C57
:100510000091E9101091EA1020E030E01058210914
:1005200031098091C410882311F40C94FF0D80913F
:10053000FB109091FC10A0E0B0E09058A109B10927
:10054000B7FF02C00C945110B595A7959795879564
:100550009C838B833FB6F89482E19EE00E944230F8
:100560002091360E3091370E3A832983AA2497FCC6
:10057000A094BA2C662457FC6094762C80914C1081
:1005800090914D10B301A201480F591F611D711DBB
:10059000DB01CA01009751E0A507B10524F08FEFF8
:1005A0009FEFA0E0B0E0B7FF02C00C94170E0E94CE
:1005B000CE1246EC41BB469A31E035B925E428B964
:1005C00050EF5BB992EA9EB987E881BB00C000C0DA
:1005D00041BB469A35B928B960ED6BB99EB981BB6C
:1005E00000C000C041BB469A35B928B95BB99EB975
:1005F00081BB6B817C8129813A81AA27629FB12DC1
:100600007303C001369FB00D811D9A1F72039A0BB0
:10061000B00D811D9A1F1124AA2797FDA095BA2F0E
:10062000880D991DAA1DBB1D2091401030914110CD
:10063000820F931FA11DB11D009731E0A307B105E3
:1006400024F08FEF9FEFA0E0B0E0B7FF02C00C9462
:10065000120E0E94CE1246EC41BB469A31E035B9EB
:1006600021E428B950EF5BB990EA9EB987E881BBD5
:1006700000C000C041BB469A35B928B960ED6BB9DE
:100680009EB981BB00C000C041BB469A35B928B9AC
:100690005BB99EB981BB49815A81AA27049FB12DBC
:1006A0001503C001509FB00D811D9A1F14039A0BB2
:1006B000B00D811D9A1F1124AA2797FDA095BA2F6E
:1006C0008C0D9D1DAE1DBF1D2091581030915910ED
:1006D000820F931FA11DB11D009751E0A507B10521
:1006E00024F08FEF9FEFA0E0B0E0B7FF02C00C94C2
:1006F0000D0E0E94CE1246EC41BB469A31E035B950
:1007000021E428B950EF5BB992EA9EB987E881BB32
:1007100000C000C041BB469A35B928B960EE6BB93C
:100720009EB981BB00C000C041BB469A35B928B90B
:100730005BB99EB981BB8EE09FE00E944230809100
:10074000320F9091330F009711F00C94AA0C0E9475
:10075000CE1246EC41BB469A31E035B925E428B9C2
:1007600050EF5BB990EA9EB987E881BB00C000C03A
:1007700041BB469A35B928B960EB6BB99EB981BBCC
:1007800000C000C041BB469A35B928B95BB99EB9D3
:1007900081BB3FBE3FB73983F8948091400E909162
:1007A000410EA091420EB091430E8B2F9927AA279C
:1007B000BB27892B8A2B8B2B11F00C94A40C8091D6
:1007C000650E823011F40C944F0C10F00C94480C10
:1007D000813011F40C94590D80E090E060915E0E30
:1007E00070915F0E0E94F31920905C0E30905D0EA8
:1007F000280E391E3092610E2092600E80913C0EC0
:1008000090913D0EA0913E0EB0913F0E4091400E52
:100810005091410E6091420E7091430E840F951FCE
:10082000A61FB71F8093400E9093410EA093420ED7
:10083000B093430E80914E1090914F10B301A201DE
:10084000480F591F611D711D4115510581E0680751
:10085000710524F04FEF5FEF60E070E0DB01CA014B
:1008600077FF02C00C94A50D0E94CE1266EC61BB0E
:10087000469A51E055B947E448B970EF7BB992EA1E
:100880009EB987E881BB00C000C061BB469A55B9DC
:1008900048B9E0EDEBB99EB981BB00C000C061BBB7
:1008A000469A55B948B97BB99EB981BB2B813C8129
:1008B000B101AA27269FB12D3703A001729FB00D69
:1008C000411D5A1F36035A0BB00D411D5A1F1124EA
:1008D000662757FD6095762F480D591D6A1D7B1DB3
:1008E0008091421090914310480F591F611D711D56
:1008F0004115510581E06807710524F04FEF5FEF66
:1009000060E070E0DB01CA0177FF02C00C94940D37
:100910000E94CE1266EC61BB469A51E055B943E4A1
:1009200048B970EF7BB990EA9EB987E881BB00C0F7
:1009300000C061BB469A55B948B9E0EDEBB99EB924
:1009400081BB00C000C061BB469A55B948B97BB9AC
:100950009EB981BB9101AA27029FB12D1303A0016B
:10096000309FB00D411D5A1F12035A0BB00D411D8F
:100970005A1F1124662757FD6095762F4C0D5D1D7B
:100980006E1D7F1D80915A1090915B10480F591F6A
:10099000611D711D4115510531E06307710524F09A
:1009A0004FEF5FEF60E070E0DB01CA0177FF02C04C
:1009B0000C948F0D0E94CE1246EC41BB469A31E05A
:1009C00035B923E428B950EF5BB992EA9EB987E8BC
:1009D00081BB00C000C041BB469A35B928B960EE62
:1009E0006BB99EB981BB00C000C041BB469A35B906
:1009F00028B95BB99EB981BB80913C0F90913D0FA6
:100A0000A0913E0FB0913F0F8B2F9927AA27BB27AC
:100A1000892B8A2B8B2B09F054C78091610F823070
:100A200009F4F3C608F0EBC6813009F4E1C780E0B1
:100A300090E060915A0F70915B0F0E94F319209122
:100A4000580F3091590F280F391F30935D0F2093A5
:100A50005C0F8091380F9091390FA0913A0FB091AF
:100A60003B0F40913C0F50913D0F60913E0F7091B4
:100A70003F0F840F951FA61FB71F80933C0F9093C5
:100A80003D0FA0933E0FB0933F0F2115310509F0A4
:100A900022C780E090E00E94CE1246EC41BB469A0D
:100AA00031E035B927E428B950EF5BB990EA9EB937
:100AB00087E881BB00C000C041BB469A35B928B960
:100AC00060EB6BB99EB981BB00C000C041BB469AC8
:100AD00035B928B95BB99EB981BB39813FBF2FB702
:100AE0002983F89480916A0E90916B0EA0916C0E00
:100AF000B0916D0E8B2F9927AA27BB27892B8A2BA4
:100B00008B2B09F0E3C680918F0E823009F494C6D6
:100B100008F08CC6813009F4BBC780E090E060919A
:100B2000880E7091890E0E94F3192090860E3090E5
:100B3000870E280E391E30928B0E20928A0E8091DD
:100B4000660E9091670EA091680EB091690E40916B
:100B50006A0E50916B0E60916C0E70916D0E840F49
:100B6000951FA61FB71F80936A0E90936B0EA093DC
:100B70006C0EB0936D0E8091501090915110B30196
:100B8000A201480F591F611D711D4115510531E02A
:100B90006307710524F04FEF5FEF60E070E0DB0169
:100BA000CA0177FF01C0CDC70E94CE1266EC61BBBF
:100BB000469A51E055B941E448B970EF7BB990EAE3
:100BC0009EB987E881BB00C000C061BB469A55B999
:100BD00048B9E0EEEBB99EB981BB00C000C061BB73
:100BE000469A55B948B97BB99EB981BB6B817C8166
:100BF0009101AA27629FB12D7303A001369FB00D0A
:100C0000411D5A1F72035A0BB00D411D5A1F11246A
:100C1000662757FD6095762F480D591D6A1D7B1D6F
:100C20008091441090914510480F591F611D711D0E
:100C30004115510531E06307710524F04FEF5FEF77
:100C400060E070E0DB01CA0177FF01C076C70E9457
:100C5000CE1266EC61BB469A51E055B945E448B9FD
:100C600070EF7BB990EA9EB987E881BB00C000C0F5
:100C700061BB469A55B948B9E0EDEBB99EB981BB65
:100C800000C000C061BB469A55B948B97BB99EB94E
:100C900081BBB101AA27069FB12D1703A001709F48
:100CA000B00D411D5A1F16035A0BB00D411D5A1F9E
:100CB0001124662757FD6095762F4C0D5D1D6E1D26
:100CC0007F1D80915C1090915D10480F591F611D30
:100CD000711D4115510581E06807710524F04FEF42
:100CE0005FEF60E070E0DB01CA0177FD22C70E9480
:100CF000CE1246EC41BB469A31E035B925E428B91D
:100D000050EF5BB992EA9EB987E881BB00C000C092
:100D100041BB469A35B928B960EE6BB99EB981BB23
:100D200000C000C041BB469A35B928B95BB99EB92D
:100D300081BB8091660F9091670FA091680FB09171
:100D4000690F8B2F9927AA27BB27892B8A2B8B2BDF
:100D500009F0EDC580918B0F823009F486C508F04B
:100D60007EC5813009F407C680E090E06091840F71
:100D70007091850F0E94F3192091820F3091830F9B
:100D8000280F391F3093870F2093860F8091620FB1
:100D90009091630FA091640FB091650F4091660F21
:100DA0005091670F6091680F7091690F840F951FC4
:100DB000A61FB71F8093660F9093670FA093680FCD
:100DC000B093690F2115310509F0B6C580E090E0B8
:100DD0000E94CE1246EC41BB469A31E035B921E47F
:100DE00028B950EF5BB992EA9EB987E881BB00C091
:100DF00000C041BB469A35B928B960EB6BB99EB9C2
:100E000081BB00C000C041BB469A35B928B95BB967
:100E10009EB981BB29812FBF3FB73983F894809158
:100E2000940E9091950EA091960EB091970E8B2FE7
:100E30009927AA27BB27892B8A2B8B2B09F072C5F0
:100E40008091B90E823009F4C7C408F0BFC4813064
:100E500009F4A7C580E090E06091B20E7091B30EE6
:100E60000E94F3192090B00E3090B10E280E391E5A
:100E70003092B50E2092B40E8091900E9091910E0A
:100E8000A091920EB091930E4091940E5091950EB8
:100E90006091960E7091970E840F951FA61FB71F35
:100EA0008093940E9093950EA093960EB093970E08
:100EB0008091521090915310B301A201480F591F15
:100EC000611D711D4115510581E06807710524F010
:100ED0004FEF5FEF60E070E0DB01CA0177FDFFC517
:100EE0000E94CE1266EC61BB469A51E055B943E4CC
:100EF00048B970EF7BB990EA9EB987E881BB00C022
:100F000000C061BB469A55B948B9E0EEEBB99EB94D
:100F100081BB00C000C061BB469A55B948B97BB9D6
:100F20009EB981BB2B813C81B101AA27269FB12D9F
:100F30003703A001729FB00D411D5A1F36035A0B93
:100F4000B00D411D5A1F1124662757FD6095762F5D
:100F5000480D591D6A1D7B1D8091461090914710C8
:100F6000480F591F611D711D4115510581E068072A
:100F7000710524F04FEF5FEF60E070E0DB01CA0124
:100F800077FDC5C50E94CE1266EC61BB469A51E062
:100F900055B947E448B970EF7BB990EA9EB987E844
:100FA00081BB00C000C061BB469A55B948B9E0EDAD
:100FB000EBB99EB981BB00C000C061BB469A55B970
:100FC00048B97BB99EB981BB9101AA27029FB12D77
:100FD0001303A001309FB00D411D5A1F12035A0B7D
:100FE000B00D411D5A1F1124662757FD6095762FBD
:100FF0004C0D5D1D6E1D7F1D80915E1090915F10E8
:10100000480F591F611D711D4115510531E06307DE
:10101000710524F04FEF5FEF60E070E0DB01CA0183
:1010200077FD71C50E94CE1246EC41BB469A31E075
:1010300035B927E428B950EF5BB992EA9EB987E841
:1010400081BB00C000C041BB469A35B928B960EEEB
:101050006BB99EB981BB00C000C041BB469A35B98F
:1010600028B95BB99EB981BB8091900F9091910F87
:10107000A091920FB091930F8B2F9927AA27BB278E
:10108000892B8A2B8B2B09F033C48091B50F8230CA
:1010900009F489C308F081C3813009F4E8C480E011
:1010A00090E06091AE0F7091AF0F0E94F319209104
:1010B000AC0F3091AD0F280F391F3093B10F209333
:1010C000B00F80918C0F90918D0FA0918E0FB091E9
:1010D0008F0F4091900F5091910F6091920F7091EE
:1010E000930F840F951FA61FB71F8093900F9093A7
:1010F000910FA093920FB093930F2115310509F032
:1011000001C480E090E00E94CE1246EC41BB469ABA
:1011100031E035B923E428B950EF5BB992EA9EB9C2
:1011200087E881BB00C000C041BB469A35B928B9E9
:1011300060EB6BB99EB981BB00C000C041BB469A51
:1011400035B928B95BB99EB981BB29812FBF3FB79B
:101150003983F8948091BE0E9091BF0EA091C00E7D
:10116000B091C10E8B2F9927AA27BB27892B8A2BD9
:101170008B2B09F0C2C38091E30E823009F4FAC2CE
:1011800008F0F2C2813009F41DC480E090E0609163
:10119000DC0E7091DD0E0E94F3192090DA0E309073
:1011A000DB0E280E391E3092DF0E2092DE0E80916B
:1011B000BA0E9091BB0EA091BC0EB091BD0E4091A5
:1011C000BE0E5091BF0E6091C00E7091C10E840F83
:1011D000951FA61FB71F8093BE0E9093BF0EA093BE
:1011E000C00EB093C10E8091541090915510B30170
:1011F000A201480F591F611D711D4115510581E064
:101200006807710524F04FEF5FEF60E070E0DB01ED
:10121000CA0177FD80C40E94CE1266EC61BB469A7B
:1012200051E055B945E448B970EF7BB990EA9EB9F1
:1012300087E881BB00C000C061BB469A55B948B978
:10124000E0EEEBB99EB981BB00C000C061BB469A1D
:1012500055B948B97BB99EB981BB2B813C81B1019D
:10126000AA27269FB12D3703A001729FB00D411D03
:101270005A1F36035A0BB00D411D5A1F1124662701
:1012800057FD6095762F480D591D6A1D7B1D809175
:10129000481090914910480F591F611D711D41154B
:1012A000510581E06807710524F04FEF5FEF60E0C2
:1012B00070E0DB01CA0177FD22C40E94CE1266EC09
:1012C00061BB469A51E055B941E448B970EF7BB92A
:1012D00092EA9EB987E881BB00C000C061BB469A14
:1012E00055B948B9E0EDEBB99EB981BB00C000C06B
:1012F00061BB469A55B948B97BB99EB981BB91018A
:10130000AA27029FB12D1303A001309FB00D411DEC
:101310005A1F12035A0BB00D411D5A1F1124662784
:1013200057FD6095762F4C0D5D1D6E1D7F1D8091C4
:10133000601090916110480F591F611D711D41157A
:10134000510531E06307710524F04FEF5FEF60E076
:1013500070E0DB01CA0177FDCEC30E94CE1246ECDD
:1013600041BB469A31E035B921E428B950EF5BB969
:1013700090EA9EB987E881BB00C000C041BB469A95
:1013800035B928B960EB6BB99EB981BB00C000C00C
:1013900041BB469A35B928B95BB99EB981BB8091EA
:1013A000BA0F9091BB0FA091BC0FB091BD0F8B2FC6
:1013B0009927AA27BB27892B8A2B8B2B09F093C24D
:1013C0008091DF0F823009F4BCC108F0B4C18130D4
:1013D00009F43CC380E090E06091D80F7091D90F80
:1013E0000E94F3192091D60F3091D70F280F391F83
:1013F0003093DB0F2093DA0F8091B60F9091B70FE7
:10140000A091B80FB091B90F4091BA0F5091BB0F96
:101410006091BC0F7091BD0F840F951FA61FB71F61
:101420008093BA0F9093BB0FA093BC0FB093BD0FE6
:101430002115310509F097C280E090E00E94CE129C
:1014400046EC41BB469A31E035B925E428B950EF66
:101450005BB992EA9EB987E881BB00C000C041BB7E
:10146000469A35B928B960EB6BB99EB981BB00C00B
:1014700000C041BB469A35B928B95BB99EB981BB5A
:1014800029812FBF3FB73983F89484EE9EE00E94F4
:1014900042302090080F3090090F809156109091A3
:1014A0005710480E591E611C711C4114510441E033
:1014B000640671042CF044244A94542C612C712C41
:1014C000D301C20177FC07C30E94CE1246EC41BB98
:1014D000469A31E035B927E428B950EF5BB990EA74
:1014E0009EB987E881BB00C000C041BB469A35B9B0
:1014F00028B960EE6BB99EB981BB00C000C041BB8A
:10150000469A35B928B95BB99EB981BB6B817C819C
:101510009101AA27629FB12D7303A001369FB00DE0
:10152000411D5A1F72035A0BB00D411D5A1F112441
:10153000662757FD6095762F480D591D6A1D7B1D46
:1015400080914A1090914B10480F591F611D711DD9
:101550004115510531E06307710524F04FEF5FEF4E
:1015600060E070E0DB01CA0177FDC1C20E94CE12CB
:1015700046EC41BB469A31E035B923E428B950EF37
:101580005BB992EA9EB987E881BB00C000C041BB4D
:10159000469A35B928B960ED6BB99EB981BB00C0D8
:1015A00000C041BB469A35B928B95BB99EB981BB29
:1015B000B101AA27069FB12D1703A001709FB00D9E
:1015C000411D5A1F16035A0BB00D411D5A1F1124FD
:1015D000662757FD6095762F4C0D5D1D6E1D7F1D96
:1015E0008091621090916310480F591F611D711D09
:1015F0004115510581E06807710524F04FEF5FEF59
:1016000060E070E0DB01CA0177FD6DC2C7D746EC30
:1016100041BB469A31E035B923E428B950EF5BB9B4
:1016200090EA9EB987E881BB00C000C041BB469AE2
:1016300035B928B960EB6BB99EB981BB00C000C059
:1016400041BB469A35B928B95BB99EB981BB80EEDA
:101650009FE00E9442308091041090910510009705
:1016600009F058C19BD746EC41BB469A31E035B9E9
:1016700027E428B950EF5BB992EA9EB987E881BBAD
:1016800000C000C041BB469A35B928B960EB6BB9C0
:101690009EB981BB00C000C041BB469A35B928B98C
:1016A0005BB99EB981BB29812FBF2091A809922FD8
:1016B0009C7111E009F010E0922F9370923009F4C0
:1016C000E4C4933009F4D6C4913009F4B5C21111C1
:1016D000F3C480E00E94F33D8091A4099091A50994
:1016E000A091A609B091A7090196A11DB11D8093F3
:1016F000A4099093A509A093A609B093A7092091E6
:10170000A8092F5F2093A8090F900F900F900F90BA
:10171000DF91CF911F910F91FF90EF90DF90CF90CD
:10172000BF90AF909F908F907F906F905F904F9001
:101730003F902F900895833009F483C1843009F0DD
:1017400049CE6091BA0F7091BB0F8091BC0F909100
:10175000BD0F2091DC0F211124C2BB27A92F982F88
:10176000872F8095909538CE833009F465C18430F9
:1017700009F00BCD6091BE0E7091BF0E8091C00E2E
:101780009091C10E2091E00E21112FC2BB27A92FED
:10179000982F872F80959095FACC833009F447C114
:1017A000843009F07CCC6091900F7091910F809102
:1017B000920F9091930F2091B20F211102C2BB277B
:1017C000A92F982F872F809590956BCC833009F4A3
:1017D000E3C0843009F03ECB6091940E7091950E79
:1017E0008091960E9091970E2091B60E2111CFC147
:1017F000BB27A92F982F872F809590952DCB8330CD
:1018000009F4F1C0843009F012C960913C0F709165
:101810003D0F80913E0F90913F0F20915E0F40EA67
:1018200051E00E94C42F8095909503C9833009F43C
:10183000F9C0843009F071C960916A0E70916B0E25
:1018400080916C0E90916D0E20918C0E2111B4C17F
:10185000BB27A92F982F872F8095909560C983303B
:1018600009F4DBC0843009F07FCA6091660F709183
:10187000670F8091680F9091690F2091880F211157
:101880008BC1BB27A92F982F872F809590956ECA63
:10189000833009F4BCC0843011F00C94EC036091E7
:1018A000400E7091410E8091420E9091430E209116
:1018B000620E40EA51E00E94C42F809590950C94EE
:1018C000EE0388E39FE00E94F12FA7C886E69EE022
:1018D0000E94F12F18C921154DEF340708F440C1BB
:1018E0008FEF9FEFD8C886EB9FE00E94F12F68CD65
:1018F0008CE89FE00E94F12FC8CB8AEB9EE00E940B
:10190000F12F39CC21154DEF340708F423C18FEFA7
:101910009FEFF9CB8115EDEF9E0708F425C18FEFFE
:101920009FEFA0CE80E99EE00E94F12F89CA82E657
:101930009FE00E94F12F0ECA21159DEF390708F490
:101940000CC18FEF9FEF44CA8CE39EE00E94F12F01
:101950000C94DF0381156DEF960708F40AC18FEF31
:101960009FEF0C94A70321154DEF340708F4FEC038
:101970008FEF9FEF63CD6091660F7091670F80913D
:10198000680F9091690F2091880F21111FC1BB270B
:10199000A92F982F872FEAC98091A40E9091A50EA8
:1019A0005BCA6091940E7091950E8091960E909105
:1019B000970E2091B60E21110EC1BB27A92F982F8B
:1019C000872F4ACA6091BE0E7091BF0E8091C00EE3
:1019D0009091C10E2091E00E2111D4C0BB27A92FF8
:1019E000982F872FD4CB80914C0F90914D0F21C809
:1019F00060913C0F70913D0F80913E0F90913F0F91
:101A000020915E0F40EA53E00E94C42F12C88091DB
:101A1000500E9091510E0C94EE038091760F9091A0
:101A2000770FA4C980917A0E90917B0E78C880912F
:101A3000A00F9091A10F35CB8091CE0E9091CF0E3B
:101A4000A6CB8091CA0F9091CB0FC6CC6091BA0FF4
:101A50007091BB0F8091BC0F9091BD0F2091DC0F56
:101A60002111C8C0BB27A92F982F872FB5CC609113
:101A7000900F7091910F8091920F9091930F209100
:101A8000B20F2111ADC0BB27A92F982F872F09CBEB
:101A900060916A0E70916B0E80916C0E90916D0E3C
:101AA00020918C0E211182C0BB27A92F982F872F40
:101AB00036C86091400E7091410E8091420E909117
:101AC000430E2091620E211157C0BB27A92F982FDA
:101AD000872F0C94EE0380E090E0DC01F5CC80E0F1
:101AE00090E0DC01FDC980E090E0DC018FCD80E07A
:101AF00090E0DC013BCD80E090E0DC012ECC80E08A
:101B000090E0DC01DACB80E090E0DC018BCA80E081
:101B100090E0DC0137CA80E090E0DC017CCB80E023
:101B200090E0DC010C94DA0480E090E0DC010C949D
:101B3000880480E090E0DC01DAC880E090E0DC011D
:101B400086C880E090E0DC012FC880E090E0DC01F6
:101B50000C943404C9019D5FD6CAC9019D5F38C980
:101B6000C9019D5F0C944B059D5F7CCDC9019D5FB4
:101B700065CC9D5F0C94A70340EA53E00E94041AD1
:101B80000C94EE0340EA53E00E94041A00CB40EAB2
:101B900051E00E94041A30CE40EA51E00E94041A3B
:101BA00074CE40EA51E00E94041ADBCD40EA53E0D3
:101BB0000E94041A0C948F0540EA51E00E94041A16
:101BC0004BCE40EA51E00E94041AFDCD40EA53E0BA
:101BD0000E94041ACBC840EA53E00E94041A3CC990
:101BE00040EA53E00E94041A5CCA40EA51E00E94B5
:101BF000041AD0CD40EA53E00E94041AEDCB1C82B7
:101C00001B820C94AA028090201090902110959431
:101C10008794840C951C0C946D0280E090E0DC01AC
:101C20000C94790380E090E0DC010C94290380E0BF
:101C300090E0DC010C94D7020E94E955809151128A
:101C4000882309F433C28091BB10882379F0815036
:101C50008093BB108091030D811131C28091040DDE
:101C600081112DC28091020D811147C38091B41062
:101C7000882309F407C28091B2109091B31040916B
:101C8000641050916510209140103091411024173C
:101C9000350708F402C34217530770F4B901641BF7
:101CA000750BAB018617970708F4AC01241B350BA5
:101CB000309341102093401040917010509171105A
:101CC00020914C1030914D102417350708F4D9C2DB
:101CD0004217530770F4F901E41BF50BAF018E179F
:101CE0009F0708F4AC01241B350B30934D10209353
:101CF0004C1040917C1050917D10209158103091E3
:101D000059102417350708F4B0C24217530770F46E
:101D1000B901641B750BAB018617970708F4AC017A
:101D2000241B350B309359102093581040916610A6
:101D300050916710209142103091431024173507BD
:101D400008F487C24217530770F4F901E41BF50B3E
:101D5000AF018E179F0708F4AC01241B350B30939D
:101D600043102093421040917210509173102091B3
:101D70004E1030914F102417350708F45DC24217FA
:101D8000530770F4B901641B750BAB0186179707F5
:101D900008F4AC01241B350B30934F1020934E10E8
:101DA00040917E1050917F1020915A1030915B101D
:101DB0002417350708F433C24217530770F4F901AA
:101DC000E41BF50BAF018E179F0708F4AC01241B31
:101DD000350B30935B1020935A104091681050914E
:101DE000691020914410309145102417350708F4EC
:101DF00009C24217530770F4B901641B750BAB019C
:101E00008617970708F4AC01241B350B3093451057
:101E100020934410409174105091751020915010EF
:101E2000309151102417350708F4DFC142175307CA
:101E300070F4F901E41BF50BAF018E179F0708F44E
:101E4000AC01241B350B309351102093501040915E
:101E500080105091811020915C1030915D102417FA
:101E6000350708F4B5C14217530770F4B901641B74
:101E7000750BAB018617970708F4AC01241B350BD3
:101E800030935D1020935C1040916A1050916B105C
:101E900020914610309147102417350708F48BC164
:101EA0004217530770F4F901E41BF50BAF018E17CD
:101EB0009F0708F4AC01241B350B30934710209387
:101EC0004610409176105091771020915210309129
:101ED00053102417350708F461C14217530770F4F3
:101EE000B901641B750BAB018617970708F4AC01A9
:101EF000241B350B309353102093521040918210C5
:101F00005091831020915E1030915F102417350797
:101F100008F437C14217530770F4F901E41BF50BBD
:101F2000AF018E179F0708F4AC01241B350B3093CB
:101F30005F1020935E1040916C1050916D102091B5
:101F40004810309149102417350708F40DC1421785
:101F5000530770F4B901641B750BAB018617970723
:101F600008F4AC01241B350B309349102093481022
:101F70004091781050917910209154103091551063
:101F80002417350708F4E3C04217530770F4F9012A
:101F9000E41BF50BAF018E179F0708F4AC01241B5F
:101FA000350B30935510209354104091841050916C
:101FB000851020916010309161102417350708F4C6
:101FC000B9C04217530770F4B901641B750BAB011C
:101FD0008617970708F4AC01241B350B309361106A
:101FE0002093601040916E1050916F1020914A1014
:101FF00030914B102417350708F089C0421B530B52
:102000008417950708F477C1420F531F50934B1064
:1020100040934A1040917A1050917B1020915610B5
:10202000309157102417350708F05EC0421B530B40
:102030008417950708F45DC1420F531F5093571042
:102040004093561040918610509187102091621055
:102050003091631024173507A8F5421B530B8417E2
:10206000950708F444C1420F531F509363104093E7
:10207000621008C022FD45CB812F0E944B23812F87
:102080000E94EB262091A8093CCB85E290E10E94BA
:1020900024318091C81088700E94552C2091A80985
:1020A00030CB0196A11DB11D0C94A4028091BB10F0
:1020B000882309F4CFCDCBCD0E9418370ACB0E94DC
:1020C0000B58D0CD42175307E8F6F901E41BF50B86
:1020D000AF018E179F0708F4AC01241B350B30931A
:1020E000631020936210CECF4217530708F0AACF97
:1020F000B901641B750BAB018617970708F4AC0197
:10210000241B350B30935710209356109BCF42174A
:10211000530708F07FCFF901E41BF50BAF018E17D1
:102120009F0708F4AC01241B350B30934B10209310
:102130004A1070CF421B530B8417950708F4D5C083
:10214000420F531F50936110409360104BCF421BBE
:10215000530B8417950708F4C6C0420F531F5093C2
:1021600055104093541021CF421B530B84179507F1
:1021700008F4B7C0420F531F5093491040934810C2
:10218000F7CE421B530B8417950708F4A8C0420FE3
:10219000531F50935F1040935E10CDCE421B530BE4
:1021A0008417950708F499C0420F531F509353109A
:1021B00040935210A3CE421B530B8417950708F48B
:1021C0008AC0420F531F509347104093461079CE58
:1021D000421B530B8417950708F47BC0420F531F13
:1021E00050935D1040935C104FCE421B530B8417ED
:1021F000950708F46CC0420F531F50935110409341
:10220000501025CE421B530B8417950708F45DC070
:10221000420F531F5093451040934410FBCD421B77
:10222000530B8417950708F44EC0420F531F509369
:102230005B1040935A10D1CD421B530B8417950766
:1022400008F43FC0420F531F50934F1040934E105D
:10225000A7CD421B530B8417950788F1420F531FDC
:1022600050934310409342107ECD421B530B841772
:10227000950718F1420F531F50935910409358106F
:1022800055CD421B530B84179507A8F0420F531FDF
:1022900050934D1040934C102CCD421B530B841780
:1022A000950738F0420F531F509341104093401050
:1022B00003CDAC01F7CFAC01E9CFAC01DBCFAC0172
:1022C000CDCFAC01BFCFAC01B0CFAC01A1CFAC0141
:1022D00092CFAC0183CFAC0174CFAC0165CFAC0120
:1022E00056CFAC0147CFAC0138CFAC0129CFAC0100
:1022F000BACEAC01A1CEAC0187CE0E948C58B6CC30
:10230000E82FF0E0EE0FFF1FE75DFE4E8081918128
:1023100008958038910538F4FC01E45EFE4F208179
:1023200030E0C90108952FEF3FEFFBCFCF93DF934C
:10233000CFE8D7E1E881F98185EA96E1A1E6B0E04E
:1023400081939193A193B193F983E883DF91CF9126
:102350000895AFE8B7E1ED91FC9111978191ED936C
:10236000FC930895AFE8B7E1ED91FC91119781914D
:10237000ED93FC930895AFE8B7E1ED91FC911197CF
:10238000808191813296ED93FC930895AFE8B7E197
:10239000ED91FC91119760817181828193813496D6
:1023A000ED93FC930895E82FE695E695E695F0E029
:1023B000E659F54F9081992351F08770E82FF0E0AE
:1023C000EC5BF84F2081292381E009F0089580E03B
:1023D0000895FC01A18DBB27A1950CF4B095AA0F1F
:1023E000BB1F119620853185428553850E94287731
:1023F00064877587868797870895CF92DF92EF92DB
:10240000FF92CF93603E710581059105F8F4DC01E0
:10241000CB019F5FAF4FBF4FCC24D82EE92EFA2EB1
:10242000A0E0B0E020E030E0EBBEF601C791A40FE1
:10243000B51FCC932F5F3F4FD9018FEFC81AD80A31
:10244000E80AF80A211581E0380771F7CF91FF906B
:10245000EF90DF90CF900895CF93DF93BC0180E0A1
:1024600090E04FE855E1C9DFCFE8D5E1D093901770
:10247000C0938F171092911789DF653A7641814694
:10248000910551F080E092E0FE019C0111922150F3
:102490003040E1F780E004C065DF8093911781E070
:1024A000DF91CF910895AF92BF92CF92DF92EF92DA
:1024B000FF920F931F93CF93DF935C01C12CD12C1C
:1024C0007601C0E0D0E0062F10E00EC0A601415713
:1024D0005A4EBE016A0D7B1D80E090E08EDF219692
:1024E0002FEFD21AE20AF20AC017D10778F3CFE829
:1024F000D5E1D0939017C0938F171092911746DFB4
:10250000653A76418146910551F080E092E0FE0106
:102510009C01119221503040E1F780E004C022DF9D
:102520008093911781E0DF91CF911F910F91FF90E0
:10253000EF90DF90CF90BF90AF9008956095E9E75E
:10254000F4E19081982B6923608386EC81BB469AE5
:10255000362F330F962F9695262F221F2227221FC4
:10256000832F8670282B20646071832F880F8072E0
:10257000862B307C832B9270906C31E035B928B972
:102580008BB99EB987E881BB85E08A95F1F7000099
:10259000E8E7F4E180818F5F808308959C01232F19
:1025A000332726952695722F66EC61BB469A522FEB
:1025B000550F452F46704068207133272260352F14
:1025C000330F3072322B507C352B272F26952270FB
:1025D000206215B848B93BB92EB957E851BB96955A
:1025E000879596958795282F61BB469A482F440F6B
:1025F000382F3695221F2227221F642F6670262B24
:102600002068807199278260942F990F9072982B7F
:10261000407C942B327015B828B99BB93EB951BB98
:1026200008950F931F93072F069510E00F7711273A
:10263000282F2F7740914F124F704069E0919219E7
:10264000F091931963E070E082E999E109951F9197
:102650000F9108950F93262F4F772F778F708068F3
:10266000E0919219F0919319042F482F63E070E0E4
:1026700082E999E109950F910895EF92FF920F93E6
:102680001F93CF93DF93EC01162FF42EE22E80914F
:10269000B719843071F1C230D10509F453C0C33089
:1026A000D10571F1C130D105F9F1C430D105C8F5BA
:1026B000E091AE19F091AF19309739F00E2D2F2D12
:1026C000412FBE0182E999E10995E091B019F0919D
:1026D000B119309739F00E2D2F2D412FBE0182E90F
:1026E00099E10995DF91CF911F910F91FF90EF90A4
:1026F0000895E091AC19F091AD193097F9F6D8CF63
:10270000862F807F803A09F48DC008F041C0803860
:1027100009F456C0803961F6E0919619F091971945
:1027200042C0C0E0D0E0C4CF683F50F1E091A819AA
:10273000F091A919309709F4BBCF612F82E999E193
:102740000995C3CF862F807F803D09F455C0803F17
:1027500009F440C0803C09F0ABCFE091A019F091A2
:10276000A119309709F4A4CF133F09F43FC0113FDA
:10277000E9F1612F6F704F2D82E999E10995A5CF9D
:10278000663F09F095CFE091AA19F091AB19D2CF2D
:10279000803ED9F0803FA9F1803B09F089CFE091DC
:1027A0009419F0919519309709F482CF123F99F15D
:1027B000612F6F702E2D4F2D82E999E1099585CFFC
:1027C000E0919819F0919919EECFE0919C19F09150
:1027D0009D19E9CF633F59F1613F09F069CFE0915D
:1027E000A619F091A719309709F462CF4F2D612FE8
:1027F00082E999E1099569CFE091A219F091A319B5
:10280000B0CF623F09F054CFE0919E19F0919F192B
:10281000309709F44DCF2E2D4F2D62EF82E999E1CB
:10282000099553CFE0919A19F0919B19BCCFE09193
:10283000A419F091A5193097C9F63ACF86EC81BB5F
:10284000469A15B880E488B980E58BB980E68EB9E0
:1028500087E881BB85E08A95F1F70000089586EC52
:1028600081BB469A15B880E488B980ED8BB980E6C3
:102870008EB987E881BB85E08A95F1F7000008955D
:1028800086EC81BB469A15B885E488B980E58BB99A
:1028900080E68EB987E881BB85E08A95F1F7000074
:1028A0000895EF92FF920F931F93CF93DF93F82E2B
:1028B000E62EABEA8A9FA12D1124A695A695A69592
:1028C0001A2F1F5F50E0A83008F06AC08A2F90E0EE
:1028D000880F991FFC01EE0FFF1FEE0FFF1FEE0F79
:1028E000FF1FE80FF91FE40FF51FEE0FFF1FE75D55
:1028F000FE4EC081D181183008F476C0FA01EE0F87
:10290000FF1FEB5DFD4E0190F081E02DDA01AA0F73
:10291000BB1FAF5FBD4E8D919C919F01281B390B52
:10292000A12FB0E017970E9460726E0F7F1F811D6C
:10293000911D6115710521E08207910508F06AC0BB
:102940008B010C1B1D0B3E2D20E09BEAF99E912D67
:102950001124969596959695892F880F890F880F43
:10296000880F6F2D681B862F90E0A0E0B0E07727DE
:102970006627620F731F811D911D2CE030E040E03F
:1029800050E00E946977D8010E941E77C80FD91FB6
:10299000CE01DF91CF911F910F91FF90EF9008959D
:1029A000FA01EE0FFF1FEB5DFD4E0190F081E02D6F
:1029B000EA01CC0FDD1FCF5FDD4E888199819F0139
:1029C000281B390BB0E017970E9460726E0F7F1FB3
:1029D000811D911D6115710521E082079105F8F4B3
:1029E000EB01183008F08ACF812F90E0880F991FF3
:1029F000FC01EE0FFF1FEE0FFF1FEE0FFF1FE80F92
:102A0000F91FE40FF51FEE0FFF1FE75DFE4E60811B
:102A1000718196CF6FEF7FEF80E090E091CF6FEF05
:102A20007FEF80E090E0EB01DCCFFF920F931F93EC
:102A3000CF93DF93F82EABEA8A9FA12D1124A695A0
:102A4000A695A6951A2F1F5F462F50E0A83008F0D4
:102A500063C08A2F90E0880F991FFC01EE0FFF1FC3
:102A6000EE0FFF1FEE0FFF1FE80FF91FE40FF51F1A
:102A7000EE0FFF1FE75DFE4EC081D181183008F4D4
:102A80006FC0FA01EE0FFF1FEB5DFD4E0190F0816C
:102A9000E02DDA01AA0FBB1FAF5FBD4E8D919C9157
:102AA0009F01281B390BA12FB0E017970E9460727D
:102AB0006E0F7F1F811D911D6115710521E0820739
:102AC000910508F063C08B010C1B1D0B9BEAF99E5E
:102AD000912D1124969596959695892F880F890F9B
:102AE000880F880F6F2D681B862F90E0A0E0B0E064
:102AF000772766272CE030E040E050E00E946977BD
:102B0000D8010E941E77C80FD91FCE01DF91CF9147
:102B10001F910F91FF900895FA01EE0FFF1FEB5DDB
:102B2000FD4E0190F081E02DEA01CC0FDD1FCF5F5B
:102B3000DD4E888199819F01281B390BB0E01797E2
:102B40000E9460726E0F7F1F811D911D61157105BE
:102B500021E082079105F8F4EB01183008F091CFDD
:102B6000812F90E0880F991FFC01EE0FFF1FEE0FE1
:102B7000FF1FEE0FFF1FE80FF91FE40FF51FEE0F09
:102B8000FF1FE75DFE4E608171819DCF6FEF7FEF8C
:102B900080E090E098CF6FEF7FEF80E090E0EB0176
:102BA000DCCFEF92FF920F931F93CF93DF93ECE86C
:102BB000F0E11192119280E1E03BF807D1F7109219
:102BC000B1101092B0108091D110823009F4F4C08D
:102BD000833009F4D7C0813039F0DF91CF911F9154
:102BE0000F91FF90EF900895C0918A10D0918B10B3
:102BF0001091D010110F60E0812F17DF7C0180E071
:102C00007FDB9701281B390BDE010E9460729093D5
:102C10008D1080938C1061E0812F07DF7C0181E0B3
:102C20006FDB9701281B390BDE010E9460729093C5
:102C30008F1080938E1062E0812FF7DE7C0182E09E
:102C40005FDB9701281B390BDE010E9460729093B5
:102C500091108093901063E0812FE7DE7C0183E088
:102C60004FDB9701281B390BDE010E9460729093A5
:102C700093108093921064E0812FD7DE7C0184E072
:102C80003FDB9701281B390BDE010E946072909395
:102C900095108093941065E0812FC7DE7C0185E05C
:102CA0002FDB9701281B390BDE010E946072909385
:102CB00097108093961066E0812FB7DE7C0186E046
:102CC0001FDB9701281B390BDE010E946072909375
:102CD00099108093981067E0812FA7DE7C0187E030
:102CE0000FDB9701281B390BDE010E946072909365
:102CF0009B1080939A1068E0812F97DE7C0188E01A
:102D0000FFDA9701281B390BDE010E946072909355
:102D10009D1080939C1069E0812F87DE7C0189E003
:102D2000EFDA9701281B390BDE010E946072909345
:102D30009F1080939E106AE0812F77DE7C018AE0ED
:102D4000DFDA9701281B390BDE010E946072909335
:102D5000A1108093A0106BE0812F67DE8C018BE0C7
:102D6000CFDA9801281B390BDE010E946072909324
:102D7000A3108093A210DF91CF911F910F91FF902C
:102D8000EF9008952091D010A0918A10B0918B10EF
:102D900030E00E9460729B01AC01A5E5B5E10E94A4
:102DA0001E779093B1108093B010DF91CF911F9157
:102DB0000F91FF90EF9008952091D010A0918A106C
:102DC000B0918B1030E00E9460729B01AC01A5E5D0
:102DD000B5E10E941E77BB2797FDB095AB2F90936E
:102DE000A5108093A4109093A7108093A6109093A1
:102DF000A9108093A8109093AB108093AA10909381
:102E0000AD108093AC109093AF108093AE10DF9113
:102E1000CF911F910F91FF90EF90089521E030E046
:102E200002C0220F331F8A95E2F7D901A095B09511
:102E30008091290A90912A0A8A239B2390932A0A37
:102E40008093290AE0912B0AF0912C0AEA23FB23B4
:102E5000F0932C0AE0932B0A662371F0822B932BBC
:102E600090932A0A8093290A442331F02E2B3F2B7A
:102E700030932C0A20932B0A089521E030E002C001
:102E8000220F331F8A95E2F7F901E095F0958091C2
:102E9000290A90912A0A8E239F2390932A0A8093CD
:102EA000290A40912B0A50912C0A4E235F235093FC
:102EB0002C0A40932B0A662331F0282B392B3093B0
:102EC0002A0A2093290A0895CF93DF931F92CDB742
:102ED000DEB790E069831DDA80932D0A6981862F21
:102EE00090E017DA80932E0A0F90DF91CF9108952A
:102EF00024E630E040E050E00E9442772AE030E0F3
:102F000040E050E00E944277605D822F805DDCCF20
:102F100021E02093330A009721F48FEF8093320A47
:102F200008951092320ABC0189E39AE00E949176DA
:102F300062EA79E088E39AE00C9486761092820B3C
:102F40001092840B8FEF8093810B8093800B1092F3
:102F50007A0B10927B0B10927C0B10927D0B1092CF
:102F60008D0B10928F0B80938C0B80938B0B109298
:102F7000850B1092860B1092870B1092880B109283
:102F8000980B10929A0B8093970B8093960B10924C
:102F9000900B1092910B1092920B1092930B109237
:102FA000A30B1092A50B8093A20B8093A10B109200
:102FB0009B0B10929C0B10929D0B10929E0B1092EB
:102FC000AE0B1092B00B8093AD0B8093AC0B1092B4
:102FD000A60B1092A70B1092A80B1092A90B10929F
:102FE000B90B1092BB0B8093B80B8093B70B109268
:102FF000B10B1092B20B1092B30B1092B40B089558
:103000001F93CF93DF93D82FC92F162F8091C40B16
:1030100068130AC046E050E06CEB7BE08D2F0E9405
:103020005876009711F424C089DF1093C40B46E052
:1030300050E06FEF70E08CEB9BE00E947F76ED2F0D
:10304000FC2FACEBBBE080E091919F3F19F488230B
:1030500041F004C09D938F5F8630B1F71092BC0B96
:1030600007C086E0ECEBFBE0DF011D928A95E9F7F3
:10307000DF91CF911F910895CF93DF9300D000D0BF
:1030800000D0CDB7DEB786E0E2EDF6E0DE011196C6
:1030900001900D928A95E1F760E0CE010196B0DFD4
:1030A00026960FB6F894DEBF0FBECDBFDF91CF914D
:1030B0000895EF92FF920F931F93CF93DF9300D069
:1030C00000D000D0CDB7DEB746E050E06FEF70E043
:1030D0008E010F5F1F4FC8010E947F76F12CE12CFB
:1030E0008F2D61D98823A9F0F801EE0DF11DE7FCC1
:1030F000FA95F082EE2021F089819F2D981B908314
:10310000E39485E08E152CF461E0CE01019678DF22
:1031100005C0F39490E8F912E3CFF6CF26960FB6E8
:10312000F894DEBF0FBECDBFDF91CF911F910F91FD
:10313000FF90EF90089586E0ECEBFBE0A3E1B1E1B6
:1031400001900D928A95E1F7089555E05A95F1F7AF
:10315000000036EC31BB469A80EE87B997E09AB909
:103160008DB915B880E488B91BB880E28EB987E4C0
:1031700081BB82E08A95F1F700C026B199B18CB18C
:1031800031BB479A37EE37B937EF3AB932EE3DB92E
:10319000422F4695437050E8259F90011124422B01
:1031A000292F2071422B292F269526952870422BF6
:1031B00096959076492B90E0880F991F84709927F7
:1031C000842B08951092CD0B1092CE0B1092CF0B42
:1031D0001092D00B8FEF8093320C80931C118FEFE5
:1031E0009FEFDC0180931D1190931E11A0931F117E
:1031F000B093201108958F929F92AF92BF92CF9279
:10320000DF92EF92FF920F931F934A015B016801D7
:103210007901BC0180E090E00E94C1739058A50143
:1032200094010E94FC720E946973A70196010E949A
:1032300021750E949573CB011F910F91FF90EF9024
:10324000DF90CF90BF90AF909F908F9008950F9395
:103250001F938091091190910A1100E010E42CE174
:1032600035E440E050E86BE376E480959095C3DF69
:103270009093BA108093B9101F910F910895809187
:103280006A0A90916B0A892B90916C0A892B909114
:103290006D0A892B90916E0A892B90916F0A892B68
:1032A0009091700A892B9091710A892B9091720AE2
:1032B000892B9091730A892B9091740A892B909194
:1032C000750A892B9091760A892B9091770A892B20
:1032D0009091780A892B9091790A982B21E009F432
:1032E00020E08091980B90918D0B892B9091A30BEE
:1032F000892B9091AE0B892B9091820B892B909109
:10330000B90B892B59F48FEF9FEFDC018093B51037
:103310009093B610A093B710B093B8102223A1F0E9
:1033200080917E14811110C08091A4099091A5090B
:10333000A091A609B091A7098093B5109093B610FB
:10334000A093B710B093B81020937E1408950F93F4
:103350001F93CF93DF93EC018A899B8900E01FEFD5
:103360002FE737E440E050E26BE476E480959095F7
:1033700042DFAC0160E070E0088C04C0440F551FD0
:10338000661F771F0A94D2F7488759876A877B8719
:10339000DF91CF911F910F910895CF93DF93EC01AF
:1033A000888D681739F0688FCE01D1DFCE01DF91AB
:1033B000CF910FC8DF91CF910895CF93DF93EC01A8
:1033C000598B488B8A899B896817790749F07B8BD1
:1033D0006A8BCE01BCDFCE01DF91CF910C94E91155
:1033E000DF91CF910895AC01AA27469FB12D579F39
:1033F0009001749FB00D211D3A1F569FB00D211DE5
:103400003A1F1124C9010895A72F8F3FF9F0282FE3
:103410002F5F30E0220F331FE82FF0E0EE0FFF1F89
:10342000E40FF51F60817181FA01E20FF31F8081C3
:103430009181861B970B892F9927A89F9001A99F9F
:10344000300D1124260F371FC90108952EEF31E0EA
:10345000E3CF8FBF0895F89481E008958FBF08955A
:10346000EFE8F7E1A081B1818C9380819181019691
:10347000918380830895EFE8F7E1A081B1818C9377
:10348000808191810196918380830895CF93DF930A
:10349000EFE8F5E180E092E0DF019C011D92215010
:1034A0003040E1F7F0939017E0938F17C1E9D7E12F
:1034B00084E088830E9496118881DF91CF91DBCFD1
:1034C000AFE8B7E1ED91FC91119781939193ED9362
:1034D000FC930895F89481E00895CF93DF93DFB7CC
:1034E000F9DF882309F448C08CE5EDEBF0E1DF015A
:1034F0001D928A95E9F720E030E83093DC102093A4
:10350000DB103093E2102093E1104FEF5FEF509308
:10351000E6104093E5103093EA102093E9105093A1
:10352000F6104093F5105093DA104093D910309371
:10353000061120930511309312112093111130932D
:103540000C1120930B1185E08093D010C1E0C09343
:10355000D110C093CA10C093CC10C093D21082E097
:103560008093D31046E050E06FEF70E083E191E18B
:103570000E947F76C093BD108D2FDF91CF916ECFCB
:10358000CF92DF92EF92FF920F931F93CF93DF932F
:103590001F92CDB7DEB7F82E8B01EFB699839ADF75
:1035A00099818823F1F08F2D0E942C12EFE8F6E12B
:1035B0006F018FE895E1C81AD90A82918823C1F377
:1035C000F092921723E937E1EFE8F5E1A601BF0198
:1035D000C9010E9465769FEFC91AD90AF801D18204
:1035E000C0828E2D0F90DF91CF911F910F91FF9090
:1035F000EF90DF90CF9032CF0F931F93CF93DF9355
:10360000182FEB010FB766DF811104C0802F26DF72
:1036100081E016C0812F992787FD909588539F4F91
:103620000E942C12811108C0802F18DF80E008C092
:103630000E94B211899301C011E8115039F3F8CFFB
:10364000DF91CF911F910F9108951F93CF93DF9337
:10365000EC011FB73FDF811104C0812FFFDEC1E005
:103660005EC0CE010E942C12882309F455C010922E
:10367000CF10109213119FEF909314119093151186
:1036800090931611909317119093181180919117A0
:10369000811102C0C1E041C0C0E00E94BB11EC2F0B
:1036A000F0E0EE0FFF1FE952FF4E91838083CF5F62
:1036B000C93199F7D0E00E94B211ED2FF0E0E35448
:1036C000FF4E8083DF5FD731B1F78091CD108093BB
:1036D000D610809191178230E8F20E94BB11EC2F36
:1036E000F0E0EE0FFF1FE952FF4E91838083CF5F22
:1036F000CE3199F70E94B2118093D4100E94B2117A
:103700008093D510C3E1D1E10E94B211899381E188
:10371000C931D807C9F7A1CFC0E0812F9FDE8C2F18
:10372000DF91CF911F9108951F93CF93DF93182FAF
:10373000DFB7D0DE882309F448C08CE5EDEBF0E17B
:10374000DF011D928A95E9F720E030E83093DC1024
:103750002093DB103093E2102093E1104FEF5FEFE6
:103760005093E6104093E5103093EA102093E9104F
:103770005093F6104093F5105093DA104093D910FF
:1037800030930611209305113093121120931111DB
:1037900030930C1120930B1185E08093D010C1E081
:1037A000C093D110C093CA10C093CC10C093D21054
:1037B00082E08093D31046E050E06FEF70E083E149
:1037C00091E10E947F76111105C08D2FDF91CF917D
:1037D0001F9144CEC093BD10F8CFFF920F931F935B
:1037E000CF93DF93FFB676DE811104C08F2D36DED6
:1037F000C1E064C062E08CED90E00E945312882327
:1038000009F459C08FE380935012109252128091A4
:103810009117882319F0C9E2D1E113C0C1E04CC06F
:103820000E94BB11FE01E00FF11F918380830E5FA8
:103830001F4F04321105A1F7A49682E1C934D807BD
:1038400019F000E010E0ECCF0E94BB1190934C12F5
:1038500080934B120E94BB1190934A12809349129D
:103860000E94B21180934D120E94A91180934E12B2
:1038700080919117823090F20E94B2118093501281
:103880000E94A91180934F1280919117833030F2DA
:103890000E94B2118093511280919117843008F4E4
:1038A000BDCF0E94A911809352128091911785304B
:1038B00008F09CCFB3CFC0E08F2DD0DD8C2FDF91EF
:1038C000CF911F910F91FF900895833061F089315E
:1038D00051F08F3141F091E08F3019F0803109F0D3
:1038E00090E0892F089591E0892F0895BF92CF929B
:1038F000DF92EF92FF920F931F93CF93DF9310927B
:103900007F14C0E0D0E0B4E2BB2E0CC00193119351
:1039100013870287778B668B8150C1F72196C83059
:10392000D10591F16C2F772767FD7095872F972F21
:103930000E94C3736B017C012DEB3EE140EC55E42A
:103940000E94217520E030E44CE955E40E94957214
:103950000E9495738B0121E33CE043E455E4C701E9
:10396000B6010E94217520E030E44CE156E40E944B
:1039700095720E949573BC9EF001BD9EF00D1124BE
:10398000E75DFE4E86E0C2CFDF91CF911F910F9190
:10399000FF90EF90DF90CF90BF900895CF93CFB777
:1039A00099DD8823B1F02AE231E0E9E2F1E1DF01BB
:1039B000C9011D920197E9F720E030E830934A12DF
:1039C000209349128FEF80934E128FE38093501211
:1039D0008DDF8C2FCF9142CD8FBF0895E7E7F4E1C3
:1039E00080818F5F80830895F89481E008958C3FF3
:1039F00059F08138C1F19091030D933039F19091D4
:103A0000040D9330B1F008958091030D8330E9F1F6
:103A10008091040D8330B9F7E091060EEE2399F3FF
:103A2000E150E093060EF0E0EB57F24F8FEF80830A
:103A300008959091060E97FDE6CFE92FF0E0EB5741
:103A4000F24F80839F5F9093060E08959091050E2C
:103A500097FDD5CFE92FF0E0ED5FF24F82839F5FB6
:103A60009093050ECCCF8091030D8330E1F08091CF
:103A7000040D833041F61092060E40E850E06FEFDF
:103A800070E085E89DE00C947F76E091050EEE23D2
:103A900009F4BECFE150E093050EF0E0ED5FF24F88
:103AA0008FEF8283B5CF1092050E40E850E06FEFA4
:103AB00070E085E09DE00E947F76D9CFCF93DF93C1
:103AC000EC016A8F88819981AA81BB81892B8A2B1D
:103AD0008B2B51F46091A4097091A5098091A609DE
:103AE0009091A7090E94E6760E94E3766883798325
:103AF0008A839B83DF91CF9108950F931F93CF9378
:103B0000DF93FC018BE1DF011D928A95E9F707E75E
:103B100012E160E070E080E89FEBC0E0D0E01BC005
:103B2000BE01882777FD8095982F0E94C37321E8F6
:103B300030E840E85BE30E94217520E030E040E897
:103B40005FE30E9495722BED3FE049E450E40E9450
:103B500021750E94F97220E030E040E85FE30E94A6
:103B6000957220E03FEF4FEF56E40E9421750E94CE
:103B70009573F801619371938F012196C115F1E05E
:103B8000DF0771F6DF91CF911F910F9108950F9389
:103B90001F93082F10E0F801E45BFE4F8491F801B9
:103BA000E45BFD4F9491F801E45BFC4F049110E05D
:103BB00020E030E0980111270027192B082BB801CD
:103BC000C9011F910F91089510922D0A10922E0A8B
:103BD00010922A0A1092290A10922C0A10922B0A8B
:103BE0001092330A0895CF93DF9320914E1227FD50
:103BF0000BC06F7070E0332727FD30956217730795
:103C000019F0DF91CF91089580914D128823C9F367
:103C10004436B8F7C42FD0E080914B1290914C12EB
:103C2000C817D90771F3CE0110DD882351F3D09363
:103C30004C12C0934B1210921B110E949855DF91A9
:103C4000CF910C94874E0F931F93CF93DF93CDB7F3
:103C5000DEB7E6970FB6F894DEBF0FBECDBF92E297
:103C6000E8EDF6E0DE01119601900D929A95E1F7EC
:103C7000813019F580914E12992787FD9095029613
:103C800061E170E00E948172815080934E120E9427
:103C9000985580914E12E1E0F0E0EC0FFD1F92E0AC
:103CA0008902E00DF11D112462817381CE0183969A
:103CB0000E94917667EC78E023C0823049F58091CC
:103CC0004F12992787FD9095019660E170E00E9460
:103CD000817280934F120E94985580914F12E1E0BB
:103CE000F0E0EC0FFD1F92E08902E00DF11D1124C0
:103CF00062817381CE0183960E9491766DEC78E0AB
:103D0000CE0183960E948676CE01839601D9C2C0E9
:103D1000833081F48091110C9091120C90934A128F
:103D2000809349120E9498550E94443383ED98E095
:103D3000EFD8B0C08430C9F480917612992787FDFE
:103D40009095019666E070E00E948172182F809332
:103D5000761265EE78E0CE0183960E9491761F5C24
:103D60001DA3CE018396D4D895C08530E1F510917E
:103D7000501200917612212F30E0002E02C03595AE
:103D800027950A94E2F720FF12C069EE78E0CE0191
:103D900083960E94917621E030E0002E01C0220F30
:103DA0000A94EAF7209521232093501210C061EF66
:103DB00078E0CE0183960E94917681E090E0002E1B
:103DC00001C0880F0A94EAF7812B809350120E9459
:103DD0009855809176128F5C8DA3CE01839698D8EA
:103DE0000E94874E57C0863051F40E94066488EFC7
:103DF00098E08ED80E949F4F0E94874E4BC088301B
:103E000011F580915112992787FD9095019663E0F5
:103E100070E00E948172809351120E9498558091A7
:103E20005112813041F0823051F0811131C087E070
:103E300099E06ED82DC080E199E06AD829C08AE166
:103E400099E066D825C08930D1F480915212992723
:103E500087FD9095019662E070E00E9481728093E8
:103E600052120E94985580915212882321F084E2C8
:103E700099E04ED80DC08EE299E04AD809C0811170
:103E800009C02BDB81E080931B1189E399E040D8C6
:103E90000E94874EE6960FB6F894DEBF0FBECDBFE8
:103EA000DF91CF911F910F9108951F93CF93DF93CF
:103EB00000D0CDB7DEB780914E1287FD0EC06F7077
:103EC00070E0992787FD90956817790731F00F907A
:103ED0000F90DF91CF911F910895411138C030911B
:103EE0004D12223008F47DC0332389F3842F805192
:103EF0008E31B0F1842F80558E3108F04CC0E42F04
:103F0000F0E0EE0FFF1FE95CFF4E4081518130E091
:103F1000CA0196958795969587958F7799278217E9
:103F20009307A9F2CA0188279E7F220F331F220F11
:103F3000331F822B932B9183808381E080931B110D
:103F40000F900F90DF91CF911F910C94874E4130CD
:103F500009F460C0403409F46CC030914D12C4CFF4
:103F6000E42FF0E0EE0FFF1FE954FF4E80819181B6
:103F700030E0AC01452F552746954217530709F409
:103F8000A6CF8C7F9170322F2227330F822B932B59
:103F900091838083D2CF842F80538A3108F097CFCA
:103FA000E42FF0E0F09730E0DF01A65FB84F4C91CE
:103FB00087E090E0841B910902C0359527958A958A
:103FC000E2F7822FDF01A354BF4E9C91291709F419
:103FD0004AC02C9311E07197C9F1112309F477CFEE
:103FE000ACCF632F772767FD7095822F90E068171D
:103FF000790709F479CF20934D122A8349830E94CF
:1040000098550E949F4F0E94874E30914D122A81F1
:1040100049816ACF822F880F10928810809389106F
:104020002A8349830E94263230914D122A81498188
:104030005BCF211107C00F900F90DF91CF911F919F
:104040000C944D3E81E08093C50B41CF882369F0ED
:1040500030D886E0ECEBFBE0A3E1B1E101900D92FA
:104060008A95E1F7BACF10E0B6CF06D8F2CF20910B
:104070008F17309190172F5835412130324038F446
:10408000BC0180E090E04FE855E10C946F55089535
:10409000FF920F931F93CF93DF938C01FFB61ADA31
:1040A000882309F438C0F2D9C0E0EC2FF0E0EE0F1D
:1040B000FF1FE952FF4E8081918102DACF5FC93143
:1040C000A1F78091D6108093CD10D0E0ED2FF0E0D5
:1040D000E354FF4E8081CFD9DF5FD731B9F7EC2FA2
:1040E000F0E0EE0FFF1FE952FF4E80819181E8D989
:1040F000CF5FCE31A1F78091D410BDD98091D5107A
:10410000BAD9C3E1D1E18991B6D981E1C931D807E2
:10411000D1F7C801ACDF8F2DDF91CF911F910F91A7
:10412000FF909CC9609127118A3030F5681305C053
:10413000862F865F8093271114C0462F552747FD91
:104140005095282F332727FD3095265F3F4F421784
:10415000530729F4862F8A508093271102C0809339
:1041600027118FEF9FEFDC0180932311909324118F
:10417000A0932511B093261180912711861749F03D
:104180000E94783480914D12811103C08BED90E034
:104190007FCF0895FF920F931F93CF93DF93F82E55
:1041A000EB010FB797D9882371F070D911E802C0DD
:1041B000899161D91150E1F78F2D992787FD90954D
:1041C00088539F4F54DF802FDF91CF911F910F9124
:1041D000FF9044C9BF92CF92DF92EF92FF920F936C
:1041E0001F93CF93DF93B62E082F112707FD10954D
:1041F000E801CD5FD24F9881691761F0992329F1C9
:10420000933009F44EC0923009F45DC082E0B816D4
:1042100059F0B882DF91CF911F910F91FF90EF90ED
:10422000DF90CF90BF900895F801EE0FFF1FE95F78
:10423000F14F8FEF9FEF918380838FEF9FE79093F4
:104240000F0E80930E0EB882E5CF7801F694FE2C07
:10425000EE24F794E79445E0C42E4DE0D42ECE0C26
:10426000DF1CB601C9D9882331F1FE01EE5FFE4F94
:1042700080E88083F701EC57F24F80818F3F31F661
:10428000DE01AE5FBE4F8FE78C93F701EC57F24F24
:104290008EE792919F3F09F0B9CF8C938150C8F778
:1042A000B5CFB8017695762F6627779567956B5FC2
:1042B000724F70DFABCF40E850E06FEF70E0C601A7
:1042C0000E947F76D2CF60E00E9480489FCFCF933C
:1042D000DF93DFB789DB882309F472C007DB0E9414
:1042E000965660E080E090E00E94A02EC2E18C2F04
:1042F0000E944C2E8C2F86500E94812ECF5FC83199
:10430000B1F781E00E94232E60E08FEF9FEF0E94C3
:10431000962E60E080E090E00E948C2EC0E06C2F32
:104320006E5E8C2F0E94633DCF5FC630C1F780E088
:104330000E94232E81E00E941B2E60E080E090E02E
:104340000E94962E60E08FEF9FEF0E948C2E6C2FC4
:10435000645F8C2F0E94633DCF5FCC30C1F780E05B
:104360000E941B2E60E080E090E00E94962E60E0AC
:1043700080E090E00E948C2E60E08FEF9FEF0E9423
:10438000A02E8C2F0E944C2ECF5FC231D1F7CCE0F3
:104390006C2F6A5F8C2F0E94633DCF5FC231C1F7E3
:1043A00060E080E090E00E94A02E8C2F0E944C2EB6
:1043B000CF5FC831D1F70E94033A06DC0E949855BE
:1043C0008D2FDF91CF9108CB0F931F93CF93DF9366
:1043D000182FEB010E94204F209709F04BC112319A
:1043E00091F575DF30C081E0113109F080E0E82FF0
:1043F000F0E0ED5FF24F9081913001F128F09230C2
:1044000001F1933001F512C090911911923031F4FD
:1044100063E0E0DE85E08093191115C090912811CA
:10442000992311F061E00EC062E00CC091E0209190
:104430004D12211101C090E09093191162E0CADE83
:1044400002C060E0C7DE8091030D811104C080913D
:10445000040D8823E1F0209709F443C01D3009F0D2
:104460000FC181E09091040D911101C080E0E82F0F
:10447000F0E0ED5FF24F9081933011F462E001C003
:1044800063E0A8DE85E08093191101E02BC000E015
:10449000209741F19091020D1A3049F481E091305A
:1044A00009F480E06091010D0E9442481BC01B305E
:1044B000C9F4923081F018F09330A1F406C06091F5
:1044C000010D83E00E9442480DC06091010D82E021
:1044D0000E94424807C06091010D80E00E9442485E
:1044E00001C000E08091020D882379F0209709F443
:1044F000CDC01D3009F0C6C061E09091010D911151
:1045000060E00E94424801E02DC0173289F42097F4
:1045100019F00E94591802C00E943C180E949B1872
:1045200080914D1281111BC08BED90E0B1DD17C061
:10453000209789F01E3079F480914D12882391F0F4
:1045400080911911882319F0109219110BC081E084
:104550008093191107C01F3011F4C0932811CD2B7F
:1045600009F482C08091B80980FF03C0812F6BDB02
:104570007BC01C30A9F480914D12811103C08BEDDA
:1045800090E086DD81E090914D12911180E0809362
:104590004D120E9498550E949F4F0E94874E64C002
:1045A000909119111D30B1F4011114C0923011F025
:1045B000943061F481E090914D12911101C080E03E
:1045C000809319118FEF80931A114EC082E080936F
:1045D00019114AC0953021F4812F0E942F2C44C01C
:1045E000911103C0812F9EDD3FC01A3008F03CC0FE
:1045F000923069F018F49130B9F503C09530A0F508
:104600000CC010931A1183E0809319112DC01093E0
:104610001A1184E08093191127C080911A112AE0A1
:10462000829F100D1124812F10931A11943021F4C0
:10463000992787FD90952CDD80911A11992787FD88
:10464000909503D8882359F080911A11992787FDF6
:10465000909590934C1280934B120E9498558FEF37
:1046600080931A110E949F4FDF91CF911F910F915C
:104670000C94874E812F8051823008F0E4CEB3CE67
:1046800000E008CF173209F055CF43CF173209F0B9
:1046900062CF42CF99CE2F923F924F925F926F920C
:1046A0007F928F929F92AF92BF92CF92DF92EF92C2
:1046B000FF920F931F93CF93DF93CDB7DEB763972E
:1046C0000FB6F894DEBF0FBECDBF3FB6F894882377
:1046D00009F434C1912CA92CAA0CAA0CAA0CB6EC92
:1046E0008B2E1FE7E12EF12C8E01055F1F4F81BA43
:1046F000469A992D990F292F26702064892F880FAB
:104700008072907C892B992D9695927031E035B905
:1047100028B98BB99EB987E881BB8DE08A95F1F7FE
:10472000000081BA469A80EE87B997E09AB98DB9B0
:1047300035B980E488B91BB88EB987E481BBE2E063
:10474000EA95F1F700C046B199B18CB181BA479AA8
:10475000242F26952370F0E84F9FA0011124242BCD
:10476000392F3071232B392F369536953870232BFE
:1047700096959076292B90E0880F991F8470992741
:10478000282B87EE87B987EF8AB982EE8DB9BA2CCC
:1047900030E068ED762E7A0C70EC472E4A0CCC2473
:1047A000CA94EFE7DE2EFAE05F2EA8EA6A2E6A0CC2
:1047B00007C08250808326953F5FB394383011F153
:1047C000EB2DF0E0E755F64F8081982F9E7F89F71B
:1047D000922F91708170981771F3892F8A6080836E
:1047E0008FE38B1580F1692F772767FD70958B2DEF
:1047F0002A8B3B8B4FDF2A893B8926953F5FB394F9
:104800003830F1F69394E8E0AE0EFFE0F91508F0C9
:104810006ECF3FBE63960FB6F894DEBF0FBECDBF1E
:10482000DF91CF911F910F91FF90EF90DF90CF908C
:10483000BF90AF909F908F907F906F905F904F90C0
:104840003F902F900895492F552747FD509580910F
:104850002811882361F1452B09F4ADCFEAEFF6E08A
:10486000DE011196852D01900D928A95E1F7F801F0
:1048700086E011928A95E9F7862D830F8093BC100C
:1048800080930B0E8093FB0C4AE050E0BE01665F04
:104890007F4F992787FD90952A8B3B8B0E94EF765F
:1048A000CE0101960E9488172A893B8984CF272C44
:1048B000230E452B11F55091020D511142C08091EC
:1048C000BC1040E050E8692F820D2A8B3B8B998BFE
:1048D0000E947E3F8091BC10820D99892A893B8974
:1048E000911152C040E4682F80914F122A8B3B8B6C
:1048F0000E942A132A893B895ECF8091030D813063
:1049000009F463C08091040D813009F46AC05091AC
:10491000020D511116C08091030D833021F080915A
:10492000040D833061F6822D2A8B3B8B998B5FD8E7
:104930000E945F3599893B892A89C1CF08E0902E72
:10494000CACE442D430F992331F1A8E7BCE0FD0105
:1049500005C08CE0E83FF80709F49CC081918F3FC7
:10496000C1F3513009F489C080E090E005C00196A0
:104970008038910509F41FCF5D915F3FC1F7FC01BD
:10498000E858F34F408317CF60E070E80E9411139E
:104990002A893B8910CF8091010D882369F151301C
:1049A00009F45BC0E8E7FCE080E090E005C0019618
:1049B0008038910509F4FFCE51915413F8CFFC01D2
:1049C000E858F34F40684083F6CE62E080E02A8BDF
:1049D0003B8B998BFFDB0E945F3599893B892A8944
:1049E00091CF62E02A8B3B8B998BF4DB0E945F3581
:1049F0002A893B8999898BCF513011F1E8E7FCE096
:104A000080E090E004C001968038910541F051911A
:104A10005413F9CFFC01E858F34F8FEF8083E8E798
:104A2000FCE081918F3F09F0C6CE8CE0E83FF807AB
:104A3000C1F72A8B3B8B0E940E482A893B89BBCE4B
:104A400050E0FA01E858F34F8FEF8083F701E41B41
:104A5000F50BE858F34F8083E2CF50E0FA01E858B5
:104A6000F34F808180688083F701E41BF50BE858E1
:104A7000F34F8081806880839ECE842F90E0FC017C
:104A8000E858F34F4083F701E81BF90BE858F34F60
:104A9000408391CE80915112811163CFD092FE0C50
:104AA000C092FD0C5ECF96EC91BB469A982F9695DE
:104AB000969596958295880F807E95B990E498B9E1
:104AC0001BB88EB987E881BB85E08A95F1F70000B5
:104AD000089536EC20EE97E0A0E8F7E4E7EE77EFF4
:104AE00062EE5FB7F89431BB469A27B99AB92DB9EF
:104AF00015B8A8B99BB91EB8F1BB42E04A95F1F7C9
:104B000000C046B1B9B1BCB131BB479AE7B97AB977
:104B10006DB95FBF55E05A95F1F7000042FFE1CF54
:104B20005FB7F89496EC91BB469A382F330F982FC5
:104B30009695232F26702068482F441F4427441F32
:104B4000242B80718360432F440F4072842B307C70
:104B5000832B9270906215B828B98BB99EB987E8FB
:104B600081BB85E08A95F1F700005FBF089526ECD0
:104B700090EE87E0F0E8E7E477EE67EF52EE4FB7AC
:104B8000F89421BB469A97B98AB99DB915B8F8B976
:104B90008BB91EB8E1BB32E03A95F1F700C036B1EF
:104BA000A9B1ACB121BB479A77B96AB95DB94FBF1A
:104BB00045E04A95F1F7000032FFE1CF8FB7F89456
:104BC00096EC91BB469A15B892E898B993EC9BB9CC
:104BD00090E29EB997E891BB95E09A95F1F70000B5
:104BE0008FBF089526EC90EE87E0F0E8E7E477EEDB
:104BF00067EF52EE4FB7F89421BB469A97B98AB93E
:104C00009DB915B8F8B98BB91EB8E1BB32E03A9539
:104C1000F1F700C036B1A9B1ACB121BB479A77B961
:104C20006AB95DB94FBF45E04A95F1F7000032FF20
:104C3000E1CF8FB7F89496EC91BB469A15B894E8FB
:104C400098B993E19BB992E29EB997E891BB95E040
:104C50009A95F1F700008FBF089526EC90EE87E05B
:104C6000F0E8E7E477EE67EF52EE4FB7F89421BB38
:104C7000469A97B98AB99DB915B8F8B98BB91EB8D3
:104C8000E1BB32E03A95F1F700C036B1A9B1ACB161
:104C900021BB479A77B96AB95DB94FBF45E04A95DC
:104CA000F1F7000032FFE1CF8FB7F89496EC91BB9B
:104CB000469A15B892E898B993E09BB990E29EB9EC
:104CC00097E891BB95E09A95F1F700008FBF0895A2
:104CD00026EC90EE87E0F0E8E7E477EE67EF52EE3F
:104CE0004FB7F89421BB469A97B98AB99DB915B8C0
:104CF000F8B98BB91EB8E1BB32E03A95F1F700C0C4
:104D000036B1A9B1ACB121BB479A77B96AB95DB9DF
:104D10004FBF45E04A95F1F7000032FFE1CF9FB762
:104D2000F89486EC81BB469A15B887E888B923EDDC
:104D30002BB922E22EB981BB85E08A95F1F70000FC
:104D40009FBF0895CF93DF93E6ECFBE08081C8EC32
:104D5000DBE0688190E070E00E948172A091C90B55
:104D6000B091CA0BA80FB91F2C913FB7F89480815E
:104D700090E00196688170E00E94817280833FBF5D
:104D8000822FDF91CF91A5CECF93DF930E94A518FC
:104D9000C82FD0E00E94A518382F20E0C22BD32BBB
:104DA00081E081DE81E07FDE86EC81BB469A15B82A
:104DB00082E488B91BB880E48EB987E881BB85E0BE
:104DC0008A95F1F7000082E06EDEC095D095CE01A5
:104DD000DF91CF910895CF93882339F180912F0AE5
:104DE0008F5F80932F0A853148F081E09091300ADF
:104DF0009111CDC08093300A10922F0AC091330ACE
:104E0000C11179C050912D0A90912E0AE091340A77
:104E1000E13009F4DEC008F4AFC0E23009F4C4C0E8
:104E200020E0F0E0E75DF54F2487AFB7F89456EC4B
:104E300051BB469A41E045B980E488B91BB880E28D
:104E40008EB937E831BB00C000C080E190E000902F
:104E5000340A02C0880F991F0A94E2F7282F51BB29
:104E6000469A782F770F682F6695221F2227221FD8
:104E7000972F9670292B20648071972F990F90722D
:104E8000982B707C972B627045B928B99BB96EB985
:104E900031BB00C000C0E091340AF0E0E75DF54F9F
:104EA000848551BB469A582F550F982F9695252FDC
:104EB00026702064682F661F6627661F262B682FC2
:104EC0006071852F880F8072862B507C852B9270A5
:104ED000906245B928B98BB99EB931BBAFBF8091FB
:104EE000340A90E0019663E070E00E948172809342
:104EF000340ACF9108954091310A4F5F4093310AAF
:104F0000E8E3FAE001900020E9F7E953FA40209144
:104F1000320A332727FD3095C90101966E2F772776
:104F200067FD70950E948172F901E75DF54F278555
:104F300030E02038310588F15FEFE82FFF27E7FDEB
:104F4000F095E75DF54F278530E02038310550F5C5
:104F5000F901E45EFE4F9081403108F457CF809311
:104F6000320A1092310A811151CF1C160CF04ECF2B
:104F7000C150C093330A4ACF2091290A8091300A48
:104F8000882309F44ECF80912B0A28274ACF80E04E
:104F90008093300A10922F0A31CFF901E45EFE4F60
:104FA0005081CBCF9FEFD8CF292F2F778091290A1F
:104FB00090912A0A90FD206880912B0A90912C0AEA
:104FC00090FF2FCF8091300A882309F42ACF2058F0
:104FD00028CF252F2F778091290A90912A0A91FDB9
:104FE000206880912B0A90912C0A91FF1ACFEACF6A
:104FF000CF9380912F0A8F5F80932F0A853148F0DD
:1050000081E09091300A9111D3C08093300A1092C0
:105010002F0AC091330ACC2309F441C04091310AD0
:105020004F5F4093310AE8E3FAE001900020E9F78E
:10503000E953FA402091320A332727FD3095C90100
:1050400001966E2F772767FD70950E948172F90196
:10505000E75DF54F278530E02038310508F4A3C01F
:105060005FEFE82FFF27E7FDF095E75DF54F278518
:1050700030E02038310508F09DC0F901E45EFE4FB4
:105080009081403180F08093320A1092310A811170
:105090000AC01C1644F4C150C093330A04C0509196
:1050A0002D0A90912E0AE091340AE13009F499C05A
:1050B00008F46EC0E23009F47FC020E0F0E0E75D64
:1050C000F54F2487AFB7F89456EC51BB469A41E0B0
:1050D00045B980E488B91BB880E28EB937E831BBA6
:1050E00000C000C080E190E00090340A02C0880F48
:1050F000991F0A94E2F7282F51BB469A782F770F11
:10510000682F6695221F2227221F972F9670292B22
:1051100020648071972F990F9072982B707C972B39
:10512000627045B928B99BB96EB931BB00C000C0E7
:10513000E091340AF0E0E75DF54F848551BB469A73
:10514000582F550F982F9695252F26702064682F7D
:10515000661F6627661F262B682F6071852F880FB4
:105160008072862B507C852B9270906245B928B94D
:105170008BB99EB931BBAFBF8091340A90E00196E4
:1051800063E070E00E9481728093340ACF910895A9
:105190002091290A8091300A882309F48FCF8091C9
:1051A0002B0A28278BCFF901E45EFE4F508159CF9F
:1051B00080E02BCF9FEF65CF292F2F778091290A91
:1051C00090912A0A90FD206880912B0A90912C0AD8
:1051D00090FF74CF8091300A882309F46FCF205854
:1051E0006DCF252F2F778091290A90912A0A91FD62
:1051F000206880912B0A90912C0A91FF5FCF8091BB
:10520000300A882309F45ACFEACF86EC81BB469A4C
:1052100015B896E898B993E09BB91EB897E891BB8A
:10522000EFE9FFE03197F1F700C0000081BB469A3B
:1052300015B823E828B923E12BB922E02EB991BB98
:10524000FAE0FA95F1F700C081BB469A20EE27B943
:1052500097E09AB92DB915B820E828B99BB91EB8BE
:1052600097E491BB92E09A95F1F700C096B199B19D
:105270009CB181BB479A87EE87B987EF8AB982EEE6
:105280008DB9EAE0EA95F1F700C0089526EC90EEBA
:1052900087E0F0E8E7E477EE67EF52EE4FB7F89477
:1052A00021BB469A97B98AB99DB915B8F8B98BB997
:1052B0001EB8E1BB32E03A95F1F700C036B1A9B1B2
:1052C000ACB121BB479A77B96AB95DB94FBF45E028
:1052D0004A95F1F7000032FFE1CF8FB7F89496ECD2
:1052E00091BB469A15B891E898B993ED9BB990E2B5
:1052F0009EB997E891BB95E09A95F1F700008FBFB2
:1053000008950F931F93CF93DF9380E492E4AFE06F
:10531000B0E036EC20EE17E0D1E0C0E4F0E2E7E4E4
:1053200077EE67EF52EE04C00097A105B10521F1B9
:1053300031BB469A27B91AB92DB9D5B9C8B91BB826
:10534000FEB9E1BB42E04A95F1F700C046B109B1B0
:105350000CB131BB479A77B96AB95DB90197A10918
:10536000B10942FDE1CF892B8A2B8B2B29F0DF91EC
:10537000CF911F910F910895DF91CF911F910F91C0
:105380000C94EE1C80915112813009F00895683F11
:10539000E9F06A3FD9F78FEF9FEF9093080E809363
:1053A000070E2FEF3FE730930F0E20930E0E9093D2
:1053B0000A0E8093090E9093F90C8093F80C3093A9
:1053C000FE0C2093FD0C1092BB1008958091BB1031
:1053D0008F5F8093BB1008951F93CF93DF93D82FD7
:1053E000D86F86958695869528E030E001C0220F1B
:1053F0008A95EAF7C22FC095CD231FB7F894CB0149
:105400000E94CE12E6ECE1BB469A3D2F330F367078
:1054100031649D2F96959270906A71E075B938B994
:10542000A0EFABB99EB967E861BB85E08A95F1F75B
:105430000000E1BB469AFC2FFF0F4C2F46955C2FD6
:10544000551F5527551F8F2F8670582B5064C071DC
:105450008F2F880F80728C2BF07C8F2B4270406ACC
:1054600075B958B98BB94EB961BB8AE08A95F1F725
:1054700000C0E1BB469A75B938B9ABB99EB961BBFA
:105480008AE08A95F1F700C01FBFDF91CF911F918D
:1054900008950F931F93CF93DF9380E492E4AFE0DE
:1054A000B0E036EC20EE17E0D1E0C0E4F0E2E7E453
:1054B00077EE67EF52EE04C00097A105B10521F128
:1054C00031BB469A27B91AB92DB9D5B9C8B91BB895
:1054D000FEB9E1BB42E04A95F1F700C046B109B11F
:1054E0000CB131BB479A77B96AB95DB90197A10987
:1054F000B10942FFE1CF892B8A2B8B2B29F0DF9159
:10550000CF911F910F910895DF91CF911F910F912E
:105510000C94EE1C1F93CF93DF9380E492E4AFE0F2
:10552000B0E036EC20EE17E0D1E0C0E4F0E2E7E4D2
:1055300077EE67EF52EE04C00097A105B10519F1AF
:1055400031BB469A27B91AB92DB9D5B9C8B91BB814
:10555000FEB9E1BB42E04A95F1F700C046B149B15E
:105560004CB131BB479A77B96AB95DB90197A109C6
:10557000B10941FDE1CF892B8A2B8B2B21F0DF91E3
:10558000CF911F910895DF91CF911F910C94EE1C44
:105590001F93CF93DF9380E492E4AFE0B0E036EC6A
:1055A00020EE17E0D1E0C0E4F0E2E7E477EE67EF49
:1055B00052EE04C00097A105B10519F131BB469A1E
:1055C00027B91AB92DB9D5B9C8B91BB8FEB9E1BB0D
:1055D00042E04A95F1F700C046B149B14CB131BB48
:1055E000479A77B96AB95DB90197A109B10941FF35
:1055F000E1CF892B8A2B8B2B21F0DF91CF911F914B
:105600000895DF91CF911F910C94EE1C2F923F9241
:105610004F925F926F927F928F929F92AF92BF92C2
:10562000CF92DF92EF92FF920F931F93CF93DF936E
:10563000CDB7DEB728970FB6F894DEBF0FBECDBF4B
:105640008D832FB72E83F894282F259525952595A2
:10565000259580E290E002C0959587952A95E2F71E
:105660009D819F70982B86EC81BB469A492F440FF1
:10567000292F2695392F331F3327331F842F867008
:10568000382B30649071842F880F8072892B407C76
:10569000842B2270206491E095B938B98BB92EB96A
:1056A00087E881BB35E03A95F1F700002D8133277B
:1056B00027FD30953A832983F901EC5DF84FC080CE
:1056C000D12C80E190E08C199D092FEF3FEF082E3F
:1056D00002C0369527950A94E2F702C0220F331FC5
:1056E0008A95E2F73C832B83E12CF12C00E010E853
:1056F0002FEF3FEF56ECA52E60EEB62E77E0272E6B
:1057000033243394E0E44E2EF0E25F2EA7E46A2EB9
:10571000B7EE7B2E87EF882E92EE992E0AC0200FCF
:10572000311F16950795AFEFEA1AFA0ACE14DF0477
:1057300034F1C9012F8338870E94CE1282E08A9506
:10574000F1F700C0A1BA469AB7B82AB8BDB835B8C3
:1057500048B81BB85EB861BA92E09A95F1F700C0FC
:1057600086B189B19CB1A1BA479A77B88AB89DB879
:105770002F81388585FDD3CF201B310BD2CF86EC0E
:1057800081BB469A81E085B987E488B980EF8BB9FF
:1057900082E48EB987E881BBB5E0BA95F1F70000E5
:1057A000EB81FC812E233F23E981FA81EE0FFF1F5D
:1057B000EF50F44F31832083232F3327E981FA817F
:1057C000E353F44F848190E0821B930B97FD1DC03F
:1057D000059704F53E813FBF28960FB6F894DEBFCB
:1057E0000FBECDBFDF91CF911F910F91FF90EF9032
:1057F000DF90CF90BF90AF909F908F907F906F90F1
:105800005F904F903F902F900895919581959109C9
:10581000059704F3248381E090E0A0E0B0E00D80E0
:1058200004C0880F991FAA1FBB1F0A94D2F740918A
:10583000CD0B5091CE0B6091CF0B7091D00B842B80
:10584000952BA62BB72B8093CD0B9093CE0BA093CB
:10585000CF0BB093D00B2D812093320CBBCF909106
:10586000030D933021F09091040D9330E9F48130D1
:10587000C1F028F0823079F08330B1F406C081E9BC
:1058800099E00E94881781E80DC087E999E00E949D
:1058900088178EEF07C08CE999E00E9488178DEF7A
:1058A00001C08CEF0C94F71C0895CF92DF92EF9219
:1058B000FF92CF939091BF102091C210992309F4C9
:1058C00094C04091DB105091DC1060E070E0222326
:1058D00009F485C0C090E110D090E210E12CF12CC9
:1058E0008823A1F0992381F08091C81085FD0CC018
:1058F0008091201090912110AA2797FDA095BA2F92
:10590000480F591F6A1F7B1F211174C0CFB7F8942D
:105910004115510521E06207710524F04FEF5FEF5B
:1059200060E070E0DB01CA0177FD79C00E94CE1211
:1059300046EC41BB469A31E035B921E428B950EF35
:105940005BB992EA9EB987E881BB00C000C041BB49
:10595000469A35B928B960E76BB99EB981BB00C0DA
:1059600000C041BB469A35B928B95BB99EB981BB25
:10597000D701C601C114D10421E0E206F10424F0EC
:105980008FEF9FEFA0E0B0E0B7FD45C00E94CE12C0
:1059900046EC41BB469A31E035B927E428B950EFCF
:1059A0005BB992EA9EB987E881BB00C000C041BBE9
:1059B000469A35B928B960E76BB99EB981BB00C07A
:1059C00000C041BB469A35B928B95BB99EB981BBC5
:1059D000CFBFCF91FF90EF90DF90CF900895CC2470
:1059E000CA94DC2CE12CF12C7BCF4FEF5FEF60E011
:1059F00070E06DCF8091C81084FD88CF8091201019
:105A000090912110AA2797FDA095BA2FC80ED91EF4
:105A1000EA1EFB1E7BCF80E090E0DC01B7CF80E088
:105A200090E0DC0183CF8095909179148923809355
:105A3000791496EC91BB469A482F440F282F26954F
:105A4000382F331F3327331F942F9670392B306430
:105A50008071942F990F9072982B407C942B227018
:105A6000206C81E085B938B99BB92EB987E881BB34
:105A700085E08A95F1F70000809178148F5F80931C
:105A8000781408958091791480618093791496EC4C
:105A900091BB469A382F330F982F9695282F221FA7
:105AA0002227221F832F8670282B2064832F880FA4
:105AB00080728061307C832B9270906C31E035B9BC
:105AC00028B98BB99EB987E881BB85E08A95F1F743
:105AD0000000809178148F5F8093781408958091EE
:105AE000791481608F7E8093791496EC91BB469AED
:105AF000382F330F982F9695881F8827881F232FBC
:105B00002670822B8064232F220F2072307C232B5F
:105B10009270906C31E035B988B92BB99EB987E89D
:105B200081BB85E08A95F1F70000809178148F5F42
:105B300080937814089530917914832F88608E7F34
:105B40008093791496EC91BB469A282F220F982FB8
:105B50009695881F8827881F422F4670842B806463
:105B6000207C30713062232B9270906C31E035B91B
:105B700088B92BB99EB987E881BB85E08A95F1F792
:105B80000000809178148F5F80937814089540917D
:105B90007914242F22602093791486EC81BB469AD5
:105BA000322F330F922F9695221F2227221F832FE9
:105BB0008670282B2064832F880F80724071842B7D
:105BC000307C832B9270906C31E035B928B98BB959
:105BD0009EB987E881BB85E08A95F1F70000809146
:105BE00078148F5F8093781408954FB7F89480915C
:105BF000770C96EC91BB469A382F330F982F9695D9
:105C0000232F26702064582F551F5527551F252BED
:105C1000582F5071832F880F8072852B307C832BF7
:105C20009270906631E035B928B98BB99EB987E892
:105C300081BB4FBF08959091770C977F8111986039
:105C40009093770CD2CF9091770C9E7F81119160C9
:105C50009093770CCACF9091770C9B7F81119460C1
:105C60009093770CC2CF9091770C9F7B81119064B9
:105C70009093770CBACF9091770C9F7E81119061B1
:105C80009093770CB2CFE82FF0E0EE0FFF1FE95CA6
:105C9000F34F718360830895E82FF0E0EE0FFF1F4C
:105CA000E95CF34F118210820895E82FF0E0EE0FC7
:105CB000FF1FE95CF34F86EC94E99183808308959C
:105CC000E82FF0E0EE0FFF1FE95CF34F83E094E66E
:105CD000918380830895E82FF0E0EE0FFF1FE95CC9
:105CE000F34F82EA9BEB918380830895E82FF0E0E5
:105CF000EE0FFF1FE95CF34F83E99BE591838083FF
:105D00000895E82FF0E0EE0FFF1FE95CF34F8FEFEF
:105D10009FEF91838083089560FD05C090936C0C84
:105D200080936B0C0895BC018AE156CB60FD05C0E1
:105D300090936A0C8093690C0895BC0189E14CCB67
:105D400060FD05C09093740C8093730C0895BC01A2
:105D50008EE142CBFC01623009F43BC018F16330A4
:105D600069F1643011F511A210A2268D378D468994
:105D70005789AA27249FB12D359FC001529FB00D8E
:105D8000811D9A1F349FB00D811D9A1F112482A37B
:105D900093A34089518962897389408351836283C7
:105DA00073830895613009F443C011A210A213A2B5
:105DB00012A21082118212821382089511A210A2DF
:105DC0008689978993A382A31082118212821382FB
:105DD00008952689378944895589AA27429FB12D7C
:105DE000539FC001349FB00D811D9A1F529FB00D6B
:105DF000811D9A1F112480A391A340955095AA2735
:105E0000429FB12D539FC001349FB00D811D9A1F39
:105E1000529FB00D811D9A1F112482A393A3448524
:105E200055856685778540835183628373830895A2
:105E300026893789468D578DAA27429FB12D539FBA
:105E4000C001349FB00D811D9A1F529FB00D811D5E
:105E50009A1F112480A391A340955095AA27429F91
:105E6000B12D539FC001349FB00D811D9A1F529FC9
:105E7000B00D811D9A1F112482A393A340855185E3
:105E800062857385408351836283738308951F9372
:105E9000CF93DF93EC01898D0E94C71D18A5012EB9
:105EA00004C096958795779567950A94D2F724E074
:105EB000660F771F881F991F2A95D1F76887798702
:105EC0008A879B878B8D0E94C71D012E04C09695E3
:105ED0008795779567950A94D2F734E0660F771F18
:105EE000881F991F3A95D1F76C877D878E879F878A
:105EF0008D8D0E94C71D04C09695879577956795EF
:105F00001A95D2F744E0660F771F881F991F4A95AC
:105F1000D1F7688B798B8A8B9B8B69A5CE01DF913A
:105F2000CF911F9117CF0F931F93FC01808D918DFF
:105F30008617970721F0718F608F61E001C060E0E4
:105F4000828D938D8417950719F0538F428F61E0EE
:105F5000848995898217930719F0358B248B61E02A
:105F6000848D958D8017910719F0158F048F02C0CD
:105F7000662321F0CF011F910F9189CF1F910F91BF
:105F80000895FC0160A783CF211107C0BB27A92F6B
:105F9000982F872FBC01CB010895A72FE82F8F3FA3
:105FA000E9F08F5F90E0880F991FF0E0EE0FFF1F80
:105FB000E40FF51F20813181FA01E80FF91F80817C
:105FC0009181821B930B892F9927A89FB001A99FCC
:105FD000700D1124620F731FCB0108958EEF91E0B5
:105FE000E4CFFC011482158216821782108211827E
:105FF0001282138281A58F5F81A7833009F43BC091
:10600000853009F434C0823009F008952689378933
:1060100035A324A344895589AA27429FB12D539FB4
:10602000C001349FB00D811D9A1F529FB00D811D7C
:106030009A1F112480A391A340955095AA27429FAF
:10604000B12D539FC001349FB00D811D9A1F529FE7
:10605000B00D811D9A1F112482A393A344855585F9
:10606000668577854083518362837383089511A683
:1060700015A214A2089511A210A28689978993A34C
:1060800082A30895CF92DF92EF92FF92CF93DF9396
:10609000EC01CC80DD80EE80FF808F2D9927AA2730
:1060A000BB27892B8A2B8B2B09F042C089A5823014
:1060B00009F433C070F5813009F444C040E050E089
:1060C0002AA13BA1AA27429FB12D539FC001349F13
:1060D000B00D811D9A1F529FB00D811D9A1F112472
:1060E00028A139A1820F931F9DA38CA348815981B8
:1060F0006A817B814C0D5D1D6E1D7F1D4C835D8310
:106100006E837F83DF91CF91FF90EF90DF90CF90F0
:1061100008958330A1F0843089F68EA1811122C0C8
:10612000BB27AF2D9E2D8D2DAC0140955095C8CF2E
:10613000CE0157DFCC80DD80EE80FF80B7CF4C8969
:106140005D89BECF8EA1811105C077276F2D5E2D91
:106150004D2DB6CF40EA53E0C701B6010E94041AA4
:10616000AC01AECF40EA51E0C701B6010E94041A6B
:10617000DBCFFF920F931F93CF93DF93EC01F62EAB
:106180001C821D821E821F820E891F896CA17DA127
:10619000CB01A0E0B0E077276627980140E050E00F
:1061A0000E9469773F8F2E8FF11023C084E089A76A
:1061B00019A218A2AA27209FB12D319FC001129FBA
:1061C000B00D811D9A1F309FB00D811D9A1F1124A3
:1061D0008AA39BA388899989AA89BB898883998383
:1061E000AA83BB83FFA2DF91CF911F910F91FF90F4
:1061F000089581E089A7CE01EBD5FFA2DF91CF9171
:106200001F910F91FF900895FC0111A210A2268DFD
:10621000378D46895789AA27249FB12D359FC00104
:10622000529FB00D811D9A1F349FB00D811D9A1F82
:10623000112482A393A34089518962897389408381
:1062400051836283738308958F929F92AF92BF921E
:10625000CF92DF92EF92FF920F931F93CF93DF9332
:10626000EC010C811D812E813F81832F9927AA2764
:10627000BB27892B8A2B8B2B09F054C04A8D6C8548
:106280007D858E859F85433009F473C008F02FC04B
:10629000413009F4B7C0EC89FD89060F171F281F8C
:1062A000391F0C831D832E833F839F0130584889FB
:1062B0005989AA27249FB12D3503C001529FB00DE3
:1062C000811D9A1F34039A0BB00D811D9A1F112452
:1062D0008E8B9F8BDF91CF911F910F91FF90EF904D
:1062E000DF90CF90BF90AF909F908F9008954430F3
:1062F00009F463C0453009F0CECF6801790149E067
:10630000F694E794D794C7944A95D1F7F601DD8ABD
:10631000CC8A498D442309F4C0CFE095F095FD8BDC
:10632000EC8BBBCFE1E0898DE81BE98FE11172C0F6
:10633000C12CD12C7601CC82DD82EE82FF82FF2738
:10634000E1950CF4F095DF01AA0FBB1F119628858B
:1063500039854A855B850E9428776C877D878E8783
:106360009F874A8D41115CC0FD8BEC8B97018601A4
:1063700092CFF12EE22F2F3F09F465C0422F4F5FDD
:1063800050E0440F551FF0E0EE0FFF1FE958FD4E9F
:10639000A081B181FA01E958FD4E408151814A1B2B
:1063A0005B0B452F5527F49EF001F59EF00D11244F
:1063B000EA0FFB1FFD8BEC8B70CF4B8942954F7022
:1063C00088809980AA80BB80FB2D880C991CAA1C10
:1063D000BB1CEF2FEE1FEE27EE1FEF2EE294E6948C
:1063E000A7E0EA22EE25EF27F695EF27E1708E2A47
:1063F000415050F788829982AA82BB82F4019D8A1B
:106400008C8A4BCFC12ED22EE32EFF24F601DD8ADB
:10641000CC8A43CFCC24CA94DC2CEC2CF12C8BCF2F
:10642000423019F0970186012ECF0E94E3767D8BD2
:106430006C8B4A8D6C857D858E859F850C811D8139
:106440002E813F8120CF4EEF51E09DCFCF92DF9242
:10645000EF92FF920F931F93CF93DF938091C7101A
:10646000C82FCC0FC80FCF5F6091C6108AE090E1B3
:106470000E945E1D6C2F8AE090E10E94CD198091F0
:10648000B5109091B610A091B710B091B8108F3F91
:106490002FEF9207A207B20709F49CC020910911BF
:1064A00030910A112115324008F05DC0CFEFDFEFC7
:1064B000E0908810F09089100090D21002C0F694FD
:1064C000E7940A94E2F740910111509102114115AD
:1064D00082E0580708F4ACC09A01325080910D1147
:1064E00090910E119695879596958795811542E026
:1064F000940708F472C08C0112508091D410882344
:1065000009F471C0AE01AA27249FB12D359FC001A7
:10651000529FB00D811D9A1F349FB00D811D9A1F8F
:1065200011246091FF1070910011AC018AE090E19C
:106530000E94DD19C801809590958E159F0508F081
:106540007AC04FEF5FEF60910B1170910C1185E2F3
:1065500090E1DF91CF911F910F91FF90EF90DF902D
:10656000CF900C94DD192091B9103091BA1040E011
:1065700050E0820F931FA41FB51FC090A409D090B4
:10658000A509E090A609F090A709C816D906EA0661
:10659000FB0600F1C090A409D090A509E090A609DF
:1065A000F090A709C81AD90AEA0AFB0AC216D3064C
:1065B000E406F50608F07ACF9E2D8D2D7C2D6627FA
:1065C0000E946977F901EE0FFF1FE056FC4FC08172
:1065D000D1816ECFC0E0D0E06BCF00E010E08091C1
:1065E000D41081118FCFC901809590958E159F058C
:1065F00030F54FEF5FEF6091FF10709100118AE06E
:1066000090E10E94DD199E01AA27029FB12D139FE0
:10661000C001309FB00D811D9A1F129FB00D811DCA
:106620009A1F112460910B1170910C11AC018FCF46
:1066300020E030E053CFA8014E0D5F1D84CFA901AB
:106640004E0D5F1DD8CF80914E1287FD09C06F702F
:1066500070E0992787FD90956817790709F00895EC
:1066600080E8289F90011124242B3052220F331FE1
:10667000220F331F30938B1020938A100E94D11564
:106680006FEF81E00C94D55A4F925F926F927F9298
:106690008F929F92AF92BF92CF92DF92EF92FF9232
:1066A0000F931F93CF93DF938091491290914A12D9
:1066B0009093010180930001C0900401D0900501E6
:1066C0007C01EC18FD08C80ED91EC0910201D091C2
:1066D000030197012C1B3D0B40E050E0812C912CD5
:1066E000A12CF0E8BF2EC501B4010E9469772901F1
:1066F0003A0120930601309307014093080150931B
:1067000009018E010095109598012C193D0940E072
:1067100050E0C501B4010E94697749015A012093F4
:106720000A0130930B0140930C0150930D018091AD
:10673000110C9091120C08171907E0F48FEF9FE7E6
:1067400090938B1080938A100E94D1156FEF81E097
:10675000DF91CF911F910F91FF90EF90DF90CF903D
:10676000BF90AF909F908F907F906F905F904F9071
:106770000C94D55A8C179D07C0F0AC0160E070E016
:106780008E159F0530F0C816D90690F080E090E095
:10679000D7CFCB01BA016C1B7D0B81099109A301F5
:1067A00092010E9466729058CBCF80E090E8C8CFEB
:1067B0009A01AB012C193D0941095109C501B401E8
:1067C0000E94667290589058BBCFCF93DF93CDB79D
:1067D000DEB728970FB6F894DEBF0FBECDBF92E0AC
:1067E0009D8394E09E8397E09F839CE0988795E04B
:1067F000998393E09A8391E09B831C82823081F19C
:1068000034F4882361F0813009F069C013C084300A
:1068100009F450C0D4F1853009F061C05AC0440F6A
:10682000551F661F771F8091C6108170842B80933F
:10683000C61055C08091C8108F7C4130510561054C
:10684000710521F480618093C81049C04230510520
:106850006105710509F001C080628093C8103FC0D6
:10686000DB01CA0181709927AA27BB2721E0822773
:106870008093CC10427055276627772775956795CA
:10688000579547954093D6102AC0DB01CA01817005
:106890009927AA27BB2721E082278093CA1042703C
:1068A00055276627772775956795579547954093A0
:1068B000CB1015C0FE01E40FF51F85818093D01029
:1068C00028960FB6F894DEBF0FBECDBFDF91CF91F3
:1068D000DBCEFE01E40FF51F81818093D210289654
:1068E0000FB6F894DEBF0FBECDBFDF91CF910895F4
:1068F000BF92CF92DF92EF92FF920F931F93CF93AD
:10690000DF93CDB7DEB764970FB6F894DEBF0FBE46
:10691000CDBF009127118CE00802800111240056A0
:106920001A4F0E94E218D80112966D917C9113972C
:10693000CE0101960E94917660EA79E0CE0101963F
:106940000E948676F80180818130D9F020F0823073
:1069500009F05EC029C0E181EE0FFF0BE952FF4E46
:10696000808191819093221180932111A0E0B0E069
:1069700080931D1190931E11A0931F11B0932011AD
:1069800047C0E181FF27E7FDF095E354FF4E80818A
:10699000F801E80FF11DE80FF11D64817581CE014A
:1069A00001960E94867634C08AE1EDEBF0E1A2E91F
:1069B000B7E101900D928A95E1F7C12CD12C7601B7
:1069C000B701A601F801818100DF4AE150E06DEBDB
:1069D00070E182E997E10E945876009771F4F8011E
:1069E0008C2D92E08902E00DF11D112464817581E6
:1069F000CE0101960E9486760BC0AFEFCA1ADA0A62
:106A0000EA0AFA0AB4E0CB16D104E104F104C1F6B3
:106A1000CE0101960E94881764960FB6F894DEBFE7
:106A20000FBECDBFDF91CF911F910F91FF90EF90DF
:106A3000DF90CF90BF900895CF93C82F6C2F86EC36
:106A40009BE00E94525981110FC086EC9BE00E948E
:106A50007D59882399F30E94A2266C2F86EC9BE037
:106A60000E945259882389F3CF910895EF92FF92A3
:106A70000F93CF93DF931F92CDB7DEB77B016115E4
:106A8000710539F40F90DF91CF910F91FF90EF9046
:106A90000895842F2983D0DF298182E0E816F1044C
:106AA00088F3822FC9DFE2E0EE16F10459F3802F5C
:106AB0000F90DF91CF910F91FF90EF90BDCFCF92CC
:106AC000DF92EF92FF920F931F93CF938091030D6C
:106AD000833009F49CC08091040D833009F4B7C061
:106AE00080911911882309F4B4C0813009F4DFC002
:106AF00080911A1187FDD6C060E2805D0E94641704
:106B000060914D1284E00E943D178091191181110E
:106B10005EC061E080914D12882309F458C086E080
:106B20000E943D176091B809617087E00E943D178F
:106B30008091030D41E0823009F467C061E081116A
:106B400001C060E080E00E940E178091040D41E0DA
:106B5000823009F458C061E0811101C060E081E039
:106B60000E940E1761E08091020D813009F060E013
:106B700082E00E943D178091020D41E0823009F0D1
:106B800040E061E0823008F460E083E00E940E178C
:106B90008091020D81111DC08091030D8330C9F0D9
:106BA0008091040D8330A9F08091191161E0823049
:106BB00019F0843009F060E0462F85E0CF911F91F5
:106BC0000F91FF90EF90DF90CF900C940E1760E044
:106BD000A6CF8091010D882359F061E085E0CF9127
:106BE0001F910F91FF90EF90DF90CF900C943D1785
:106BF0008091030D61E0833089F38091040D83302F
:106C000069F360E0EBCF40E0A6CF40E097CF209162
:106C1000040D81E090E0233011F080E090E08D5F82
:106C2000924FFC01EE5FFE4FC0816C2F70E080E060
:106C300090E00E94781741E0C03809F040E061E040
:106C4000C43608F460E089E00E940E1759CF23E0B3
:106C5000E0CF60E089E00E943D1780911D11909186
:106C60001E11A0911F11B0912011B7FD1BC0E09122
:106C70001C11E031E9F12091211130912211A4E69B
:106C8000B0E00E945D776C01FF24D7FCF094EF2CFC
:106C90008E2F0E94651C811118C0C701B6010E9489
:106CA00078172ECF60E280E20E94641729CF6091AE
:106CB0004B1270914C1280E090E00E947817609126
:106CC0001B1189E00E943D171BCF82E3C81AD1082F
:106CD000D7FC2AC0EE24D7FCE094FE2C6091221150
:106CE0006095661F6627661F89E00E943D17D5CF15
:106CF0008091110C9091120CA0910001B0910101B2
:106D0000E0900401F090050160910201709103018F
:106D10009B01209530952817390750F493E6C92E2A
:106D2000D12CE12CF12CB4CFD194C194D108D2CF85
:106D30008617970760F18C0120E030E06D01CE18D6
:106D4000DF088C159D0538F5A9019801261B370B26
:106D50004109510960910601709107018091080174
:106D6000909109010E9466729C013058442737FDBA
:106D70004095542F30584F4F5F4FA4E6B0E00E942B
:106D80001E776C01FF24D7FCF094EF2C81CFC12C2F
:106D9000D12C76017DCFAE0DBF1DA817B90730F0FD
:106DA00082E3C82ED12CE12CF12C72CFA9019801DD
:106DB0002A1B3B0B4109510960910A0170910B019B
:106DC00080910C0190910D010E9466729058CCCF79
:106DD000FC0126893789468D578DAA27429FB12D00
:106DE000539FC001349FB00D811D9A1F529FB00D5B
:106DF000811D9A1F112480A391A340955095AA2725
:106E0000429FB12D539FC001349FB00D811D9A1F29
:106E1000529FB00D811D9A1F112482A393A3408518
:106E2000518562857385408351836283738308959E
:106E30009091810B8091800B2091820B211131C0A8
:106E40002091370F2111EBC120918D0B21116CC0C6
:106E50002091610F211151C12091980B211156C031
:106E600020918B0F2111B7C02091A30B211140C09D
:106E70002091B50F21118AC12091AE0B21112AC09A
:106E80002091DF0F2111F0C02091B90B211114C006
:106E900020910910211156C09093810B8093800B93
:106EA00008952091370F2111CFCF1092820B1092AD
:106EB000840B8FEF9FEFC8CF209109102111ECCFE9
:106EC0001092B90B1092BB0B2FEF2093B80B2093AD
:106ED000B70BE2CF2091DF0F2111D6CF1092AE0B6E
:106EE0001092B00B2FEF2093AD0B2093AC0BCCCFB7
:106EF0002091B50F2111C0CF1092A30B1092A50BBA
:106F00002FEF2093A20B2093A10BB6CF20918B0FD4
:106F10002111AACF1092980B10929A0B2FEF209369
:106F2000970B2093960BA0CF2091610F211194CF46
:106F300010928D0B10928F0B2FEF20938C0B2093C0
:106F40008B0B8ACF1092071010920510109204102C
:106F50001092E40F1092E50F1092E60F1092E70FD7
:106F60001092FF0F1092FE0F109209101092011054
:106F70001092001010920310109202101092E00F65
:106F80001092E10F1092E20F1092E30F10920B0F8C
:106F90001092090F1092080F1092E80E1092E90E4D
:106FA0001092EA0E1092EB0E1092030F1092020F45
:106FB00010920D0F1092050F1092040F1092070FF0
:106FC0001092060F1092E40E1092E50E1092E60E4B
:106FD0001092E70E61CF1092890F1092870F1092D6
:106FE000860F1092660F1092670F1092680F109222
:106FF000690F1092810F1092800F10928B0F1092D8
:10700000830F1092820F1092850F1092840F1092AE
:10701000620F1092630F1092640F1092650F10921E
:107020008D0E10928B0E10928A0E10926A0E109294
:107030006B0E10926C0E10926D0E1092850E1092C7
:10704000840E10928F0E1092870E1092860E109260
:10705000890E1092880E1092660E1092670E109292
:10706000680E1092690E00CF1092DD0F1092DB0FA8
:107070001092DA0F1092BA0F1092BB0F1092BC0F41
:107080001092BD0F1092D50F1092D40F1092DF0FF7
:107090001092D70F1092D60F1092D90F1092D80FCE
:1070A0001092B60F1092B70F1092B80F1092B90F3E
:1070B0001092E10E1092DF0E1092DE0E1092BE0EB4
:1070C0001092BF0E1092C00E1092C10E1092D90EE7
:1070D0001092D80E1092E30E1092DB0E1092DA0E80
:1070E0001092DD0E1092DC0E1092BA0E1092BB0EB2
:1070F0001092BC0E1092BD0EC7CE10925F0F109270
:107100005D0F10925C0F10923C0F10923D0F109289
:107110003E0F10923F0F1092570F1092560F109281
:10712000610F1092590F1092580F10925B0F10922E
:107130005A0F1092380F1092390F10923A0F109286
:107140003B0F1092630E1092610E1092600E10921F
:10715000400E1092410E1092420E1092430E109269
:107160005B0E10925A0E1092650E10925D0E1092E8
:107170005C0E10925F0E10925E0E10923C0E1092FA
:107180003D0E10923E0E10923F0E66CE1092B30F3F
:107190001092B10F1092B00F1092900F1092910FA9
:1071A0001092920F1092930F1092AB0F1092AA0FA1
:1071B0001092B50F1092AD0F1092AC0F1092AF0F4E
:1071C0001092AE0F10928C0F10928D0F10928E0FA6
:1071D00010928F0F1092B70E1092B50E1092B40E3F
:1071E0001092940E1092950E1092960E1092970E89
:1071F0001092AF0E1092AE0E1092B90E1092B10E08
:107200001092B00E1092B30E1092B20E1092900E19
:107210001092910E1092920E1092930E2DCE10920B
:10722000350F1092330F1092320F1092120F1092EE
:10723000130F1092140F1092150F10922D0F109221
:107240002C0F1092370F10922F0F10922E0F1092BA
:10725000310F1092300F10920E0F10920F0F1092EC
:10726000100F1092110F1092390E1092370E1092CB
:10727000360E1092160E1092170E1092180E1092D3
:10728000190E1092310E1092300E10923B0E109289
:10729000330E1092320E1092350E1092340E109260
:1072A000120E1092130E1092140E1092150ECCCDD9
:1072B000EF92FF920F931F93CF93DF937C01EB012B
:1072C000142F40FF09C020917A1430917B14282795
:1072D00039272C7F232B71F511FF0AC080917C1474
:1072E00090917D148C279D2788279E7F892B39F4C8
:1072F000DF91CF911F910F91FF90EF9008950D2F87
:10730000069540914F124F70406BE0919219F091A9
:10731000931921E063E070E082E999E10995D09347
:107320007D14C0937C14DF91CF911F910F91FF903A
:10733000EF90089590589C013595279535952795A0
:10734000092F06952F77332740914F124F70406ECB
:10735000E0919219F091931963E070E082E999E16C
:107360000995F0927B14E0927A14B6CF8091770C55
:107370008E7F9091BD10911181608093770C0E9457
:10738000F52D8091770C877F9091C01091118860C6
:107390008093770C0E94F52D8091770C8D7F9091D2
:1073A000BE10911182608093770C0E94F52D809120
:1073B000770C8F7E9091C110911180618093770C32
:1073C0000E94F52D8091770C8B7F9091C3109111C5
:1073D00084608093770C0E94F52D8091770C8F7DCF
:1073E0009091C410911180628093770C0E94F52DCA
:1073F0008091770C8F7B9091C51091118064809360
:10740000770C0C94F52D6F927F929F92AF92BF9262
:10741000CF92DF92EF92FF920F931F93CF93DF9360
:107420001F92CDB7DEB767E3662E6CE0762E60E084
:1074300008E010E076ECC72EDD24D394E0EFBE2EFA
:10744000F7E8EF2EF301819191913F0158EFF52E6E
:10745000F62A262F269526952695A80102C0440FC8
:10746000551F2A95E2F7942E90949F20AFB6F8947A
:1074700069830E94CE12C1BA469A3F2D330F3670EF
:1074800031649F2D96959270906AD5B838B9BBB883
:107490009EB9E1BA55E05A95F1F70000C1BA469A93
:1074A000792D770F492D4695592D551F5527551F75
:1074B000872F8670582B5064292D2071872F880FB5
:1074C0008072822B707C872B4270406AD5B858B985
:1074D0008BB94EB9E1BA8AE08A95F1F700C0C1BA1A
:1074E000469AD5B838B9BBB89EB9E1BAEAE0EA9590
:1074F000F1F700C0AFBE69816F5F603209F0A2CFC3
:107500000F90DF91CF911F910F91FF90EF90DF903F
:10751000CF90BF90AF909F907F906F900C94F52D7F
:1075200060917F14663028F46F5C81E60E946417D6
:107530000BC06C3028F4655D82E60E94641704C0BD
:107540006B5D86E60E9464170E94F8275CCFCF929D
:10755000DF92EF92FF92CF93C9E1E2DFC150E9F7EA
:1075600010927914109278146AE081E10E949E12C0
:107570000E94C426C0E8C12CD12C76010E94C72DE0
:107580000E949B2D0E9481290E946F2D0E94492AF2
:107590000E94422D0E948A2A80E10E94132D0E949F
:1075A000422D0E94C82A8AE00E94132D0E94C42600
:1075B000C80ED91EE11CF11CB3DF80917714853011
:1075C00050F4C150D9F6B601C701CF91FF90EF90AA
:1075D000DF90CF900895CC24CA94DC2C7601B601BC
:1075E000C701CF91FF90EF90DF90CF900895CF9299
:1075F000DF92EF92FF92CF93C9E192DFC150E9F79A
:1076000010927914109278146AE081E10E949E121F
:107610000E94C4260E94C72D0E949B2D0E94812992
:107620000E946F2D0E94492A0E94422D0E948A2AA0
:1076300080E10E94132D0E94422D0E94C82A8AE0F8
:107640000E94132D0E94C4266C01E12CF12C68DFEE
:1076500080917714853008F002C10E94C72D0E94E6
:107660009B2D0E9481290E946F2D0E94492A0E9411
:10767000422D0E948A2A80E10E94132D0E94422DF1
:107680000E94C82A8AE00E94132D0E94C426C80EB8
:10769000D91EE11CF11C44DF80917714853008F07D
:1076A000DEC00E94C72D0E949B2D0E9481290E944E
:1076B0006F2D0E94492A0E94422D0E948A2A80E151
:1076C0000E94132D0E94422D0E94C82A8AE00E9427
:1076D000132D0E94C426C80ED91EE11CF11C20DF08
:1076E00080917714853008F0BAC00E94C72D0E949F
:1076F0009B2D0E9481290E946F2D0E94492A0E9481
:10770000422D0E948A2A80E10E94132D0E94422D60
:107710000E94C82A8AE00E94132D0E94C426C80E27
:10772000D91EE11CF11CFCDE80917714853008F035
:1077300096C00E94C72D0E949B2D0E9481290E9405
:107740006F2D0E94492A0E94422D0E948A2A80E1C0
:107750000E94132D0E94422D0E94C82A8AE00E9496
:10776000132D0E94C426C80ED91EE11CF11CD8DEC0
:1077700080917714853008F072C00E94C72D0E9456
:107780009B2D0E9481290E946F2D0E94492A0E94F0
:10779000422D0E948A2A80E10E94132D0E94422DD0
:1077A0000E94C82A8AE00E94132D0E94C426C80E97
:1077B000D91EE11CF11CB4DE80917714853008F0ED
:1077C0004EC00E94C72D0E949B2D0E9481290E94BD
:1077D0006F2D0E94492A0E94422D0E948A2A80E130
:1077E0000E94132D0E94422D0E94C82A8AE00E9406
:1077F000132D0E94C426C80ED91EE11CF11C90DE78
:1078000080917714853058F50E94C72D0E949B2DDA
:107810000E9481290E946F2D0E94492A0E94422DB8
:107820000E948A2A80E10E94132D0E94422D0E940C
:10783000C82A8AE00E94132D0E94C426C80ED91EB1
:10784000E11CF11C6DDE80917714853040F4B601A7
:10785000C701CF91FF90EF90DF90CF900895CC2497
:10786000CA94DC2C7601B601C701CF91FF90EF904E
:10787000DF90CF900895CF92DF92EF92FF92CF9357
:10788000DF93D82FC9E14CDEC150E9F7109279148B
:10789000109278146AE081E10E949E120E94C42630
:1078A000C12CD12C760124C00E94C72D0E949B2D93
:1078B0000E9481290E946F2D0E94492A0E94422D18
:1078C0000E948A2A80E10E94132D0E94422D0E946C
:1078D000C82A8AE00E94132DD1500E94C426C80EE7
:1078E000D91EE11CF11C1CDE80917714853058F400
:1078F000D111DACFB601C701DF91CF91FF90EF90A0
:10790000DF90CF900895CC24CA94DC2C7601F2CF7E
:107910002F923F924F925F926F927F928F929F929F
:10792000AF92BF92CF92DF92EF92FF920F931F938D
:10793000CF93DF93CDB7DEB729970FB6F894DEBFAC
:107940000FBECDBF782E662E4A831092771470E05A
:1079500080E090E00E94C1739B01AC0160E070E0A8
:1079600080E090E40E94847524EA30ED42E851E41E
:107970000E9421759B01AC0160E074E284EF99E400
:107980000E94FC726B837C838D839E83262D235003
:1079900081E090E0022E01C0880F0A94EAF7898303
:1079A0001EE0512E00E010E88FEF9FEF9987888747
:1079B000E22FFF27E1950CF4F0954F01AA2497FCE4
:1079C000A094BA2C672D8A810E94151528853985C7
:1079D0008217930760F5B901872D0E94432E898194
:1079E0004ADF6B017C016F3F3FEF7307830793070B
:1079F00009F44FC0C501B4010E94C3739B01AC01DF
:107A000060E070E080E090E40E9484751B01482EE5
:107A10009F83C701B6010E94C1739B01AC01FF8027
:107A2000622D732D842D9F2D0E94217504C06FEF50
:107A30007FEF8FE79FE7BB81AC81ED81FE802B2F2D
:107A40003A2F4E2F5F2D0E94AD7418163CF4888596
:107A50009985800F911F9987888706C0E885F985E9
:107A6000E01BF10BF987E887169507955A9409F002
:107A7000A9CF22E1629EF0011124E70DF11DEE0F66
:107A8000FF1FE75DFE4E888599859183808380E0A6
:107A900001C08FEF29960FB6F894DEBF0FBECDBFA1
:107AA000DF91CF911F910F91FF90EF90DF90CF90DA
:107AB000BF90AF909F908F907F906F905F904F900E
:107AC0003F902F9008950F931F93CF93DF93D82F5C
:107AD000062F80937F14862F0E94812EDC3008F0C1
:107AE00057C013E04CE0612F8D2F12DF811103C0CE
:107AF0001F5F1730B9F7ED2FF0E0DF01AA0FBB1FB2
:107B0000AB56BE4E8D919C919C01220F331FDF011D
:107B1000AA0FBB1FA754BE4E4D915C91241B350B81
:107B2000DF01AA0FBB1FAF58BE4E2D933C93A90196
:107B3000440F551F481B590BDF01AA0FBB1FA35B46
:107B4000BE4E4D935C93440F551FDF01AA0FBB1F20
:107B5000A75DBE4E421B530B4D935C93DF01AA0FF2
:107B6000BB1FAB5DBD4ECF01880F991F8F5F9D4E30
:107B7000EC0128813981220F331FEE0FFF1FE352E2
:107B8000FE4E80819181281B390B2D933C9323C09D
:107B900014E044E2612F8D2FBBDE882341F0ED2FEE
:107BA000F0E0EE0FFF1FE754FE4E44E004C01F5FFD
:107BB000183079F7F4CFDF01949720813181220FBB
:107BC000331F84A195A1281B390B11963C932E934A
:107BD0004150FD0181F7802F0E944C2EDF91CF9103
:107BE0001F910F9110CC882349F086EC9BE00E94F6
:107BF0007D59811101C008950C94A2260E948D59CF
:107C0000F4CFFC01268937892617370721F0778BB7
:107C1000668B0C94472F08950F931F93CF93DF9398
:107C20008B014091071150910811AA27049FB12D93
:107C3000159FB001509FB00D611D7A1F149FB00DAC
:107C4000611D7A1F112440955095640F751F9AE2AB
:107C50008902E0011124CE018E5E914FD2DF409166
:107C6000051150910611AA27049FB12D159FB0014F
:107C7000509FB00D611D7A1F149FB00D611D7A1FBA
:107C8000112440955095640F751FCE01825F904F6F
:107C9000DF91CF911F910F91B4CF1092C50B8091BE
:107CA000C30B80FF04C09091830B911188C081FFAA
:107CB00004C090918E0B911169C082FF04C0909115
:107CC000990B91114AC083FF04C09091A40B9111AC
:107CD0002BC084FF04C09091AF0B91110CC085FFA5
:107CE00009C08091BA0B882329F08091BB0B8823AF
:107CF00009F47EC008959091B00B9111F0CF0E94CD
:107D00003F1964E081E00E94D55A60E08AEB9EE072
:107D10000E94B93060E086EB9FE00E94B93010927B
:107D2000AF0B8091C30BDBCF9091A50B9111D1CFFD
:107D30000E943F1963E081E00E94D55A60E080E92B
:107D40009EE00E94B93060E08CE89FE00E94B9306C
:107D50001092A40B8091C30BBCCF90919A0B911100
:107D6000B2CF0E943F1962E081E00E94D55A60E0E4
:107D700086E69EE00E94B93060E082E69FE00E94C5
:107D8000B9301092990B8091C30B9DCF90918F0BBE
:107D9000911193CF0E943F1961E081E00E94D55A72
:107DA00060E08CE39EE00E94B93060E088E39FE0F1
:107DB0000E94B93010928E0B8091C30B7ECF9091B0
:107DC000840B911174CF0E943F1960E081E00E9402
:107DD000D55A60E082E19EE00E94B93060E08EE01A
:107DE0009FE00E94B9301092830B8091C30B5FCF4C
:107DF0000E943F1965E081E00E94D55A60E084EE60
:107E00009EE00E94B93060E080EE9FE00E94B930B1
:107E10001092BA0B0895AF92BF92CF92DF92EF9279
:107E2000FF920F931F93CF93DF931F92CDB7DEB7CF
:107E3000F82E8B0149830E943F196F2D81E00E942B
:107E4000D55A4981442329F08091020D882309F4F1
:107E500047C08F2D9AE289026001112482E1A82E89
:107E60008EE0B82EAC0CBD1CF50114821582168272
:107E7000178264A175A1CB01A0E0B0E07727662747
:107E80002689378940E050E00E946977F501378FF5
:107E9000268FEE24E394E1A6C5010E94E836F501A1
:107EA000E7A28EE09FE0C80ED91EF601148215826B
:107EB0001682178264A175A1CB01A0E0B0E07727FC
:107EC00066272689378940E050E00E946977F601ED
:107ED000378F268FE1A6C6010E94E836F601E7A299
:107EE000B8018F2D0F90DF91CF911F910F91FF90CF
:107EF000EF90DF90CF90BF90AF908ECE2F923F92B9
:107F00004F925F926F927F928F929F92AF92BF92A9
:107F1000CF92DF92EF92FF920F931F93CF93DF9355
:107F2000882E742E652E86958695869590E0E82D90
:107F3000E770F0E0EC5BF84F2081FC01E659F54F6B
:107F4000662309F4B6C08081822B8083E82DF0E09F
:107F5000EE0FFF1FE658F54F40835183312CC09040
:107F6000A409D090A509E090A609F090A7098091F6
:107F7000C40B882309F405C18091C20B882331F119
:107F8000282D30E0823009F4E5C7813011F40C94DB
:107F9000D84780E090E028173907A1F0E82FE69550
:107FA000E695E695F0E0E659F54F4081442351F01F
:107FB000FC01E770FF27EC5BF84F5081542311F070
:107FC0003324339401968038910529F790E0DCEB57
:107FD000AD2EDBE0BD2E1BE0212E99249394482C7E
:107FE000512C06E010E0E50189915E018F3F09F414
:107FF0004DC0C92FDD27C7FDD0952C9E90012D9E29
:10800000300D11242659354FF901E85EFE4F90825C
:10801000F901E75EFE4F9082F901E65EFE4F908225
:10802000F901EC5EFE4F70826182F901EA5EFE4F5B
:108030008082F901E95EFE4FA201480F511D408385
:10804000F901E05FFE4FC082D182E282F382432DCC
:10805000672D762D892FDFDE4091C30B04C0C92F19
:10806000DD27C7FDD095CE010196B8010E9481722F
:108070009C01982FF901EC5BF84F8081842379F300
:10808000D2ECAD16DBE0BD0609F0ADCFDF91CF91AC
:108090001F910F91FF90EF90DF90CF90BF90AF9026
:1080A0009F908F907F906F905F904F903F902F9018
:1080B000089520958081282320839090820B7090D2
:1080C000800B072D10E0A0908D0BA0918B0BB0E0E2
:1080D000E090980B2091960B30E0F090A30B60910C
:1080E000A10B70E0C090AE0B4091AC0B50E0B09093
:1080F000B90BC091B70B2C2E312C8091C20B823062
:1081000009F49CC280E090E0992009F420C2A110FB
:10811000E2C3B110F2C1D82EE82FE695E695E695B8
:10812000F0E0E659F54FA081AA2309F471C3FC01E0
:10813000E770FF27EC5BF84FE081EA2309F468C39E
:108140000817190709F464C3EE2021F0281739072E
:1081500009F45EC3FF2021F06817790709F458C3BA
:10816000CC2021F04817590709F452C3FC01EE0F47
:10817000FF1FE658F54F708061808D2C33243394B7
:10818000EECEE091C30BCE2FC170E0FF17C08091FF
:10819000820B882309F4E3C280917A0B90917B0BC8
:1081A000A0917C0BB0917D0B8C159D05AE05BF0594
:1081B00028F48091810B881609F408CF4FEF5FEF08
:1081C000BA019FEF8E2F8270E1FF17C020918D0BB7
:1081D000222309F4D5C20091850B1091860B2091C2
:1081E000870B3091880B0C151D052E053F0528F4D3
:1081F00020918C0B821609F40EC724E0A22EAE2229
:10820000E2FF17C03091980B332309F4D5C20091D7
:10821000900B1091910B2091920B3091930B0C15B8
:108220001D052E053F0528F43091970B831609F4A0
:10823000EFC608E0B02EBE22E3FF17C0F091A30BFB
:1082400000919B0B10919C0B20919D0B30919E0BEC
:10825000FF2309F4A7C20C151D052E053F0528F4C0
:10826000F091A20B8F1609F4D0C6AE2FA071E4FFD7
:1082700017C0F091AE0B0091A60B1091A70B2091A7
:10828000A80B3091A90BFF2309F4A8C20C151D05FA
:108290002E053F0528F4F091AD0B8F1609F4B2C6F8
:1082A000BE2FB072E5FF17C0E091B90BEE2309F4C1
:1082B0009FC24091B10B5091B20B6091B30B709182
:1082C000B40B4C155D056E057F0528F44091B80B85
:1082D000841609F49BC29F3F09F079CEC11191C168
:1082E0004FEF5FEFBA018823E1F010918B0BE12F84
:1082F000E695E695E695F0E0E659F54FD081D11187
:1083000086C30091850B1091860B2091870B3091CD
:10831000880B041715072607370718F4B901A801B9
:1083200091E0AA20E1F01091960BE12FE695E695F9
:10833000E695F0E0E659F54FD081D11140C30091A8
:10834000900B1091910B2091920B3091930B04178D
:1083500015072607370718F4B901A80192E0BB20DA
:10836000E1F01091A10BE12FE695E695E695F0E09E
:10837000E659F54FD081D11136C300919B0B109176
:108380009C0B20919D0B30919E0B0417150726071F
:10839000370718F4B901A80193E0AA23E1F010917E
:1083A000AC0BE12FE695E695E695F0E0E659F54F42
:1083B000D081D11122C30091A60B1091A70B20915F
:1083C000A80B3091A90B041715072607370718F4D7
:1083D000B901A80194E0BB23B1F01091B70BE12FD4
:1083E000E695E695E695F0E0E659F54FD081DD2378
:1083F00009F4D5C2E12FE770F0E0EC5BF84FE081C3
:10840000ED2309F4CCC29F3F09F0E1CDE091C20B0E
:10841000CC2309F475C4E13009F4C0C508F026C5C1
:1084200040917A0B50917B0B60917C0B70917D0B8E
:108430004F3FFFEF5F076F077F0709F090E0811163
:108440006AC4F82DAA2009F47BC4E13009F478C588
:1084500008F03EC50091900B1091910B2091920B6A
:108460003091930B041715072607370708F466C5E4
:108470008A019B01B901A801BB2009F46BC40091DA
:108480009B0B10919C0B20919D0B30919E0B041720
:1084900015072607370718F4B901A80193E0AA23A6
:1084A00009F462C40091A60B1091A70B2091A80BB0
:1084B0003091A90B041715072607370708F448C59C
:1084C0008A019B01BB2381F0B901A8010091B10B86
:1084D0001091B20B2091B30B3091B40B0417150718
:1084E0002607370708F492C19F3F09F4CFCD6FCD1F
:1084F00001968038910509F4DAC0D82EE82FE69568
:10850000E695E695F0E0E659F54FA081AA2381F3C0
:10851000FC01E770FF27EC5BF84FE081EA2341F3B1
:108520000817190729F3EE2019F02817390701F366
:10853000FF2019F068177907D9F2CC2019F04817F5
:108540005907B1F22816390609F010CED1CFB11073
:1085500065C1A1102EC0D82EE82FE695E695E695C8
:10856000F0E0E659F54FA081AA23C9F0FC01E770BD
:10857000FF27EC5BF84FE081EA2389F0EE2019F049
:108580002817390761F0FF2019F06817790739F0CB
:10859000CC2009F4EBCD4817590709F0E7CD019637
:1085A00080389105C1F68DC001968038910509F497
:1085B00081C0D82EE82FE695E695E695F0E0E659DD
:1085C000F54FC081CC2381F3FC01E770FF27EC5B02
:1085D000F84FE081EC2341F3A817B90729F3EE2007
:1085E00019F02817390701F3FF2019F068177907E8
:1085F000D9F2CC2009F4BACD4817590709F0B6CD05
:10860000D3CF5091800BE52FE695E695E695F0E007
:10861000E659F54F40814111DCC140917A0B5091F0
:108620007B0B60917C0B70917D0B4F3FEFEF5E07F2
:108630006E077E0709F457CE90E055CEFF2009F46F
:10864000F0C1EE2009F420C2EFE7F0E0A1107BC2F8
:10865000CF01DE2EAE2FA695A695A695B0E0A65921
:10866000B54FFC90FF20F9F0DF01A770BB27AC5B92
:10867000B84FAC91AF21B9F0992019F00E171F0730
:1086800091F02E173F0779F06E177F0761F0CC202D
:1086900019F04E175F0739F0BB2009F467CD2E168D
:1086A0003F0609F063CD319798F6992019F07814B8
:1086B00009F40BC3AA2029F080918B0B881509F4CB
:1086C000B5C38091980B882329F08091960B88156B
:1086D00009F493C38091A30B882329F08091A10B07
:1086E000881509F471C38091AE0B882329F080911D
:1086F000AC0B881509F44FC38091B90B882309F49A
:10870000C5CC8091B70B8811C1CC1092BB0B809166
:10871000C50B8111BBCC1092BA0B0E943F1965E0CA
:1087200081E00E94D55A60E084EE9EE00E94B9305C
:1087300060E080EE9FE0DF91CF911F910F91FF905D
:10874000EF90DF90CF90BF90AF909F908F907F90F1
:108750006F905F904F903F902F900C94B930409164
:108760007A0B50917B0B60917C0B70917D0B4F3F8E
:10877000DFEF5D076D077D0709F423CD90E022CD83
:108780000091850B1091860B2091870B3091880BFF
:10879000041715072607370708F02FCDB901A801E0
:1087A00091E02BCD041715072607370708F05DCD9C
:1087B000B901A80193E059CD0091900B1091910B54
:1087C0002091920B3091930B04171507260737075A
:1087D00008F02FCDB901A80192E02BCD04171507A1
:1087E0002607370708F05CCDB901A80194E058CD01
:1087F0000091B10B1091B20B2091B30B3091B40BDF
:10880000041715072607370708F065CD95E0DFCB7D
:1088100001968038910509F07ECC49CFC1102DC05A
:10882000D82EE82FE695E695E695F0E0E659F54F67
:1088300040814423C1F0FC01E770FF27EC5BF84F57
:108840005081542381F0AA2019F0A817B90759F0D4
:10885000EE2019F02817390731F0F11038C028162A
:10886000390609F083CC019680389105C9F622CFEC
:1088700001968038910509F41DCFD82EE82FE69592
:10888000E695E695F0E0E659F54F1081112381F366
:10889000FC01E770FF27EC5BF84FE081E12341F337
:1088A000AA2019F0A817B90719F3EE2019F0281714
:1088B0003907F1F2FF2019F068177907C9F2481754
:1088C0005907B1F22816390609F050CCD1CF6817F4
:1088D000790729F6C8CFE11034C0D82EE82FE695E5
:1088E000E695E695F0E0E659F54F20812223F9F070
:1088F000FC01E770FF27EC5BF84F30813223B9F0C1
:1089000008171907A1F0A817B90789F0FF2019F077
:108910006817790761F0CC2019F04817590739F02A
:10892000BB2009F423CC2816390609F01FCC019688
:108930008038910591F6BBCE01968038910509F4F7
:10894000B6CED82EE82FE695E695E695F0E0E65906
:10895000F54FE080EE2081F3FC01E770FF27EC5B30
:10896000F84FE081EE2141F38017910729F38A1730
:108970009B0711F382179307F9F2FF2019F086176E
:108980009707D1F2CC2019F084179507A9F2BB20E4
:1089900009F4ECCB8215930509F0E8CBCDCF00911B
:1089A000B10B1091B20B2091B30B3091B40B0417A3
:1089B00015072607370708F026CD95E008CBE12FED
:1089C000E770F0E0EC5BF84FE081ED2309F0C7CCF5
:1089D000B6CC5770E52FF0E0EC5BF84F5081542394
:1089E00009F07ECC1ACEE12FE770F0E0EC5BF84F97
:1089F000E081ED2309F0D1CCC0CCE12FE770F0E0AD
:108A0000EC5BF84FE081ED2309F0E5CCD4CCE12F0D
:108A1000E770F0E0EC5BF84FE081ED2309F081CCEA
:108A200070CC6FE770E0992009F4F9C0A110C8C0BC
:108A3000CB01D62EE62FE695E695E695F0E0E659D1
:108A4000F54FA081AA23E1F0FB01E770FF27EC5B63
:108A5000F84FE081EA23A1F00617170789F0EE200E
:108A600019F02617370761F0CC2019F04617570781
:108A700039F0BB2009F47ACB2616370609F076CBFD
:108A800061507109A8F613CE2FE730E091102CC089
:108A9000C901D22EE22FE695E695E695F0E0E6597B
:108AA000F54F10811123E1F0F901E770FF27EC5B2E
:108AB000F84FE081E123A1F0AA2019F0A217B30733
:108AC00079F06217730761F0CC2019F04217530751
:108AD00039F0BB2009F44ACB2216330609F046CB05
:108AE00021503109A8F6E6CDC901D22EE22FE69534
:108AF000E695E695F0E0E659F54FF080FF20F9F0B5
:108B0000F901E770FF27EC5BF84FE081EF21B9F046
:108B100002171307A1F0AA2019F0A217B30779F0E2
:108B20006217730761F0CC2019F04217530739F030
:108B3000BB2009F41BCB2216330609F017CB2150BA
:108B4000310990F6B4CDCF01DE2EEE2EE694E694F8
:108B5000E694F12CCAE64C2ECAE05C2EE40CF51C1F
:108B6000E7016880662049F1C7E0EC2EF12CEE2287
:108B7000FF22D4E44D2ED7E05D2EE40CF51CE70176
:108B8000F880F620D1F0992019F0E017F107A9F04C
:108B9000EA17FB0791F0E217F30779F0E617F707FA
:108BA00061F0CC2019F0E417F50739F0BB2009F487
:108BB000DDCAE215F30509F0D9CA319720F675CD63
:108BC000CB01D62EE62FE695E695E695F0E0E65940
:108BD000F54FF080FF20F9F0FB01E770FF27EC5B19
:108BE000F84FE081EF21B9F006171707A1F0A6179B
:108BF000B70789F0EE2019F02617370761F0CC206F
:108C000019F04617570739F0BB2009F4AFCA2616EA
:108C1000370609F0ABCA6150710990F648CDB11022
:108C200029C0CB01D62EE62FE695E695E695F0E035
:108C3000E659F54FC081CC23C9F0FB01E770FF274F
:108C4000EC5BF84FE081EC2389F0AA2019F0A6171D
:108C5000B70761F0EE2019F02617370739F0CC205E
:108C600009F484CA4617570709F080CA6150710990
:108C7000C0F620CDCB01D62EE62FE695E695E695FB
:108C8000F0E0E659F54F10811123D9F0FB01E770B0
:108C9000FF27EC5BF84FE081E12399F0AA2019F05F
:108CA000A617B70771F0EE2019F02617370749F01D
:108CB000CC2019F04617570721F02616370609F081
:108CC00055CA61507109B0F6F5CC1092840B8091B1
:108CD000C50B8111EFCC1092830B0E943F1960E00D
:108CE00081E00E94D55A60E082E19EE00E94B930A6
:108CF00060E08EE09FE00E94B930A0908D0BDACC4E
:108D0000882309F443C0E13009F4EAC008F0A7C0A1
:108D10004FEF5FEFBA010091850B1091860B209108
:108D2000870B3091880B041715072607370708F4BF
:108D3000D5C08A019B01B901A801F82DA1108ACBE9
:108D4000BB2041F0E13009F4E0C008F498CBE230F8
:108D500009F4ABC0AA2341F0E13009F4DFC008F404
:108D6000A1CBE23009F4AAC0BB2309F4BDCBE130AA
:108D700009F4DDC008F4AACBE23009F0B5CB80914C
:108D8000B80B8F1708F0B0CB95E021C9F82D4FEF45
:108D90005FEFBA0157CB1092B00B8091C50B8111D8
:108DA000ABCC1092AF0B0E943F1964E081E00E94AF
:108DB000D55A60E08AEB9EE00E94B93060E086EB15
:108DC0009FE00E94B93098CC1092A50B8091C50B02
:108DD000811189CC1092A40B0E943F1963E081E0BD
:108DE0000E94D55A60E080E99EE00E94B93060E0C0
:108DF0008CE89FE00E94B93076CC10929A0B80915B
:108E0000C50B811167CC1092990B0E943F1962E04B
:108E100081E00E94D55A60E086E69EE00E94B9306B
:108E200060E082E69FE00E94B93054CC10928F0B34
:108E30008091C50B811145CC10928E0B0E943F1979
:108E400061E081E00E94D55A60E08CE39EE00E94E0
:108E5000B93060E088E39FE00E94B93032CCF82D51
:108E6000E23071F04FEF5FEFBA01ECCAE23009F087
:108E700047CFF091810BF81578F1F82D882391F305
:108E800080918C0B8F1710F4F82F91E0AA2009F431
:108E9000B5C04FEF5FEFBA018091970B8F1710F4B9
:108EA000F82F92E0BB2009F455CF8091A20B8F17C9
:108EB00010F4F82F93E0AA2309F456CF8091AD0B5C
:108EC0008F1710F4F82F94E0BB2309F40DCB57CF84
:108ED000E23009F035CFE0CF90E0D0CF91E02BCF5A
:108EE000882DF0918C0B8F1788F1F82FAA2009F4A8
:108EF00085C08F2F4FEF5FEFBA01F091970B8F175F
:108F000018F1F82FBB2009F425CF8091A20BF81798
:108F1000C8F08F2FF82FAA2309F426CF8091AD0B2C
:108F2000F81710F4F82F94E0BB2309F4DDCA809100
:108F3000B80BF81708F0D8CA95E049C892E09ACA69
:108F40008F2FDBCF93E0E6CF92E0DCCF91E0CECF66
:108F500094E0B8CA80E090E007C0332433940196CF
:108F60008038910509F432C828173907C1F3E82F72
:108F7000E695E695E695F0E0E659F54F4081442305
:108F800071F3FC01E770FF27EC5BF84F508154232D
:108F900031F3281739070CF479C8DFCFF091810B32
:108FA0008F1650F1F82D882309F45CCF8F2F99CFBD
:108FB00080E090E007C03324339401968038910517
:108FC00009F404C828173907C1F3E82FE695E69598
:108FD000E695F0E0E659F54F4081442371F3FC013A
:108FE000E770FF27EC5BF84F5081542331F3821771
:108FF00093070CF44BC8DFCF90E0D5CF4FEF5FEF76
:10900000BA019ECE94E00C94E73F93E00C94E73FC6
:1090100092E00C94E73F91E00C94E73FCF9380916E
:10902000FA0C8F3FA9F0C82FCF778091FC0C8C0FE2
:1090300040E050E060E0885E0E947E3F6091FC0C62
:109040006C0F685E40E080914F12CF910C942A1310
:10905000CF910895A8E7BCE0FD019FEF05C03196D0
:109060008CE0E83FF80749F0808187FFF8CF9083D4
:10907000F6CF8CE0A83FB80721F08D918F3FC9F360
:109080000895CCCF0F931F93CF93DF93082F162F04
:109090008091020D8017C1F0C1DFCFEFDFEFD093D9
:1090A000F90CC093F80C8FEF8093FA0C40E850E075
:1090B0006FEF70E088E79CE00E947F760E949E1729
:1090C0008091511281110FC0111104C08091010DC6
:1090D000811114C00093020D1093010DDF91CF9107
:1090E0001F910F910895D093F90CC093F80C2FEFB6
:1090F0003FE73093FE0C2093FD0CE6CFABDFEACFC9
:10910000CF92DF92EF92FF920F931F93CF93DF9353
:109110001F92CDB7DEB7082F112707FD109573E01A
:10912000E72E7DE0F72EE00EF11EF701EE5FFE4F19
:109130002081222309F44AC0F801EE0FFF1FE95FE6
:10914000F14FC080D1808FEFC81AD80AC601860FB0
:10915000911D67FD9A9530E01695102F0027179501
:1091600007950D5F124F02C07D3F69F4820F931F78
:109170000197B9010E948172F801E80FF91F72810D
:10918000C816D90689F7872F8D5F8230F8F0E7EF90
:10919000EE1AEEEFFE0AF701808140E050E060E059
:1091A000870F79830E947E3FF70160817981670F85
:1091B00040E080914F120F90DF91CF911F910F915E
:1091C000FF90EF90DF90CF900C942A130F90DF91D7
:1091D000CF911F910F91FF90EF90DF90CF90089566
:1091E000842F20914E1227FD09C06F7070E0332745
:1091F00027FD30956217730709F0089540E050E0AD
:1092000060E00C947E3F842FE0914E12E7FD09C090
:109210006F7070E0FF27E7FDF0956E177F0709F08C
:109220000895422F50E0542F4427550F41505E4F70
:1092300061E0211101C060E00C947E3F2F923F92CB
:109240004F925F926F927F928F929F92AF92BF9256
:10925000CF92DF92EF92FF920F931F93CF93DF9302
:10926000CDB7DEB72C970FB6F894DEBF0FBECDBFDB
:10927000E090F510F090F6102090ED103090EE1088
:109280008091CC108093340F8091CA108093380E57
:109290008091D610882309F4EAC463E08EE09FE051
:1092A0000E94C12F8091CB10882309F4DEC463E0B3
:1092B00082E19EE00E94C12F80915212882309F41E
:1092C000D0C480E091E0A0E0B0E02091F9103091AE
:1092D000FA102C013D01420E531E611C711C20919D
:1092E000F7103091F810AC01BD01420F531F611D02
:1092F000711D2091F3103091F4105C016D01A20EEC
:10930000B31EC11CD11CA982BA82CB82DC822091FF
:10931000F1103091F2105C016D01A20EB31EC11C60
:10932000D11CAD82BE82CF82D8862091EF103091C1
:10933000F0105C016D01A20EB31EC11CD11CA986E8
:10934000BA86CB86DC862091EB103091EC104C0174
:109350005D01820E931EA11CB11C09811A812B8113
:109360003C810115110581E02807310524F00FEF3C
:109370001FEF20E030E041155105E1E06E07710577
:1093800024F04FEF5FEF60E070E041145104F1E032
:109390006F0671042CF044244A94542C612C712CD7
:1093A0009701B2018EE09FE00E94932F9501840106
:1093B0008114910441E0A406B10424F00FEF1FEFE3
:1093C00020E030E049845A846B847C844114510449
:1093D00081E0680671042CF044244A94542C612CDA
:1093E000712C6D817E818F81988561157105E1E019
:1093F0008E07910524F06FEF7FEF80E090E0910100
:10940000A20182E19EE00E94932F8091CC10809374
:109410005E0F8091CA108093620E8091D6108823CF
:1094200009F41DC463E088E39FE00E94C12F80918E
:10943000CB10882309F411C463E08CE39EE00E9402
:10944000C12F80915212882309F403C480E09FEF5A
:10945000AFEFBFEF2091F9103091FA102C013D01D0
:10946000420E531E611C711C77FC03C42091F7103F
:109470003091F810AC01BD01420F531F611D711DE9
:1094800077FD41C42091F3103091F4105C016D011F
:10949000A20EB31EC11CD11C96018501D7FC2FC49E
:1094A0008090F1109090F2105C016D01A80CB91C35
:1094B000C11CD11CA982BA82CB82DC82D7FC1AC41F
:1094C0008090EF109090F0105C016D01A80CB91C19
:1094D000C11CD11CAD82BE82CF82D886D7FC05C408
:1094E000E091EB10F091EC104C015D018E0E9F1E8F
:1094F000A11CB11CB7FCF5C30115110581E02807BB
:10950000310524F00FEF1FEF20E030E04115510549
:10951000E1E06E07710524F04FEF5FEF60E070E06F
:1095200041145104F1E06F0671042CF044244A9474
:10953000542C612C712C9701B20188E39FE00E94AA
:10954000932F950184018114910441E0A406B10494
:1095500024F00FEF1FEF20E030E04D805E806F8041
:1095600078844114510481E0680671042CF044248D
:109570004A94542C612C712C69817A818B819C8155
:1095800061157105E1E08E07910524F06FEF7FEF23
:1095900080E090E09101A2018CE39EE00E94932F75
:1095A0008091CC108093880F8091CA1080938C0E8C
:1095B0008091D610882309F44AC363E082E69FE0D5
:1095C0000E94C12F8091CB10882309F43EC363E031
:1095D00086E69EE00E94C12F80915212882309F4F2
:1095E00030C380E092E0A0E0B0E02091F91030912B
:1095F000FA102C013D01420E531E611C711C20917A
:10960000F7103091F810AC01BD01420F531F611DDE
:10961000711D2091F3103091F4105C016D01A20EC8
:10962000B31EC11CD11CA982BA82CB82DC822091DC
:10963000F1103091F2105C016D01A20EB31EC11C3D
:10964000D11CAD82BE82CF82D8862091EF1030919E
:10965000F0105C016D01A20EB31EC11CD11CA986C5
:10966000BA86CB86DC862091EB103091EC104C0151
:109670005D01820E931EA11CB11C09811A812B81F0
:109680003C810115110581E02807310524F00FEF19
:109690001FEF20E030E041155105E1E06E07710554
:1096A00024F04FEF5FEF60E070E041145104F1E00F
:1096B0006F0671042CF044244A94542C612C712CB4
:1096C0009701B20182E69FE00E94932F95018401E9
:1096D0008114910441E0A406B10424F00FEF1FEFC0
:1096E00020E030E049845A846B847C844114510426
:1096F00081E0680671042CF044244A94542C612CB7
:10970000712C6D817E818F81988561157105E1E0F5
:109710008E07910524F06FEF7FEF80E090E09101DC
:10972000A20186E69EE00E94932F8091CC10809348
:10973000B20F8091CA108093B60E8091D610882304
:1097400009F47DC263E08CE89FE00E94C12F809104
:10975000CB10882309F471C263E080E99EE00E9487
:10976000C12F80915212882309F463C280E09EEFDA
:10977000AFEFBFEF2091F9103091FA102C013D01AD
:10978000420E531E611C711C77FCA7C22091F7107A
:109790003091F810AC01BD01420F531F611D711DC6
:1097A00077FD97C22091F3103091F4105C016D01A8
:1097B000A20EB31EC11CD11C96018501D7FC85C227
:1097C0008090F1109090F2105C016D01A80CB91C12
:1097D000C11CD11CA982BA82CB82DC82D7FC70C2A8
:1097E0008090EF109090F0105C016D01A80CB91CF6
:1097F000C11CD11CAD82BE82CF82D886D7FC5BC291
:10980000E091EB10F091EC104C015D018E0E9F1E6B
:10981000A11CB11CB7FC4BC20115110581E0280742
:10982000310524F00FEF1FEF20E030E04115510526
:10983000E1E06E07710524F04FEF5FEF60E070E04C
:1098400041145104F1E06F0671042CF044244A9451
:10985000542C612C712C9701B2018CE89FE00E947E
:10986000932F950184018114910441E0A406B10471
:1098700024F00FEF1FEF20E030E04D805E806F801E
:1098800078844114510481E0680671042CF044246A
:109890004A94542C612C712C69817A818B819C8132
:1098A00061157105E1E08E07910524F06FEF7FEF00
:1098B00080E090E09101A20180E99EE00E94932F58
:1098C0008091CC108093DC0F8091CA108093E00EC1
:1098D0008091D610882309F4AAC163E086EB9FE04B
:1098E0000E94C12F8091CB10882309F49EC163E0B0
:1098F0008AEB9EE00E94C12F80915212882309F4C6
:1099000090C180E093E0A0E0B0E02091F9103091A8
:10991000FA102C013D01420E531E611C711C209156
:10992000F7103091F810AC01BD01420F531F611DBB
:10993000711D2091F3103091F4105C016D01A20EA5
:10994000B31EC11CD11CA982BA82CB82DC822091B9
:10995000F1103091F2105C016D01A20EB31EC11C1A
:10996000D11CAD82BE82CF82D8862091EF1030917B
:10997000F0105C016D01A20EB31EC11CD11CA986A2
:10998000BA86CB86DC862091EB103091EC104C012E
:109990005D01820E931EA11CB11C09811A812B81CD
:1099A0003C810115110581E02807310524F00FEFF6
:1099B0001FEF20E030E041155105E1E06E07710531
:1099C00024F04FEF5FEF60E070E041145104F1E0EC
:1099D0006F0671042CF044244A94542C612C712C91
:1099E0009701B20186EB9FE00E94932F95018401BD
:1099F0008114910441E0A406B10424F00FEF1FEF9D
:109A000020E030E049845A846B847C844114510402
:109A100081E0680671042CF044244A94542C612C93
:109A2000712C6D817E818F81988561157105E1E0D2
:109A30008E07910524F06FEF7FEF80E090E09101B9
:109A4000A2018AEB9EE00E94932F8091CC1080931C
:109A500006108091CA1080930A0F8091D610882337
:109A600009F4DDC063E080EE9FE00E94C12F809189
:109A7000CB10882309F4D1C063E084EE9EE00E94FD
:109A8000C12F80915212882309F4C3C080E09DEF5A
:109A9000AFEFBFEF2091F9103091FA102C013D018A
:109AA000420E531E611C711C77FCFDC02091F71003
:109AB0003091F810AC01BD01420F531F611D711DA3
:109AC00077FDEDC02091F3103091F4105C016D0131
:109AD000A20EB31EC11CD11C96018501D7FCDBC0B0
:109AE0008090F1109090F2105C016D01A80CB91CEF
:109AF000C11CD11CA982BA82CB82DC82D7FCC6C031
:109B00008090EF109090F0105C016D01A80CB91CD2
:109B1000C11CD11CAD82BE82CF82D886D7FCB1C019
:109B2000E091EB10F091EC104C015D018E0E9F1E48
:109B3000A11CB11CB7FCA1C00115110581E02807CB
:109B4000310524F00FEF1FEF20E030E04115510503
:109B5000E1E06E07710524F04FEF5FEF60E070E029
:109B600041145104F1E06F0671042CF044244A942E
:109B7000542C612C712C9701B20180EE9FE00E9461
:109B8000932F950184018114910441E0A406B1044E
:109B900024F00FEF1FEF20E030E04D805E806F80FB
:109BA00078844114510481E0680671042CF0442447
:109BB0004A94542C612C712C69817A818B819C810F
:109BC00061157105E1E08E07910524F06FEF7FEFDD
:109BD00080E090E09101A20184EE9EE00E94932F2C
:109BE0002C960FB6F894DEBF0FBECDBFDF91CF919C
:109BF0001F910F91FF90EF90DF90CF90BF90AF90AB
:109C00009F908F907F906F905F904F903F902F909C
:109C1000089580E090E0DC013DCF61E02ECF61E06F
:109C200022CF80E090E0DC0170CE61E061CE61E0A7
:109C300055CE80E090E0DC019DCD61E08ECD61E00D
:109C400082CD80E090E0DC01D0CC61E0C1CC61E06D
:109C5000B5CC80E090E0DC01FDCB61E0EECB61E0D3
:109C6000E2CB80E090E0DC0130CB61E021CB61E031
:109C700015CB412C512C3201F9CB812C912C540164
:109C80005BCF1D821E821F8218864ACF19821A82DC
:109C90001B821C8235CF00E010E0980121CF40E00C
:109CA00050E0BA010FCF412C512C3201FFCE812C54
:109CB000912C5401B1CD1D821E821F821886A0CD29
:109CC00019821A821B821C828BCD00E010E0980161
:109CD00077CD40E050E0BA0165CD412C512C3201E6
:109CE00055CD812C912C540107CC1D821E821F82E0
:109CF0001886F6CB19821A821B821C82E1CB00E007
:109D000010E09801CDCB40E050E0BA01BBCBCF933F
:109D100080916A0A90916B0A892B90916C0A892B29
:109D200090916D0A892B90916E0A892B90916F0A00
:109D3000892B9091700A892B9091710A892B9091AF
:109D4000720A892B9091730A892B9091740A892B3E
:109D50009091750A892B9091760A892B9091770AB8
:109D6000892B9091780A892B9091790A982B21E080
:109D700009F420E08091980B90918D0B892B9091A4
:109D8000A30B892B9091AE0B892B9091820B892B81
:109D90009091B90B892B59F48FEF9FEFDC018093E1
:109DA000B5109093B610A093B710B093B8102223BB
:109DB00021F080917E14882361F120937E140E940B
:109DC00027190E94B6398091CE10811133C00E94AC
:109DD0003C18C09150128091C30BC81721F00E940B
:109DE0009E17C093C30BC091CF108091C20BC817B0
:109DF00031F00E949E17C33050F4C093C20B0E94F2
:109E000026321CDA0E94D115CF910C945F35C0E048
:109E1000F4CF8091A4099091A509A091A609B091D1
:109E2000A7098093B5109093B610A093B710B09384
:109E3000B810C3CF61E083E191E10E940018C9CF5F
:109E4000E82FF0E0E755F64F90819170803209F4E9
:109E500056C078F0843209F44CC0A0F1863209F47F
:109E600045C008F058C09093C41081E080931B1146
:109E70004ECF8C31C8F08C3109F444C08091C609B2
:109E800081709091C8109073892B9091C70990FDB3
:109E900047C090E0892B9091C80990FF45C092E09F
:109EA000892B8093C810E1CF8A31A8F08091C40932
:109EB00081709091C30990FD35C090E0892B80930B
:109EC000C910D3CF8232C1F018F09093C010CDCF1B
:109ED0009093BE10CACF883131F0893109F00895CE
:109EE0009093C210C2CF9093BF10BFCF9093C51074
:109EF000BCCF9093C110B9CF9093C310B6CF9093BD
:109F0000BD10B3CF9091C5098091C61090FB80F928
:109F10008093C610AACF873211F79093CE10A5CFA9
:109F200098E0B8CF92E0CACF90E0BACFCF93C8E123
:109F30008C2F86DFCF5FC832D9F7CF9108952F924B
:109F40003F924F925F926F927F928F929F92AF92C9
:109F5000BF92CF92DF92EF92FF921F93CF93DF9346
:109F6000CDB7DEB762970FB6F894DEBF0FBECDBF98
:109F700080914D12882381F180914B1290914C1267
:109F80000E94251B882371F180914D12882381F155
:109F90000E94E21810921B1181E090914D129111D4
:109FA00001C080E08093191162960FB6F894DEBF6D
:109FB0000FBECDBFDF91CF911F91FF90EF90DF904B
:109FC000CF90BF90AF909F908F907F906F905F9059
:109FD0004F903F902F9008958BED90E00E94251BAD
:109FE0008111D2CF0E946D1A80914D128111D0CF74
:109FF0009DDF80910E0190910F012091120130910F
:10A000001301A0901001B09011014501809490942B
:10A010006C01C21AD30ADA82C9822501612C712C23
:10A02000C0901401D0901501E0901601F090170136
:10A03000A901480F591F5C834B83CA01A0E0B0E01F
:10A040008D839E83AF83B8872091180130911901C9
:10A0500040911A0150911B0129873A874B875C87F1
:10A0600090911B1110E0CF86D88AE98AFA8A0FC036
:10A0700022242A94322CED85FE85EE0FFF1FE95233
:10A08000FF4E3182208291E01F5F1E31E9F1C12E27
:10A09000D12CDE86CD86F601E057F94F80818F3FC7
:10A0A00099F3E82FEE0FFF0BEF50F44F2080318033
:10A0B0000E94651C8823F9F282149304C8F22A14C2
:10A0C0003B04B0F0C101A0E0B0E0E980FA802E14BA
:10A0D0003F0488F49C01AD0124193509460957094C
:10A0E0006F85788989899A890E9466721C01C3CF1D
:10A0F000212C312CC0CFCB80DC80C214D30438F0AB
:10A10000212C80E8382EB7CF90931B1141CF9C01B2
:10A11000AD01CD80DE80EF80F8842C193D094E0919
:10A120005F0969857A858B859C850E946672905847
:10A130001C01A1CF9091770C9D7F8111926090932B
:10A14000770C4FB7F8948091770C96EC91BB469AB8
:10A15000382F330F982F9695232F26702064582F71
:10A16000551F5527551F252B582F5071832F880FAA
:10A170008072852B307C832B9270906631E035B9EC
:10A1800028B98BB99EB987E881BB4FBF08959091DC
:10A19000770C9F7D811190629093770C4FB7F89464
:10A1A0008091770C96EC91BB469A382F330F982FFD
:10A1B0009695232F26702064582F551F5527551F1D
:10A1C000252B582F5071832F880F8072852B307C60
:10A1D000832B9270906631E035B928B98BB99EB95E
:10A1E00087E881BB4FBF08952F923F924F925F92B5
:10A1F0006F927F928F929F92AF92BF92CF92DF9297
:10A20000EF92FF920F931F93CF93DF93682EE82F67
:10A21000E695E695E695F0E0E659F54FA82FA7708C
:10A22000B0E0AC5BB84F80819C91892B8083A62CD9
:10A23000B12CF501EE0FFF1FE658F54F80E090E8D6
:10A2400091838083C090A409D090A509E090A609CD
:10A25000F090A7098091C40B882309F49DC08091D8
:10A26000C20B512C882319F1823009F4D0C38130FC
:10A2700009F4F1C380E090E0A816B906A1F0E82F38
:10A28000E695E695E695F0E0E659F54F2081222324
:10A2900051F0FC01E770FF27EC5BF84F308132236F
:10A2A00011F05524539401968038910529F790E0D8
:10A2B0008CEB882E8BE0982E2BE0422E7724739423
:10A2C000212C30E8332E06E010E0F40181914F019B
:10A2D0008F3F09F44EC0C92FDD27C7FDD0954C9E96
:10A2E00090014D9E300D11242659354FF901E85E3D
:10A2F000FE4F7082F901E75EFE4F7082F901E65E63
:10A30000FE4F7082F901EC5EFE4F31822082F9012E
:10A31000EA5EFE4F6082F901E95EFE4FA501480F3B
:10A32000511D4083F901E05FFE4FC082D182E2827D
:10A33000F382452D60E070E8892F0E940B3F409129
:10A34000C30B04C0C92FDD27C7FDD095CE010196F0
:10A35000B8010E9481729C01982FF901EC5BF84FC3
:10A360008081842379F3F2EC8F16FBE09F0609F0DD
:10A37000ACCFDF91CF911F910F91FF90EF90DF90C5
:10A38000CF90BF90AF909F908F907F906F905F9095
:10A390004F903F902F900895E091C30BCE2FC17046
:10A3A000E0FD27C14FEF5FEFBA019FEF2E2F227024
:10A3B000E1FF17C080918D0B2090850B3090860BAC
:10A3C0004090870B5090880B882309F477C12C1498
:10A3D0003D044E045F0428F480918C0B681609F448
:10A3E00093C28E2F8470E2FF17C03091980B20909B
:10A3F000900B3090910B4090920B5090930B332325
:10A4000009F466C12C143D044E045F0428F4309115
:10A41000970B631609F475C23E2F3870E3FF17C01F
:10A42000F091A30B20909B0B30909C0B40909D0BC8
:10A4300050909E0BFF2309F455C12C143D044E048B
:10A440005F0428F4F091A20B6F1609F457C2AE2FE7
:10A45000A071E4FF17C0F091AE0B2090A60B3090D6
:10A46000A70B4090A80B5090A90BFF2309F444C1FF
:10A470002C143D044E045F0428F4F091AD0B6F16CC
:10A4800009F439C2BE2FB072E5FF17C0E091B90BD5
:10A49000EE2309F43BC14091B10B5091B20B609196
:10A4A000B30B7091B40B4C155D056E057F0528F458
:10A4B0004091B80B641609F437C19F3F09F097C06B
:10A4C000C111B1C04FEF5FEFBA012223E1F010914B
:10A4D0008B0BE12FE695E695E695F0E0E659F54F12
:10A4E000D081D1116AC12090850B3090860B4090AD
:10A4F000870B5090880B241635064606570618F42D
:10A50000B201A10191E08823E1F01091960BE12FB7
:10A51000E695E695E695F0E0E659F54FD081D11144
:10A5200070C12090900B3090910B4090920B509006
:10A53000930B241635064606570618F4B201A101FE
:10A5400092E03323E1F01091A10BE12FE695E6951F
:10A55000E695F0E0E659F54FD081D11166C1209023
:10A560009B0B30909C0B40909D0B50909E0B2416A3
:10A5700035064606570618F4B201A10193E0AA2356
:10A58000E1F01091AC0BE12FE695E695E695F0E051
:10A59000E659F54FD081D1113EC12090A60B3090E5
:10A5A000A70B4090A80B5090A90B24163506460621
:10A5B000570618F4B201A10194E0BB23B1F0109149
:10A5C000B70BE12FE695E695E695F0E0E659F54FF5
:10A5D000D081DD2309F405C11770E12FF0E0EC5BB9
:10A5E000F84FE081ED2309F4FCC09F3FC9F1512CE5
:10A5F0005FCE8091820B882309F44FC080917A0B43
:10A6000090917B0BA0917C0BB0917D0B8C159D05DF
:10A61000AE05BF0508F0C6CE8091810B6812C2CE90
:10A6200090E0512C45CE5091800BE52FE695E695B4
:10A63000E695F0E0E659F54F40814111C8C04091E0
:10A640007A0B50917B0B60917C0B70917D0B4F3F8F
:10A65000EFEF5E076E077E0709F437CF90E035CF46
:10A66000E091C20BCC2309F462C0E13009F4C3C10C
:10A6700008F04DC140917A0B50917B0B60917C0B9F
:10A6800070917D0B4F3FFFEF5F076F077F0709F06A
:10A6900090E0211157C0F62DD6C040917A0B509111
:10A6A0007B0B60917C0B70917D0B4F3F8FEF5807B8
:10A6B0006807780709F479CE90E078CE241635063D
:10A6C0004606570608F08DCEB201A10191E089CE71
:10A6D000241635064606570608F09ECEB201A101A3
:10A6E00092E09ACE241635064606570608F0AFCEFD
:10A6F000B201A10193E0ABCE2416350646065706FB
:10A7000008F0C0CEB201A10194E0BCCE2090B10B04
:10A710003090B20B4090B30B5090B40B241635061A
:10A720004606570608F0C9CE95E0512CC1CD22232C
:10A7300009F485C0E13009F42BC108F020C14FEFC6
:10A740005FEFBA012090850B3090860B4090870B0D
:10A750005090880B241635064606570608F4B7C1F4
:10A760001A012B01B201A101F62D811174C033230E
:10A7700041F0E13009F424C108F482C0E23009F468
:10A78000E9C0AA2341F0E13009F424C108F48DC0E6
:10A79000E23009F4E9C0BB2309F4A9C0E13009F4AF
:10A7A00023C108F496C0E23009F0A1C08091B80B33
:10A7B0008F1708F09CC095E0B8CF1770E12FF0E03C
:10A7C000EC5BF84FE081ED2309F09DCE8CCE577005
:10A7D000E52FF0E0EC5BF84F5081542309F072CE86
:10A7E0002ECF2090B10B3090B20B4090B30B509015
:10A7F000B40B241635064606570608F0F6CE95E04B
:10A8000094CF1770E12FF0E0EC5BF84FE081ED237F
:10A8100009F097CE86CE1770E12FF0E0EC5BF84F91
:10A82000E081ED2309F0C9CEB8CE1770E12FF0E03A
:10A83000EC5BF84FE081ED2309F0A1CE90CEF62D30
:10A840004FEF5FEFBA01882309F491CFE13009F4AB
:10A85000ADC008F099C02090900B3090910B4090C3
:10A86000920B5090930B241635064606570608F4B3
:10A870002CC11A012B01B201A101332309F481CFAC
:10A8800000919B0B10919C0B20919D0B30919E0B86
:10A89000041715072607370708F407C18A019B012B
:10A8A000B901A801AA2309F476CF0091A60B109153
:10A8B000A70B2091A80B3091A90B041715072607A9
:10A8C000370708F4FCC08A019B01BB2381F0B90162
:10A8D000A8010091B10B1091B20B2091B30B3091F4
:10A8E000B40B041715072607370708F41DCF9F3F41
:10A8F00009F43FCD7CCE94E0512CDACC93E0512C7E
:10A90000D7CC92E0512CD4CC91E0512CD1CCE23078
:10A9100009F00DCFF091810BF61508F4C4C0F62DA7
:10A92000222309F470C02F2FF0918C0BF21708F43A
:10A93000B8C0F22F4FEF5FEFBA01882309F417CFA9
:10A940008091970B8F1708F4B2C08F2F332309F42F
:10A95000C2C0F82F8091A20B8F1708F4AAC08F2FC6
:10A96000AA2309F4BAC0F82F8091AD0B8F1708F411
:10A97000B0C08F2FBB2309F4BACFF82F17CFE23026
:10A9800009F05DCF262DD0CFE23009F0F0CED8CF40
:10A99000F62D20918C0BF21708F493C02F2FF22F75
:10A9A0004FEF5FEFBA01882309F4E1CE8091970B56
:10A9B000F81708F482C08F2F332309F48CC0F82FC6
:10A9C0008091A20BF81708F476C08F2FAA2309F400
:10A9D00084C0F82F8091AD0BF81708F460C08F2F5A
:10A9E000BB2309F484CFF82F8091B80BF81708F037
:10A9F0007ECF95E09ACEF091810B6F1608F463C07C
:10AA0000F62D2111C6CF4FEF5FEFBA011CCF80E0CA
:10AA100090E007C05524539401968038910509F4BD
:10AA200046CCA816B906C1F3E82FE695E695E6955B
:10AA3000F0E0E659F54F2081222371F3FC01E77025
:10AA4000FF27EC5BF84F3081322331F3A816B906AB
:10AA50000CF48FCCDFCF80E090E007C055245394F6
:10AA600001968038910509F422CCA816B906C1F3E5
:10AA7000E82FE695E695E695F0E0E659F54F20815A
:10AA8000222371F3FC01E770FF27EC5BF84F308164
:10AA9000322331F38A159B050CF46BCCDFCF94E0A5
:10AAA0009FCF91E047CF90E03BCF93E0F9CE92E08B
:10AAB0004DCF93E055CF93E089CF92E07DCF94E0E6
:10AAC00004CF91E06CCF90E09CCF92E0D4CE91E0A7
:10AAD00049CE94E04FCFF82F54CEF82F5CCE603E95
:10AAE00071058105910508F00895DC01CB019F5F98
:10AAF000AF4FBF4F6627782F892F9A2F0C9400F8FD
:10AB000080918F17909190178F5895418130924086
:10AB100070F44FE855E16CED70E080E090E0DFDF2D
:10AB20004FE856E16DED70E080E090E0D8CF0895F9
:10AB3000FF920F931F93CF93DF93FFB60E946A1A81
:10AB4000882309F43EC00E94461AC9E2D1E111C02F
:10AB5000FE01E00FF11F808191810E94601A0E5F5B
:10AB60001F4F04321105A1F7A49682E1C934D8071A
:10AB700019F000E010E0ECCF80914B1290914C1254
:10AB80000E94601A8091491290914A120E94601AA4
:10AB900080914D120E943B1A80914E120E94301AF1
:10ABA000809150120E943B1A80914F120E94301ADD
:10ABB000809151120E943B1A809152120E94301AC9
:10ABC0009FDF8F2DDF91CF911F910F91FF900C94FC
:10ABD0002E1A0F931F93CF93DF934FB7F89436EC51
:10ABE00031BB469A80EE87B997E09AB98DB981E07A
:10ABF00085B980E488B91BB880E28EB987E481BB4F
:10AC000052E05A95F1F700C026B199B18CB131BB31
:10AC1000479AC22FC695C37050E8259F9001112412
:10AC2000C22B292F2071C22B292F269526952870FB
:10AC3000C22B96959076C92B90E0880F991F84704F
:10AC40009927C82B87EE87B987EF8AB982EE8DB92D
:10AC50004FBF8091CE10882391F080918014C5FF62
:10AC600040C08C2785FD10C080915112823039F18F
:10AC7000C0938014DF91CF911F910F91089580911F
:10AC800080148C2785FFF0CFD091020DD11137C0F1
:10AC9000C5FF44C00E944D3E00E040914F124F70EE
:10ACA000406BE0919219F091931920E463E070E019
:10ACB00082E999E10995809151128230C9F6C0FF6D
:10ACC000D7CF8091801480FDD3CF8091BB108F5F50
:10ACD0008093BB10C0938014DF91CF911F910F918F
:10ACE000089585FFBECF0E94591886E0ECEBFBE08B
:10ACF000A3E1B1E101900D928A95E1F7B5CF11E0A2
:10AD0000C5FF05C010E08091010D81110CC0D093EA
:10AD1000020D1093010D0E945F35A6CF81E0809354
:10AD2000C50B0FE7BACF0E942A48F1CF0E94E41D5D
:10AD300061E088E00E943D178BE10E944C2E80E08C
:10AD40000E94232E80E0F6D980E00E941B2E80E036
:10AD50000E943B2E80E01BDA80E00E94332E80E0D0
:10AD60000E942B2E60E080E090E00E94A02E8CE1FB
:10AD70000E944C2E8FE10E944C2E88E10E944C2EA6
:10AD80008DE10E944C2E0E941E140E942F140C94E0
:10AD90004014CF93DF9300D000D01F92CDB7DEB721
:10ADA000C5DFC12CD12C96ECA92E8824839420E4F5
:10ADB000B22E30EE932E47EF342E52EE252E02E1C6
:10ADC00010E0FFB60E94F41C882309F43FC0A1BA2A
:10ADD000469A85B8B8B81BB81EB887E881BB9DE015
:10ADE0009A95F1F70000A1BA469A97B8E7E0EAB958
:10ADF0009DB885B8B8B81BB8BEB8F7E4F1BB82E01F
:10AE00008A95F1F700C046B199B12CB1A1BA479A21
:10AE1000C42EC694E3E0CE22F0E84F9FA001112497
:10AE2000C42A892F8071C82A392F369536953870F3
:10AE3000C32A96959076C92A30E0220F331F2470DA
:10AE40003327C22A87EE87B93AB82DB88F2D0E94D2
:10AE5000EC1CC1FE08C08D2D90E00196B8010E9447
:10AE60008172D82E09C0C2FE07C08D2D90E0419698
:10AE7000B8010E948172D82ED0927F149BE09D155C
:10AE800018F48FEF9FEF02C080E090E060E00E9436
:10AE9000A02E8D2D66E00E947572E92EF12C412CBA
:10AEA000512CE414F50419F46FEF7FEF02C060E059
:10AEB00070E0842D8E5E0E94432E842D845F0E945C
:10AEC000812E842D0E94812E842D8A5F0E94812EE6
:10AED000EFEF4E1A5E0AF6E04F16510411F785E0C7
:10AEE0008D1518F08FEF9FEF02C080E090E060E0DA
:10AEF0000E94962E95E09D1510F08FEF01C080E026
:10AF00000E94232E2D2D2650263018F48FEF9FEF10
:10AF100002C080E090E060E029830E948C2E2981AD
:10AF2000263010F48FEF01C080E00E941B2EEBE072
:10AF30008D2DED1550F00E94762E0E94F73A2B01D0
:10AF40003C018D2D0E946B2E09C00E94602E0E9434
:10AF5000F73A2B013C018D2D0E94552E0E94A73AF5
:10AF6000AB01BC0192E1892F49835A836B837C83B7
:10AF70009D830E944C2E9D819F5F49815A816B81E8
:10AF80007C81983181F74419550966097709BB27F7
:10AF900077FDBA95A72F962F852F84369105A105A9
:10AFA000B10524F083E690E0A0E0B0E02C013D0183
:10AFB0008D39FFEF9F07AF07BF0734F4ADE94A2E85
:10AFC00055245A94652C752CC20157FE03C09195E7
:10AFD00081959109BC01882777FD8095982F0E9463
:10AFE0007817C301B201662797FD639577278827F5
:10AFF000992789E00E943D17F2E3FF2E8FE39CE939
:10B000000197F1F700C000000E94F8270E94033A60
:10B01000FA94A1F7D6CECF932091100E3091110E55
:10B020002F3F8FEF3807C1F080910E0E90910F0ED9
:10B03000019690930F0E80930E0E8217930760F087
:10B0400010920F0E10920E0E8091030D8230A1F11E
:10B050008091040D823011F0CF9108956091060E19
:10B060006623D1F38091090E90910A0E019670E04B
:10B070000E94817290930A0E8093090EFC01EB5797
:10B08000F24FC081CD3F41F36FEF81E00E948048D5
:10B090008C2F8D5F823000F380910B0E8C0FA4D823
:10B0A00080910B0E60E070E88C0F0E94111380916C
:10B0B0000B0E80930D0ED0CF6091050E662341F2EA
:10B0C0008091070E9091080E019670E00E948172A7
:10B0D0009093080E8093070EFC01ED5FF24FC28142
:10B0E000CD3F09F4B5CF6FEF80E00E9480488C2FF0
:10B0F0008D5F823008F4ACCF80910B0E8C0F74D82A
:10B1000080910B0E60E070E88C0F0E94111380910B
:10B110000B0E80930C0E9CCFCF938091020D882351
:10B1200061F12091FF0C3091000D2F3F8FEF380718
:10B1300021F18091FD0C9091FE0C01969093FE0CF4
:10B140008093FD0C82179307C0F01092FE0C1092B2
:10B15000FD0CE8E7FCE004C08CE0E83FF80769F08C
:10B1600081918F3FC9F30E940E488091020D823079
:10B17000E1F0833019F1813009F1CF9108956150E8
:10B1800071098109910960687F6F8F6F9F6F6F5F91
:10B190007F4F8F4F9F4FFB017093F90C6093F80C1A
:10B1A000E858F34F80818F3F21F50E94E3766F7757
:10B1B00077278827907897FFEECFE1CF2091F80C82
:10B1C0003091F90C07C09C01FC01E858F34F408115
:10B1D0004F3F59F4C90101968F77907897FFF3CFCD
:10B1E000019780689F6F0196EECF8093F80C909343
:10B1F000F90CC081CF778091FB0C885E8C0F0E9488
:10B20000F4508091FB0C885E60E070E88C0F0E9427
:10B210001113E091F80CF091F90CE858F34F80818C
:10B220008093FA0C8091FB0C8093FC0CA6CF26EC4B
:10B2300090EE87E0F0E8E7E477EE67EF52EE4FB785
:10B24000F89421BB469A97B98AB99DB915B8F8B94F
:10B250008BB91EB8E1BB32E03A95F1F700C036B1C8
:10B26000A9B1ACB121BB479A77B96AB95DB94FBFF3
:10B2700045E04A95F1F7000032FFE1CF8FB7F8942F
:10B2800096EC91BB469A15B890E898B993E09BB9B3
:10B2900090E29EB997E891BB95E09A95F1F700008E
:10B2A0008FBF0895CF93DF93FC01D62FCFB7F894CB
:10B2B000218130E0C90101964281642F70E00E9433
:10B2C0008172408150E08417950791F0A381B48189
:10B2D000A20FB31FDC93818190E00196628170E040
:10B2E0000E9481728183CFBF81E0DF91CF91089569
:10B2F000CFBF80E0DF91CF910895FC013FB7F89474
:10B3000021819081291728F48281820F891B3FBFF8
:10B310000895822F891B3FBF08956F928F929F924D
:10B32000AF92BF92CF92DF92EF92FF920F931F9353
:10B33000CF93DF93E091B219F091B319309719F0E0
:10B3400082E999E109958AE79AE1D7DF082F10E0B1
:10B350000115110509F478C0C0E0D0E090917A1A87
:10B3600020917C1AEE24E394F12CE3E09E2EF4E08D
:10B370008F2EA2E0AA2EBB24B394892F622F90E0D7
:10B3800070E00E948172E0917D1AF0917E1AE80FC0
:10B39000F91FF081F83F08F065C0F7FF71C0809198
:10B3A000B719843031F0F093B419F092B919E092E2
:10B3B000B8198F2F807F803B79F198F4803961F143
:10B3C000803A51F1803841F1F03F09F4B1C0F73FC4
:10B3D00009F4C3C01092B7191092B9191092B81994
:10B3E0001DC0803D09F4A1C008F49CC0803EA1F0BE
:10B3F000803F51F7EF2FE15FEF3030F7AE2FB0E035
:10B40000A45BB84F8C91813009F49BC0E8F2823084
:10B4100009F48BC08330F1F69092B7193FB7F894D6
:10B4200090917A1A892F90E0019620917C1A622FD0
:10B4300070E00E948172982F80937A1A3FBF219604
:10B44000C017D10708F499CFDF91CF911F910F91C9
:10B45000FF90EF90DF90CF90BF90AF909F908F9034
:10B460006F900895D090B719B092B71920E040E0DE
:10B470006F2F81E090E00E943D13D092B719CECF9C
:10B480006090B719662051F24091B8195091B919DE
:10B490009A01ABEABAEA0E945D776C01D694C79430
:10B4A000C601880F991F8C0D9D1D6A01C81AD90A03
:10B4B000D601AE56B64E9296FC93CA010196909371
:10B4C000B9198093B81921E0C216D104B9F022E06D
:10B4D000C216D10409F0A2CF2091B6194091B51936
:10B4E0006091B4190E943D138091B719843009F41A
:10B4F00095CFF092B919E092B81990CF22E062127C
:10B500008DCF20E04091B5196091B4190E943D1390
:10B510008091B719843009F481CFD092B919C092C3
:10B52000B8197CCF803C09F04FCFA092B71976CFE5
:10B530008092B719F093B419F092B919E092B81942
:10B540006DCF8093B71920E040E06F2F81E090E04D
:10B550000E943D131092B71961CF4091B8195091D4
:10B56000B9199A01ABEABAEA0E945D779695879578
:10B570009C01220F331F280F391FDA01A21BB30BC6
:10B58000AE56B64E9296FC93CA0101969093B919A5
:10B590008093B8192091B6194091B5196091B419EA
:10B5A0000E943D131092B71939CF2F923F924F92BC
:10B5B0005F926F927F928F929F92AF92BF92CF9243
:10B5C000DF92EF92FF920F931F93CF93DF93CDB74C
:10B5D000DEB76B970FB6F894DEBF0FBECDBF762EE9
:10B5E000882309F494C0E091E310F091E410809076
:10B5F000E5109090E6104091D7105091D8108091AE
:10B60000DD109091DE1020910F11309110114090BB
:10B610000F0C5090100C6090C9106091D310509294
:10B62000821540928115F0938415E09383159092D2
:10B6300086158092851550938815409387159093B1
:10B640008A158093891530938C1520938B15609201
:10B650008D1560938E15440C452C441C550851944F
:10B6600082011A9518870F83EE0FEF2FEE1FFF0B45
:10B67000F1958F011A951A8B098BA12CB12C7501AC
:10B680006401CC0CDD1CEE1CFF1CCC0CDD1CEE1C84
:10B69000FF1CC80CD91CEA1CFB1C13E0F694E794B1
:10B6A000D794C7941A95D1F75695479556954795CF
:10B6B00096958795969587950D2D11271C870B8755
:10B6C000052F11271A830983092F1127DD24EE2462
:10B6D000FF24662309F440C0623008F436C6ECE06B
:10B6E000F0E089819A81BF010E94817249815A816B
:10B6F000481B590B5A834983C801BF010E948172BC
:10B70000081B190B188A1F861E861D862DC04090A7
:10B710000F0C5090100C8091811590918215E09142
:10B72000E310F091E4108415950509F4E9C58090C3
:10B73000E5109090E6104091D7105091D81080916C
:10B74000DD109091DE1020910F113091101160905A
:10B75000C9106091D31063CFBA0177277E876D87B8
:10B76000DC01BB27B88BAF875091CE105D8B7091F9
:10B7700052127F8B832F99279C8B8B8B2091B41037
:10B780002E8B77FC29C1772009F426C177FCCEC423
:10B7900031E0731609F4CAC477FCDFC332E07316D4
:10B7A00009F4DBC377FCEDC233E0731609F4E9C298
:10B7B00077FCFAC134E0731609F4F6C177FC1CC0BB
:10B7C00045E07416C9F06B960FB6F894DEBF0FBE55
:10B7D000CDBFDF91CF911F910F91FF90EF90DF9040
:10B7E000CF90BF90AF909F908F907F906F905F9021
:10B7F0004F903F902F9008958091B90B882319F3B3
:10B800008091B80B282F30E0285131093C832B83DD
:10B81000020F131F2F813885442737FD4095542F81
:10B820002F83388749875A87809096109090971079
:10B83000AA2497FCA094BA2C820E931EA41EB51EB7
:10B8400089819A812B813C81820F931F97FDF6C6D7
:10B8500045E06D850E94511414012501280E391E02
:10B86000411C511C57FCA3C62114310431E043068E
:10B8700051040CF09AC58090A2109090A310AA24B5
:10B8800097FCA094BA2C2F81388549855A85820E61
:10B89000931EA41EB51E29893A89C901AA2797FDBE
:10B8A000A095BA2F880E991EAA1EBB1EC80117FDAF
:10B8B00086C64BE06F850E945114880E991EA11C0C
:10B8C000B11CB7FC7FC68114910431E0A306B1041A
:10B8D0000CF060C58B859C856110BBC50091AE10D6
:10B8E0001091AF1041E16C2D0E945114A801662700
:10B8F00057FD6095762F480F591F611D711D77FD0B
:10B90000AAC64115510531E06307710524F04FEFD8
:10B910005FEF60E070E00D89011104C01F89112301
:10B9200009F48FC68B899C89880F991F2B893C89C4
:10B93000820F931F919581959109AA2797FDA09554
:10B94000BA2F92018101080F191F2A1F3B1F37FDD3
:10B9500096C601151105E1E02E07310524F00FEF21
:10B960001FEF20E030E09801880E991EAA1EBB1E32
:10B97000B7FCA5C681149104F1E0AF06B1042CF028
:10B9800088248A94982CA12CB12C480F591F6A1F27
:10B990007B1F77FD90C64115510501E060077105D9
:10B9A00024F04FEF5FEF60E070E01E89112309F48F
:10B9B000D8C530936F1020936E1090927B108092B8
:10B9C0007A1050938710409386106110FCCE5093EC
:10B9D000631040936210F7CE8091820B882309F4A4
:10B9E000D5CE8091810B282F30E0285131093B8F33
:10B9F0002A8F200F311F4F815885662757FD60958C
:10BA0000762F4B835C836D837E8320908C103090E7
:10BA10008D104101AA2497FCA094BA2C840E951E87
:10BA2000A61EB71E89819A816A8D7B8D860F971F0E
:10BA300097FDB3C540E06D85288F398F0E94511462
:10BA400014012501280E391E411C511C288D398DE9
:10BA500057FCEAC52114310471E0470651040CF08B
:10BA6000B4C48090981090909910AA2497FCA09448
:10BA7000BA2C8B819C81AD81BE81880E991EAA1E35
:10BA8000BB1EE989FA89CF01AA2797FDA095BA2F95
:10BA9000880E991EAA1EBB1EC90137FD81C546E04E
:10BAA0006F850E945114880E991EA11CB11CB7FC11
:10BAB0007AC581149104F1E0AF06B1040CF07BC4A7
:10BAC0008B859C856110A7C42091A4103091A5108E
:10BAD0004CE06C2D288F398F0E945114288D398DA0
:10BAE000A901662757FD6095762F480F591F611DE4
:10BAF000711D77FDA8C54115510521E0620771054B
:10BB000024F04FEF5FEF60E070E03D89311103C03A
:10BB10003F893323C9F12B893C89C901AA2797FDA5
:10BB2000A095BA2F280E391E4A1E5B1E57FCBFC5B2
:10BB30002114310431E0430651042CF022242A94CC
:10BB4000322C412C512C880E991EAA1EBB1EB7FC0C
:10BB5000AAC581149104E1E0AE06B1042CF088245A
:10BB60008A94982CA12CB12C480F591F6A1F7B1F57
:10BB700077FD95C541155105F1E06F07710524F07A
:10BB80004FEF5FEF60E070E02E892111C4C4309266
:10BB900041102092401090924D1080924C10509382
:10BBA000591040935810F2CD8091AE0B882309F4C0
:10BBB00005CE8091AD0B282F30E0285131093B8F05
:10BBC0002A8F200F311F4F815885662757FD6095BA
:10BBD000762F4B835C836D837E832090941030900E
:10BBE00095104101AA2497FCA094BA2C840E951EAE
:10BBF000A61EB71E89819A816A8D7B8D860F971F3D
:10BC000097FD16C544E06D85288F398F0E94511429
:10BC100014012501280E391E411C511C288D398D17
:10BC200057FCC9C42114310471E0470651040CF0DB
:10BC3000ECC38090A0109090A110AA2497FCA0942F
:10BC4000BA2C8B819C81AD81BE81880E991EAA1E63
:10BC5000BB1EE989FA89CF01AA2797FDA095BA2FC3
:10BC6000880E991EAA1EBB1EC90137FDBEC44AE03C
:10BC70006F850E945114880E991EA11CB11CB7FC3F
:10BC8000B7C481149104F1E0AF06B1040CF0B3C362
:10BC90008B859C856110CEC32091AC103091AD1086
:10BCA00040E16C2D288F398F0E945114288D398DD9
:10BCB000A901662757FD6095762F480F591F611D12
:10BCC000711D77FDCCC44115510521E06207710556
:10BCD00024F04FEF5FEF60E070E03D89311103C069
:10BCE0003F893323F1F18B899C89880F991F2B8918
:10BCF0003C89820F931FAA2797FDA095BA2F280E83
:10BD0000391E4A1E5B1E57FCE2C42114310431E087
:10BD1000430651042CF022242A94322C412C512C1D
:10BD2000880E991EAA1EBB1EB7FCCDC481149104B7
:10BD3000E1E0AE06B1042CF088248A94982CA12C62
:10BD4000B12C480F591F6A1F7B1F77FD94C4411502
:10BD50005105F1E06F07710524F04FEF5FEF60E0F0
:10BD600070E02E89211106C43092491020924810AB
:10BD7000909255108092541050936110409360102F
:10BD80001DCD8091A30B882309F412CD8091A20BC5
:10BD9000282F30E0285131093B8F2A8F200F311F87
:10BDA0004F815885662757FD6095762F4B835C83BE
:10BDB0006D837E8320909210309093104101AA24CD
:10BDC00097FCA094BA2C840E951EA61EB71E8981DE
:10BDD0009A816A8D7B8D860F971F97FD2CC443E057
:10BDE0006D85288F398F0E94511414012501280E6A
:10BDF000391E411C511C288D398D57FCEBC3211471
:10BE0000310471E0470651040CF0EFC280909E109F
:10BE100090909F10AA2497FCA094BA2C8B819C81AF
:10BE2000AD81BE81880E991EAA1EBB1EE989FA89C2
:10BE3000CF01AA2797FDA095BA2F880E991EAA1E9A
:10BE4000BB1EC90137FDCAC349E06F850E9451146A
:10BE5000880E991EA11CB11CB7FCC3C381149104A8
:10BE6000F1E0AF06B1040CF0B6C28B859C85611081
:10BE7000FFC22091AA103091AB104FE06C2D288F9B
:10BE8000398F0E945114288D398DA901662757FDDD
:10BE90006095762F480F591F611D711D77FDE7C30F
:10BEA0004115510521E06207710524F04FEF5FEF66
:10BEB00060E070E03D89311103C02F892223E9F150
:10BEC0008B899C89919581959109880F991FAA2743
:10BED00097FDA095BA2F280E391E4A1E5B1E57FCEF
:10BEE00002C421143104E1E04E0651042CF0222456
:10BEF0002A94322C412C512C880E991EAA1EBB1E4E
:10BF0000B7FCEDC381149104F1E0AF06B1042CF04D
:10BF100088248A94982CA12CB12C480F591F6A1F91
:10BF20007B1F77FDD8C34115510521E062077105DC
:10BF300024F04FEF5FEF60E070E03E893111FEC208
:10BF400030924710209246109092531080925210D7
:10BF500050935F1040935E102BCC8091980B8823F8
:10BF600009F420CC8091970B282F30E0285131091B
:10BF70003B8F2A8F200F311F4F815885662757FD31
:10BF80006095762F4B835C836D837E832090901029
:10BF9000309091104101AA2497FCA094BA2C840EF1
:10BFA000951EA61EB71E89819A816A8D7B8D860F8C
:10BFB000971F97FD28C342E06D85288F398F0E9417
:10BFC000511414012501280E391E411C511C288DC5
:10BFD000398D57FC25C32114310471E04706510403
:10BFE0000CF0CCC180909C1090909D10AA2497FCDE
:10BFF000A094BA2C8B819C81AD81BE81880E991E44
:10C00000AA1EBB1EE989FA89CF01AA2797FDA09530
:10C01000BA2F880E991EAA1EBB1EC90137FDF9C290
:10C0200048E06F850E945114880E991EA11CB11C16
:10C03000B7FCF2C281149104F1E0AF06B1040CF038
:10C0400093C18B859C85611022C22091A8103091EC
:10C05000A9104EE06C2D288F398F0E945114288D25
:10C06000398DA901662757FD6095762F480F591F16
:10C07000611D711D77FDEBC24115510521E062077D
:10C08000710524F04FEF5FEF60E070E03D89311102
:10C0900003C02F892223D1F18B899C89880F991F96
:10C0A000AA2797FDA095BA2F280E391E4A1E5B1E9F
:10C0B00057FC25C321143104E1E04E0651042CF055
:10C0C00022242A94322C412C512C880E991EAA1E0F
:10C0D000BB1EB7FC10C381149104F1E0AF06B1049C
:10C0E0002CF088248A94982CA12CB12C480F591F2D
:10C0F0006A1F7B1F77FDFBC24115510521E06207D6
:10C10000710524F04FEF5FEF60E070E03E89311180
:10C11000EFC13092451020924410909251108092BD
:10C12000501050935D1040935C103CCB80918D0B70
:10C13000882309F431CB80918C0B282F30E02851D3
:10C1400031093B8F2A8F200F311F4F815885662779
:10C1500057FD6095762F4B835C836D837E832090A3
:10C160008E1030908F104101AA2497FCA094BA2C15
:10C17000840E951EA61EB71E89819A816A8D7B8DBD
:10C18000860F971F97FD42C241E06D85288F398F3A
:10C190000E94511414012501280E391E411C511C06
:10C1A000288D398D57FC12C22114310471E04706E5
:10C1B00051040CF0E9C080909A1090909B10AA2432
:10C1C00097FCA094BA2C8B819C81AD81BE81880E96
:10C1D000991EAA1EBB1EE989FA89CF01AA2797FDDD
:10C1E000A095BA2F880E991EAA1EBB1EC90137FD45
:10C1F00003C247E06F850E945114880E991EA11C4E
:10C20000B11CB7FCFCC181149104F1E0AF06B1048C
:10C210000CF0A0C08B859C85611048C12091A610B0
:10C220003091A7104DE06C2D288F398F0E9451144A
:10C23000288D398DA901662757FD6095762F480F07
:10C24000591F611D711D77FD0EC24115510521E079
:10C250006207710524F04FEF5FEF60E070E03D8909
:10C26000311103C02F892223D9F18B899C899195A3
:10C2700081959109AA2797FDA095BA2F280E391EFE
:10C280004A1E5B1E57FC07C221143104E1E04E0632
:10C2900051042CF022242A94322C412C512C880E4B
:10C2A000991EAA1EBB1EB7FCF2C181149104F1E0D5
:10C2B000AF06B1042CF088248A94982CA12CB12CC0
:10C2C000480F591F6A1F7B1F77FDDDC141155105BE
:10C2D00021E06207710524F04FEF5FEF60E070E04E
:10C2E0003E893111F2C03092431020924210909258
:10C2F0004F1080924E1050935B1040935A104CCACE
:10C3000080918315909184158090E5109090E610AF
:10C31000E817F90709F00FCA8091851590918615E5
:10C320004091D7105091D8108816990609F427C269
:10C330008091DD109091DE1020910F11309110113D
:10C340006090C9106091D3106AC9188A1F861E8632
:10C350001D860ACA88248A94982CA12CB12C8B851E
:10C360009C856110A3C05ACF88248A94982CA12C54
:10C37000B12C8B859C8561108AC067CE22242A94BB
:10C38000322C412C512C2ECE22242A94322C412C9A
:10C39000512C11CF88248A94982CA12CB12C8B85F8
:10C3A0009C85662009F49ACA54C022242A94322C0F
:10C3B000412C512C60CA88248A94982CA12CB12C31
:10C3C0008B859C85611027C07FCB22242A94322C38
:10C3D000412C512C46CB88248A94982CA12CB12C2A
:10C3E0008B859C85611044C044CD22242A94322C34
:10C3F000412C512C0BCD88248A94982CA12CB12C43
:10C400008B859C85611016C047CC22242A94322C3F
:10C41000412C512C0ECC41E0641609F47EC18B8571
:10C420009C852A8D3B8D820F931F97FF4DCB80E01B
:10C4300090E04ACB41E0641609F465C18B859C8588
:10C440002A8D3B8D820F931F97FF26CC80E090E0D2
:10C4500023CC41E0641609F488C18B859C852B812F
:10C460003C81820F931F97FF39CA80E090E036CA63
:10C4700031E0631609F465C18B859C852A8D3B8D5F
:10C48000820F931F97FFF5CC80E090E0F2CC31E073
:10C49000631609F44CC18B859C852A8D3B8D820FD8
:10C4A000931F97FFD2CD80E090E0CFCD31E06316AF
:10C4B00009F451C18B859C852A8D3B8D820F931F7A
:10C4C00097FFACCE80E090E0A9CE3092671020922A
:10C4D0006610909273108092721050937F10409368
:10C4E0007E10611059C950935B1040935A1054C983
:10C4F000309269102092681090927510809274109A
:10C50000509381104093801061104CC950935D107E
:10C5100040935C1047C9309265102092641090924D
:10C5200071108092701050937D1040937C106110B8
:10C530002DC9509359104093581028C930926B1050
:10C5400020926A1090927710809276105093831008
:10C550004093821061102CC950935F1040935E107D
:10C5600027C930934B1020934A1090925710809215
:10C5700056102DCA30926D1020926C109092791046
:10C58000809278105093851040938410611016C9E2
:10C59000509361104093601011C980E090E04ACA46
:10C5A00080E090E07CCA812C912C540182CA212C1D
:10C5B000312C210159C9212C312C210133CB80E0B0
:10C5C00090E077C9812C912C54017DC9212C312C0C
:10C5D0002101EACD212C312C210111CC80E090E009
:10C5E00033CC812C912C540139CC80E090E03FCBAE
:10C5F000812C912C540145CB80E090E0FACD812C28
:10C60000912C540100CE80E090E0D5CC80E090E009
:10C61000BBCD80E090E004CD812C912C54010ACD5B
:10C62000212C312C2101D7CC212C312C210112CAF3
:10C6300080E090E0E7CA80E090E0D1CB80E090E03D
:10C6400007C99101B2C940E050E0BA0154CA40E0C4
:10C6500050E0BA0111CD40E050E0BA0152C940E0CB
:10C6600050E0BA0130CB40E050E0BA01EECD40E0FE
:10C6700050E0BA0115CC40E050E0BA0168CB00E0D0
:10C6800010E0980166C940E050E0BA011FCE812C4D
:10C69000912C54010ACE212C312C2101F5CD40E002
:10C6A00050E0BA0167CA812C912C540152CA212C46
:10C6B000312C21013DCA40E050E0BA016CC9812C07
:10C6C000912C540157C9812C912C54012FCB212C32
:10C6D000312C21011ACB40E050E0BA0124CC812C4E
:10C6E000912C54010FCC212C312C2101FACB40E0AC
:10C6F00050E0BA0101CD812C912C5401ECCC212CBD
:10C70000312C2101D7CC8A8D9B8D97FD55C09C0182
:10C71000359527953B8F2A8F91CE8A8D9B8D97FDDE
:10C720004DC09C01359527953B8F2A8F78CE8A8DF9
:10C730009B8D97FD45C09C01359527953B8F2A8F92
:10C74000AACE8A8D9B8D97FD3FC09C01359527957C
:10C750003B8F2A8F91CE8A8D9B8D97FD33C09C0194
:10C76000359527953B8F2A8FA5CE8B819C8197FD90
:10C770002DC08C01159507951C830B836ECE80917F
:10C780008715909188154817590709F0D1CD8091E8
:10C79000DD109091DE102091891530918A15821755
:10C7A0009307B1F020910F11309110116090C910D2
:10C7B0006091D3100C940F5B0196A9CF0196B1CF75
:10C7C0000196B9CF0196CBCF0196BFCF0196D1CFBD
:10C7D00020910F113091101160918B1570918C1573
:10C7E0006090C9102617370721F06091D3100C9480
:10C7F0000F5B60918D156612F8CF6091D310709128
:10C800008E1567130C940F5B0C94E35B7F928F92F1
:10C810009F92AF92BF92CF92DF92EF92FF920F93CF
:10C820001F93CF93DF9300D0CDB7DEB71A82198262
:10C83000C12CD12C08C08FEFC81AD80A84E6C816BC
:10C84000D10409F468C0C6010E94251B882399F30E
:10C85000BE016F5F7F4FC6010E94C01AE980FA8057
:10C860007FB6F89481E0E81AF108F594E794F5941E
:10C87000E7948FEFE81AF80A0E9446290E94175998
:10C880000E94B7250E94F2250E942D261E141F0427
:10C89000BCF500E010E0F801EE0FFF1FEE0FFF1FE8
:10C8A000EE56F84E8080A1809280B380882D8F77DD
:10C8B0000E9469258A2D8F770E946925892D8F779F
:10C8C0000E9469258B2D8F770E946925992D92955D
:10C8D000969594703A2D3295369536953270932B05
:10C8E0002B2D22952870922B882D881F8827881F32
:10C8F000892B0E9469250F5F1F4F0E151F055CF2E3
:10C900000E9468267FBE8FEFC81AD80A84E6C81630
:10C91000D10409F098CF0F900F90DF91CF911F9124
:10C920000F91FF90EF90DF90CF90BF90AF909F90CE
:10C930008F907F900895CF92DF92FF920F931F9375
:10C94000CF93DF9300D0CDB7DEB78C01FFB67A83EB
:10C9500069830E946A1A5A8169818823E1F0EFE8AD
:10C96000F5E120E032E0DF01C9011D920197E9F70E
:10C97000C62ED52E27E937E1462FB901CF010E94F7
:10C980006576C60181579A4E9093901780938F17C2
:10C99000C8010E9437208F2D0F900F90DF91CF910B
:10C9A0001F910F91FF90DF90CF900C942E1A2F9231
:10C9B0003F924F925F926F927F928F929F92AF922F
:10C9C000BF92CF92DF92EF92FF920F931F93CF937C
:10C9D000DF93CDB7DEB7C958D1090FB6F894DEBFE3
:10C9E0000FBECDBF839709F0F6C2809192178130B8
:10C9F00009F0F1C280919317823009F0ECC22091C6
:10CA00009417AE962FAFAE97243608F0E4C2DE013D
:10CA1000A35ABF4F80E090E09C012E56384EF9019A
:10CA20004481F0E14F9FA0011124F90123812F706F
:10CA3000242B2D9302968032910571F7A3962FAD8A
:10CA4000A397922F9295969596959370A4964FAD35
:10CA5000A497842F8F70880F880F892B982E990C9C
:10CA6000990C812CB40160957095E0967FAF6EAF04
:10CA7000E097A2968FADA297A82EA694AA0CAA0C16
:10CA8000A1963FADA197932F969596959695FF24E5
:10CA9000F394F822F294FF0CB0EEFB22F92AFF0C7B
:10CAA000FF0C582F551F5527551F2F73220F922FFC
:10CAB000952B80E0BC017058E2967FAF6EAFE29795
:10CAC0006E968FAD6E97782F770FCF57DF4F7883A5
:10CAD000C158D040AB962FADAB97922F9E7FCE57CB
:10CAE000DF4F9883C258D04042954F70A5969FADB6
:10CAF000A59717E0D12ED922D29400EFD022D42AC4
:10CB0000492F469546954695A6969FADA697092F1F
:10CB100001700295000F007E042B000F000F692F9B
:10CB2000660F660F562F587740E0BA017058E496AA
:10CB30007FAF6EAFE497492F429546954770A79611
:10CB40009FADA797A92FA170AA0FAA0FAA0FA42B78
:10CB5000B0E0A55AB84F7C91EC967FAFEC97B92E18
:10CB6000B694B29440EFB422492F4295469547704F
:10CB7000A8969FADA897A92FA170AA0FAA0FAA0FD8
:10CB8000A42BB0E0A55AB84F4C91ED964FAFED975E
:10CB9000A92FA695AF70B0E0A55AB84F6C91EE964C
:10CBA0006FAFEE97492F429546954770A9969FAD76
:10CBB000A997A92FA170AA0FAA0FAA0FA42BB0E0C2
:10CBC000A55AB84F7C91EF967FAFEF97C92EC694C8
:10CBD000C29450EFC522929596959770AA964FAD44
:10CBE000AA97A42FA170AA0FAA0FAA0FA92BB0E091
:10CBF000A55AB84F9C91C158DF4F9883CF57D0406A
:10CC0000A42FA695AF70B0E0A55AB84F6C91C0584C
:10CC1000DF4F6883C058D040881F8827881F6F96D1
:10CC20005FAD6F97652F6770660F682B962F990F12
:10CC3000990F990F80E0BC017058E6967FAF6EAFF8
:10CC4000E697952F991F9927991FA0968FADA097CA
:10CC5000182F1F73110F192B110F952F96959C7379
:10CC600082958695869583703770330F330F382BF6
:10CC700080E1389FB0011124E8967FAF6EAFE8974E
:10CC80004295469547702170220F220F220F242BC8
:10CC900040E050E029F0522F550F550F40E050541E
:10CCA000AD964FACAD97742D717041FA662760F95F
:10CCB000AC968FADAC97282F2170E9962FAFE997EE
:10CCC00043FA332730F9EA963FAFEA9744FA33271D
:10CCD00030F981FB222720F942FA222420F845FA74
:10CCE000332430F846FA442440F884FB552450F8A5
:10CCF00086FBEE27E0F9F0E0EE0FFF1F87FBEE2446
:10CD0000E0F8EE0CEE0CEE2A85FBEE27E0F9EE2AB9
:10CD100083FB662460F882FF02C082E001C080E0ED
:10CD2000680EAD967FACAD9777FA772470F88FB721
:10CD3000EB968FAFEB97CA57DF4F2883C658D0408A
:10CD4000CB57DF4F3883C558D040C957DF4F488392
:10CD5000C758D040C857DF4F5883C858D040CC5729
:10CD6000DF4F6883C458D040CD57DF4F7883C35816
:10CD7000D040C757DF4F9883C958D0400E942B1A24
:10CD8000CA57DF4F2881C658D040CB57DF4F388174
:10CD9000C558D040C957DF4F4881C758D040C85701
:10CDA000DF4F5881C858D040CC57DF4F6881C458F6
:10CDB000D040CD57DF4F7881C358D040C757DF4FA1
:10CDC0009881C958D040882309F4E7C08CE5EDEB81
:10CDD000F0E1DE01119601900D928A95E1F77093D2
:10CDE000BD106093BE10E9966FADE9976093BF10D8
:10CDF000EA967FADEA977093C0103093C1102093EC
:10CE0000C2102092C3103092C4104092C5105092AC
:10CE1000C6101092C710E092C8106092C91010920C
:10CE2000CA1081E08093CB101092CC107092CE107B
:10CE30001092CF1023E02093D0108093D11022E0E5
:10CE40002093D2108093D3108093D6101092D710D5
:10CE5000A092D810E0962EAD3FADE0973093DA1057
:10CE60002093D9101092DB10CF57DF4F3881C15873
:10CE7000D0403093DC101092DD10F092DE109092D2
:10CE8000E0108092DF101092E110CE57DF4F6881E2
:10CE9000C258D0406093E210E2962EAD3FADE297CB
:10CEA0003093E4102093E3101092E510D092E61036
:10CEB0001092E7100093E810E4966EAD7FADE49712
:10CEC0007093EA106093E9101092EB10EC967FAD2E
:10CED000EC977093EC101092ED10B092EE1010924F
:10CEE000EF10ED962FADED972093F0101092F1100A
:10CEF000EE963FADEE973093F2101092F310EF964E
:10CF00006FADEF976093F4101092F510C092F61089
:10CF10001092F710C158DF4F7881CF57D0407093EF
:10CF2000F8101092F910C058DF4F2881C058D04037
:10CF30002093FA10E6966EAD7FADE6977093FC10E5
:10CF40006093FB101092FD101093FE101092FF10D2
:10CF500090930011E8962EAD3FADE8973093021103
:10CF60002093011150930411409303111092061164
:10CF7000109205111092081110920711AE968FAD04
:10CF8000AE9790E00E9448208CE5FE013196ADEB13
:10CF9000B0E101900D928A95E1F7EB968FADEB979A
:10CFA000C757DF4F0FB6F894DEBF0FBECDBFDF917E
:10CFB000CF911F910F91FF90EF90DF90CF90BF9096
:10CFC000AF909F908F907F906F905F904F903F9029
:10CFD0002F900C94291AC757DF4F0FB6F894DEBF75
:10CFE0000FBECDBFDF91CF911F910F91FF90EF90BA
:10CFF000DF90CF90BF90AF909F908F907F906F9079
:10D000005F904F903F902F9008952F923F924F92B4
:10D010005F926F927F928F929F92AF92BF92CF92C8
:10D02000DF92EF92FF920F931F93CF93DF93803F96
:10D0300009F440C0873FB1F02091CB0B3091CC0B6D
:10D04000211592E039070CF456C041E050E020E091
:10D0500030E0F901EE56F84E80835093CC0B4093AC
:10D06000CB0B36C080919217813009F448C08111F2
:10D0700009C080919317813629F4809194178631E5
:10D0800009F448C01092CC0B1092CB0BDF91CF91DA
:10D090001F910F91FF90EF90DF90CF90BF90AF90D6
:10D0A0009F908F907F906F905F904F903F902F90C8
:10D0B0000C94874E1092CC0B1092CB0B80E092E038
:10D0C000E2E9F7E1DF019C011D9221503040E1F7D8
:10D0D000DF91CF911F910F91FF90EF90DF90CF9054
:10D0E000BF90AF909F908F907F906F905F904F9088
:10D0F0003F902F900895A9014F5F5F4FAACF809175
:10D100009317823009F0BECF8091CB0B9091CC0B5E
:10D110004EDCB8CF80919517813009F0B3CF809164
:10D12000CB0B9091CC0B049765E070E00E9481726C
:10D130001B0177FD72C0E6E9AE2EE7E1BE2EF7E9EE
:10D14000CF2EF7E1DF2EA8E9EA2EA7E1FA2E09E9B2
:10D1500017E12B01440C551C440C551C460E571E60
:10D1600039E0430E511CC4E0D0E084E0682E712CFD
:10D1700072E9872E77E1972E8C0E9D1E44E050E0D9
:10D18000B401C3018E56984E0E946E76D401149657
:10D190002C91B0E82B9FC0011124F5019081982BB0
:10D1A0009083922F92709295990F990F907CD6014F
:10D1B0008C91982B9C93922F94709295990F907EBE
:10D1C000F7018081982B9083822F88708295807FD1
:10D1D000D8019C91892B8C93B4E06B0E711C259621
:10D1E000E4E0AE0EB11CF4E0CF0ED11C24E0E20E60
:10D1F000F11C0C5F1F4FC415D50509F0B9CFC10153
:10D200000296880F991F880F991FBC0165507109FC
:10D210008091961790E08FDB35CF84E090E0F5CFDA
:10D22000EF92FF920F93CF93DF931F92CDB7DEB7AC
:10D230007B016091CB0B7091CC0B6115710529F0CE
:10D24000E61AF70A81E0E81AF108E114F10439F46A
:10D250000F90DF91CF910F91FF90EF900895842F61
:10D260002983D3DE2981E2E0EE16F10488F3822FD0
:10D27000CCDEF2E0EF16F10459F3802F0F90DF912E
:10D28000CF910F91FF90EF90C0CE1F920F920FB6EB
:10D290000F9211240F900FBE0F901F9018951F92A0
:10D2A0000F920FB60F9211240F900FBE0F901F9088
:10D2B00018951F920F920FB60F9211240BB60F9272
:10D2C0002F933F934F935F936F937F938F939F938E
:10D2D000AF93BF93CF93DF93EF93FF9334997CC0C9
:10D2E000CFB7F89456EC51BB469A70EE77B967E029
:10D2F0006AB97DB915B8D0E8D8B96BB91EB8B7E42A
:10D30000B1BB82E08A95F1F700C026B199B18CB12A
:10D3100051BB479A422F46954370E0E82E9F9001FB
:10D320001124422B292F2071422B292F2695269537
:10D330002870422B96959076492B90E0880F991F84
:10D3400084709927482BA7EEA7B9F7EFFAB9E2EE58
:10D35000EDB985E08A95F1F7000047FF54C040FF22
:10D3600052C051BB469A77B96AB97DB915B8D8B9D8
:10D370006BB980E28EB9B1BB82E08A95F1F700C04B
:10D3800026B199B18CB151BB479A622F66956370F3
:10D3900050E8259F90011124622B292F2071622BC8
:10D3A000292F269526952870622B96959076692BC5
:10D3B00090E0880F991F84709927682BA7B9FAB954
:10D3C000EDB985E08A95F1F7000044FD1AC08AE7BF
:10D3D0009AE10E945259CFBFFF91EF91DF91CF9117
:10D3E000BF91AF919F918F917F916F915F914F917D
:10D3F0003F912F910F900BBE0F900FBE0F901F907B
:10D4000018950E940529CFBFE7CF1F920F920FB644
:10D410000F9211240BB60F922F933F934F935F936C
:10D420006F937F938F939F93AF93BF93CF93DF932C
:10D43000EF93FF93CEE6D0E088818D7F888385B31C
:10D44000876085BB78940E944602F8948881826048
:10D450008883FF91EF91DF91CF91BF91AF919F9121
:10D460008F917F916F915F914F913F912F910F908D
:10D470000BBE0F900FBE0F901F901895CF93DF93A8
:10D48000CDB7DEB7AC970FB6F894DEBF0FBECDBFF9
:10D4900020E82093610010926100F89414B817B846
:10D4A0001AB81DB810BA15B8B0EEDB2ED8B81BB834
:10D4B0001EB883EE81BBCC24CA94C4B8D7B817E099
:10D4C000912E9AB8DDB880BB8CE787BD84B58260A9
:10D4D00084BD85B5836085BD80916E008260809338
:10D4E0006E00EC9A06ECB02EB1BA469AD7B89AB84C
:10D4F000DDB815B828B91BB81EB887E4582E51BA44
:10D5000032E03A95F1F700C086B189B18CB1B1BA79
:10D51000479A97EE692E67B837EF732E7AB842EEC6
:10D52000842E8DB852E1E52E5EE0F52E8BEA92E076
:10D53000D701FC011D923197E9F7E9EAF9E0DF0133
:10D540001D922A95E9F781E4E9E2FAE0DF011D92F4
:10D550008A95E9F760E2A62EA092380A85E4E3E313
:10D56000FCE0DF011D928A95E9F786E6EDECFBE031
:10D57000DF011D928A95E9F7C092320C0E94761C59
:10D580008CE591E0EAE6FAE0DF019C011D92215072
:10D590003040E1F78FE38093C30B46E050E06FEF3C
:10D5A00070E08CEB9BE00E947F761092BC0B0E9497
:10D5B00005298FE091E0E3E0FDE0DF019C011D9291
:10D5C00021503040E1F70FEF1FEF1093080E00934A
:10D5D000070E40E850E06FEF70E085E09DE00E94AC
:10D5E0007F7610930A0E0093090E40E850E06FEF2B
:10D5F00070E085E89DE00E947F768BE8E8E7FCE03C
:10D60000DF011D928A95E9F740E850E06FEF70E086
:10D61000CF010E947F761093F90C0093F80CC09212
:10D62000FA0C80E1E9E1F1E1DF011D928A95E9F769
:10D63000C0921A11C0921C118FEF9FEFDC018093F2
:10D640001D1190931E11A0931F11B093201111E092
:10D6500010931B11C09227111092B7191092B9198B
:10D660001092B81980EC80937C1A8AEB99E1909320
:10D670007E1A80937D1A10927B1A10927A1A109259
:10D680009B1910929A1910929F1910929E1910923C
:10D69000A3191092A2191092A5191092A419109210
:10D6A000A7191092A6191092AB191092AA191092EC
:10D6B000AF191092AE191092B1191092B0191092C0
:10D6C000B3191092B21986E395E39093931980935E
:10D6D000921983E099E4909397198093961980EFBB
:10D6E00098E4909399198093981985E59FE1909318
:10D6F00095198093941983EF9DE19093A1198093DC
:10D70000A01983E293E390939D1980939C1980E183
:10D7100099E69093AD198093AC1982EC99E29093BD
:10D72000A9198093A8191092CC0B1092CB0BA09240
:10D73000C80B83E592E19093CA0B8093C90B1092BA
:10D74000C70B1092C60B8AE2EEE0FFE0DF01482E25
:10D750001D924A94E9F7D701E82F1D92EA95E9F75F
:10D76000E8E3FFE0DF01482E1D924A94E9F7ECE37D
:10D77000FEE0DF01482E1D924A94E9F7E2E6FFE061
:10D78000DF01482E1D924A94E9F7E6E6FEE0DF014C
:10D79000482E1D924A94E9F7ECE8FFE0DF01482E9D
:10D7A0001D924A94E9F7E0E9FEE0DF01482E1D9260
:10D7B0004A94E9F7E6EBFFE0DF01482E1D924A9418
:10D7C000E9F7EAEBFEE0DF01482E1D924A94E9F703
:10D7D000E0EEFFE0DF01482E1D924A94E9F7E4EE07
:10D7E000FEE0DF011D928A95E9F78AE090E10E9450
:10D7F0007D1D85E290E10E947D1D61E085E290E162
:10D800000E945E1D64E085E290E10E94CD19B1BAEC
:10D81000469AD7B89AB8DDB815B980E488B91BB86C
:10D82000AEB851BAB2E0BA95F1F700C086B189B18D
:10D830009CB1B1BA479A67B87AB88DB884FDF1C186
:10D840008BED90E00E94251B811106C00E94941B65
:10D850008BED90E00E9448200E94ED1B811104C0D6
:10D860000E94CE1C0E94672181E00E944B23809180
:10D87000310C00E210E0A6E1FA2E0E94062B209166
:10D88000310C203109F4C9C1332727FD30952F5FB2
:10D890003F4F2F71307837FF06C021503109206E7D
:10D8A0003F6F2F5F3F4F822F2093310C01501109A2
:10D8B00021F781E00E94062B80E10E94062B8EE179
:10D8C0000E94062B8DE10E94062BA0900E01B090C5
:10D8D0000F0100911201109113018090100190909E
:10D8E00011019501201B310B2819390940E050E046
:10D8F000C12CD12CE12CE0E8FE2EC701B6010E941C
:10D9000069772093140130931501409316015093C9
:10D9100017019401209530952A193B09201B310BE2
:10D9200040E050E0C701B6010E94697720931801DA
:10D930003093190140931A0150931B010091491231
:10D9400010914A121093010100930001A09004016C
:10D95000B0900501809002019090030198012A196E
:10D960003B092819390940E050E0C701B6010E947F
:10D970006977209306013093070140930801509383
:10D980000901940120953095201B310B2A193B0980
:10D9900040E050E0C701B6010E94697720930A0178
:10D9A00030930B0140930C0150930D010E949F4F47
:10D9B0000E94874E8BE697E00E9488177894F6ECD9
:10D9C0002F2E9FB7F894809173128F5F80937312FC
:10D9D00021BA469A81708D871E864D845E84440CE0
:10D9E000551C440C551C920121633E872D878D8563
:10D9F00086958270806C31E035B942E448B950E5D3
:10DA00005BB98EB987E881BB9FBF1092CD0B109296
:10DA1000CE0B1092CF0B1092D00B9FEF9093320C45
:10DA20008091310C0E94062B2091310C203109F499
:10DA300024C2332727FD30952F5F3F4F2F71307859
:10DA400037FDC5C3822F2093310C0E94062B2091F5
:10DA5000310C203109F40CC2332727FD30952F5F9C
:10DA60003F4F2F71307837FDABC3822F2093310C9D
:10DA70000E94062B2091310C203109F4F4C1332788
:10DA800027FD30952F5F3F4F2F71307837FDABC3A7
:10DA9000822F2093310C0E94062B8091310C803113
:10DAA00009F4DDC1992787FD909501968F719078D3
:10DAB00097FD94C38093310C81E00E94062B80E196
:10DAC0000E94062B8EE10E94062B8DE10E94062B00
:10DAD0009090320C44244A94941002C090901C11EF
:10DAE00090921C1167E1562E951409F42EC14090B6
:10DAF000CD0B5090CE0B6090CF0B7090D00B20913F
:10DB00000E0130910F013A8B298B409112015091F7
:10DB100013015C8B4B8B8091100190911101988BBC
:10DB20008F877C01E094F094241B350B388F2F8B6A
:10DB30009C0140E050E02D8F3E8F4F8F58A3809185
:10DB4000140190911501A0911601B0911701898FD0
:10DB50009A8FAB8FBC8FAB89BC89E989FA89AE0FEC
:10DB6000BF1FBE8BAD8B9D0140E050E02DA33EA3B7
:10DB70004FA358A78091180190911901A0911A0103
:10DB8000B0911B0189A39AA3ABA3BCA390911B11D5
:10DB900080914D1200E916E037EDA32E30E1B32E4F
:10DBA000882309F417C1C92CDD24C7FCD094392C73
:10DBB0002BC0E82FFF27E7FDF095B301A201082E47
:10DBC00004C076956795579547950A94D2F740FF1C
:10DBD00014C0EE0FFF1FEF50F44F808091800E9421
:10DBE000651C882331F0E814F904E8F488248A9449
:10DBF000982CF5019182808291E0A2E0AA0EB11CDE
:10DC0000B6E00E3A1B0779F1D8018D918D018F3F57
:10DC1000A1F38311CECFF601DCCFF092310C86E177
:10DC200045CE0E94C9562F8538898216930608F47E
:10DC30007FC0A40160E070E08F89988D88169906F6
:10DC400008F079C09A01AB018D8D9E8DAF8DB8A182
:10DC5000281B390B4A0B5B0B698D7A8D8B8D9C8D44
:10DC600035D44C01C6CF90931B11FFEF3F1609F43A
:10DC70004CC0E32DEE0FFF0BEF50F44F00811181EC
:10DC8000A80160E070E080911D1190911E11A0919B
:10DC90001F11B0912011481759076A077B07A9F196
:10DCA00040931D1150931E1160931F11709320110A
:10DCB0001093221100932111832D09A75AA76BA756
:10DCC0007CA70E94651C49A55AA56BA57CA5882345
:10DCD00071F08F859889809590958017910708F04D
:10DCE00000C38FEF9FEF90932211809321110E9428
:10DCF0005F3580911C11863109F413C3803109F41A
:10DD000021C38450883008F4E9C210917312137053
:10DD1000123009F426C1133009F4D0C0113009F4CF
:10DD2000C7C10E9426326FEF80E00E94D55A49CECB
:10DD3000812C912C5ECFAD89BE89A815B90508F458
:10DD4000ABC0812C90E8992E54CFE0912711E7FDCC
:10DD5000CECE20911F0C3091200C2901612C712C0A
:10DD600080911D1190911E11A0911F11B091201151
:10DD7000481659066A067B0609F4B9CEFF27E7FD67
:10DD8000F095CF01880F991F8E0F9F1F880F991F45
:10DD9000880F991F80569A4F1CE0FC01DE011196F6
:10DDA00001900D921A95E1F7DC010C9111961C91EE
:10DDB000011132C2E12FEE0FFF0BE952FF4E31830A
:10DDC00020835524539450921B110E94874E9090AB
:10DDD0001C118DCE392C8F88988CCF84D8880FC099
:10DDE00066246A94762CD5016D927C9291E0B2E023
:10DDF000AB0EB11CE6E00E3A1E0709F434CFF80171
:10DE000081918F018F3F99F3E82FEE0FFF0BEF50B9
:10DE1000F44F608071800E94651C882321F3E61412
:10DE2000F704F0F26C147D04B8F0C301A0E0B0E098
:10DE30006814790438F59C01AD014D8C5E8C6F8CB3
:10DE400078A02419350946095709698D7A8D8B8D7B
:10DE50009C8D3CD33C01C7CF612C712CC4CFF6E123
:10DE6000F093310C29CEE6E1E093310C86E113CE3C
:10DE7000B6E1B093310C86E1FBCDA6E1A093310C65
:10DE800086E1E3CD4D885E884614570408F4B2C19C
:10DE9000612C80E8782EA7CF9A01AB018DA19EA1BD
:10DEA000AFA1B8A5281B390B4A0B5B0B69A17AA15E
:10DEB0008BA19CA10BD390584C019BCE0E94B639EC
:10DEC00000E010E423E035E440E050EE6BE276E45D
:10DED00080910311909104110E94FB189C01909372
:10DEE000B3108093B21081E0203D37400CF080E009
:10DEF0008093B41080911111909112118115A4E0BA
:10DF00009A0708F4E0C120915112222309F449C272
:10DF1000AC0160E070E0DB01CA01880F991FAA1F05
:10DF2000BB1F880F991FAA1FBB1F880F991FAA1F0D
:10DF3000BB1F840F951FA61FB71F880F991FAA1F0D
:10DF4000BB1FFD01EE0FFF1FE255F94F808191814C
:10DF50009093000D8093FF0C9093110E8093100E00
:10DF6000E2CE8091D9109091DA10EFB6F8940E9429
:10DF7000CE1221BA469A4424439445B883E488B922
:10DF800000EF0BB910EA1EB977E8572E51BA25E019
:10DF90002A95F1F7000021BA469A45B888B9E0E71A
:10DFA000FE2EFBB81EB951BA3AE03A95F1F700C01F
:10DFB00021BA469A45B888B90BB91EB951BA4AE098
:10DFC0004A95F1F700C0EFBE8091DF109091E0100C
:10DFD000EFB6F8940E94CE1221BA469A45B885E46D
:10DFE00088B90BB91EB951BA55E05A95F1F700003E
:10DFF00021BA469A45B888B9FBB81EB951BA9AE019
:10E000009A95F1F700C021BA469A45B888B90BB97C
:10E010001EB951BAAAE0AA95F1F700C0EFBE20914F
:10E020000D0C30910E0C8091B0109091B110AA2778
:10E0300097FDA095BA2F820F931FA11DB11DB7FDAB
:10E040006CC11FB7F8940097E1E0AE07B10524F06A
:10E050008FEF9FEFA0E0B0E00E94CE1221BA469A67
:10E06000F1E0F5B997E498B920EF2BB980EA8EB9C1
:10E0700067E8462E41BA35E03A95F1F7000021BA3B
:10E08000469AF5B998B930E73BB98EB941BA4AE03A
:10E090004A95F1F700C021BA469AF5B998B92BB95B
:10E0A0008EB941BA5AE05A95F1F700C01FBF3BCE76
:10E0B0008091FD109091FE100FB7F8940E94CE123F
:10E0C00021BA469A15B991E498B9F0EFFF2EFBB842
:10E0D00080EA8EB9A7E87A2E71BA25E02A95F1F781
:10E0E000000021BA469A15B998B9B0E7EB2EEBB803
:10E0F0008EB971BA3AE03A95F1F700C021BA469A62
:10E1000015B998B9FBB88EB971BA4AE04A95F1F7DA
:10E1100000C00FBF8091E7109091E810DFB6F8942F
:10E120000E94CE1221BA469A15B985E488B9FBB887
:10E1300002EA0EB971BA55E05A95F1F7000021BA1A
:10E14000469A15B988B9EBB80EB971BA9AE09A95A2
:10E15000F1F700C021BA469A15B988B9FBB80EB9D3
:10E1600071BAAAE0AA95F1F700C0DFBEDFB6F89455
:10E1700080E090E60E94CE1221BA469A15B983E457
:10E1800088B9FBB80EB971BAB5E0BA95F1F70000DD
:10E1900021BA469A15B988B9EBB80EB971BAEAE056
:10E1A000EA95F1F700C021BA469A15B988B9FBB8CB
:10E1B0000EB971BAFAE0FA95F1F700C0DFBEB3CD3F
:10E1C00021503109206E3F6F2F5F3F4F4ECC2150C1
:10E1D0003109206E3F6F2F5F3F4F34CC0197806E27
:10E1E0009F6F019667CC21503109206E3F6F2F5FE2
:10E1F0003F4F4ECC9C01AD014DA05EA06FA078A416
:10E20000241935094609570969A17AA18BA19CA156
:10E210005DD190583C01E7CD033008F0D2CD0E948B
:10E22000E2188D819E81892B09F423C18F81988505
:10E23000892B09F42EC189859A85892B09F41DC182
:10E240008B859C85892B09F404C1B301A201440F7D
:10E25000551F661F771F440F551F661F771F6B01E1
:10E26000FF24D7FCF094EF2C80912311909124117E
:10E27000A0912511B0912611C816D906EA06FB0611
:10E2800079F0F6013296EE0FFF1F44244394512C8F
:10E290004C0E5D1EE40DF51D808191810E94881752
:10E2A000013009F078C0E12FFF27E7FDF095E35436
:10E2B000FF4EC082C0922311D0922411E09225110A
:10E2C000F09226117ECDEFEFFFEFF093000DE0937B
:10E2D000FF0CF093110EE093100E25CD0E941E4905
:10E2E00014CD4F8458880415150508F46DC089892C
:10E2F0009A896B887C88861997090817190708F08E
:10E3000066C09A01AB012419350941095109698D8B
:10E310007A8D8B8D9C8DDAD0E6CC80E090E0DC01AC
:10E3200090CE00911D0C10911E0C1093891000933B
:10E3300088100E94263242E0B80180E090E00E94FE
:10E340005839E3CC8091110C9091120CE0910001AE
:10E35000F0910101A0910401B091050160910201C9
:10E36000709103019B012095309528173907D0F54E
:10E370000FEF1FE710938B1000938A100E94D115A6
:10E380006FEF81E00E94D55A41E060E070E0C80183
:10E390000E945839BACCB701A601812F0E94E533FB
:10E3A00089CF00E010E02AEF33E440E050EE6BEA62
:10E3B00076E40E94FB189093000D8093FF0C9093DD
:10E3C000110E8093100EAFCC80E090E08CCCC30196
:10E3D00069887A88860D971D8017910708F180E07B
:10E3E00090E881CC8617970788F16C01E12CF12C1D
:10E3F0008F010A1B1B0B80179107F8F4A7019601E8
:10E40000261B370B410951096091060170910701E4
:10E41000809108019091090159D08C011058AACF20
:10E420009A01AB01281B390B4109510969A17AA155
:10E430008BA19CA14BD0905856CCBD016E0F7F1F75
:10E440006817790760F100E010E094CF00E010E871
:10E4500091CF73016201CC0CDD1CEE1CFF1CC40CBF
:10E46000D51CE61CF71C6701FF24D7FCF094EF2CA9
:10E47000FBCEC12CD12C7601F7CEB301A201440F03
:10E48000551F661F771F6B01FF24D7FCF094EF2CFC
:10E49000EBCE6301FF24D7FCF094EF2CE5CEA7016F
:10E4A0009601261B370B4109510960910A017091B1
:10E4B0000B0180910C0190910D0108D09058ADCFC7
:10E4C000FCD4B7FF0895821B930B0895DB018F9353
:10E4D0009F93B4D4BF91AF91A29F800D911DA39F34
:10E4E000900DB29F900D11240895991B79E004C0FE
:10E4F000991F961708F0961B881F7A95C9F7809583
:10E50000089597FB072E16F4009406D077FD08D0E7
:10E51000A5D407FC05D03EF4909581959F4F0895B2
:10E52000709561957F4F08955058BB27AA270ED04C
:10E53000C9C192D130F097D120F031F49F3F11F44E
:10E540001EF462C10EF4E095E7FB58C1E92FDCD15F
:10E5500080F3BA17620773078407950718F071F400
:10E560009EF5F4C10EF4E0950B2EBA2FA02D0B01F1
:10E57000B90190010C01CA01A0011124FF27591B08
:10E5800099F0593F50F4503E68F11A16F040A22F0E
:10E59000232F342F4427585FF3CF4695379527957F
:10E5A000A795F0405395C9F77EF41F16BA0B620B7E
:10E5B000730B840BBAF09150A1F0FF0FBB1F661FC5
:10E5C000771F881FC2F70EC0BA0F621F731F841F08
:10E5D00048F4879577956795B795F7959E3F08F02E
:10E5E000B3CF9395880F08F09927EE0F97958795ED
:10E5F000089541D1E39577C10CD064C134D140F086
:10E600002BD130F021F45F3F19F0F8C051119FC1B8
:10E61000FBC07AD198F39923C9F35523B1F3951B25
:10E62000550BBB27AA2762177307840738F09F5F33
:10E630005F4F220F331F441FAA1FA9F333D00E2EA2
:10E640003AF0E0E830D091505040E695001CCAF70F
:10E6500029D0FE2F27D0660F771F881FBB1F2617D4
:10E6600037074807AB07B0E809F0BB0B802DBF01A7
:10E67000FF2793585F4F2AF09E3F510568F0BEC0B8
:10E6800066C15F3FECF3983EDCF38695779567951E
:10E69000B795F7959F5FC9F7880F911D9695879558
:10E6A00097F90895E1E0660F771F881FBB1F621777
:10E6B00073078407BA0720F0621B730B840BBA0B35
:10E6C000EE1F88F7E095089519F40EF097C03EC14B
:10E6D0009BC022D1C8F39638C0F707F80F92E89490
:10E6E0002BE33AEA48EB5FE7BAD10F920F920F9211
:10E6F0004DB75EB70F9272D1ECEAF0E088D04F913F
:10E700005F91EF91FF91E595EE1FFF1F49F0FE57D6
:10E71000E0684427EE0F441FFA95E1F74195550B49
:10E7200029D10F9007FE1DC10895F6D088F09F579C
:10E7300090F0B92F9927B751A0F0D1F0660F771F4D
:10E74000881F991F1AF0BA95C9F712C0B13081F02D
:10E75000FDD0B1E00895FAC0672F782F8827B85F01
:10E7600039F0B93FCCF3869577956795B395D9F78E
:10E770003EF490958095709561957F4F8F4F9F4F98
:10E780000895E89409C097FB3EF4909580957095A4
:10E7900061957F4F8F4F9F4F9923A9F0F92F96E9ED
:10E7A000BB279395F695879577956795B795F11162
:10E7B000F8CFFAF4BB0F11F460FF1BC06F5F7F4FFF
:10E7C0008F4F9F4F16C0882311F096E911C0772311
:10E7D00021F09EE8872F762F05C0662371F096E81A
:10E7E000862F70E060E02AF09A95660F771F881FE9
:10E7F000DAF7880F9695879597F9089597F99F67A7
:10E8000080E870E060E008959FEF80EC0895DF936A
:10E81000CF931F930F93FF92EF92DF927B018C01B6
:10E82000689405C0DA2EEF0118D1FE01E894A59195
:10E830002591359145915591AEF3EF0187DEFE01AB
:10E840009701A801DA9479F7DF90EF90FF900F918C
:10E850001F91CF91DF91089500240A941616170690
:10E8600018060906089500240A94121613061406C1
:10E8700005060895C9CF50D0E8F3E894E0E0BB273F
:10E880009F57F0F02AED3FE049EC06C0EE0FBB0FBA
:10E89000661F771F881F28F0B23A62077307840744
:10E8A00028F0B25A620B730B840BE3959A9572F7BA
:10E8B000803830F49A95BB0F661F771F881FD2F7F8
:10E8C000904894C1092E0394000C11F4882352F04F
:10E8D000BB0F40F4BF2B11F460FF04C06F5F7F4F8C
:10E8E0008F4F9F4F0895EF93E0FF06C0A2EA2AEDF5
:10E8F0003FE049EC5FEB2ADEE5DF0F90039401FC7B
:10E900009058E4EDF0E07EC157FD9058440F551F3C
:10E9100059F05F3F71F04795880F97FB991F61F0A1
:10E920009F3F79F087950895121613061406551F18
:10E93000F2CF4695F1DF08C0161617061806991F84
:10E94000F1CF86957105610508940895E894BB2779
:10E9500066277727CB0197F9089522D108F48FEF26
:10E9600008959B01AC0160E070E080E89FE344CE35
:10E9700045CF3AC1D1DFE8F39923D9F3940F511D64
:10E98000BBF39150504094F059F0882332F0660F59
:10E99000771F881F91505040C1F79E3F510544F7A3
:10E9A000880F911D9695879597F908955F3FACF074
:10E9B000983E9CF0BB27869577956795B79508F4A8
:10E9C000B1609395C1F7BB0F58F711F460FFE8CF22
:10E9D0006F5F7F4F8F4F9F4FE3CFB9CFFA01DC01BD
:10E9E000AA0FBB1F9B01AC01BF5728F42227332776
:10E9F000442750781FC0B75188F4AB2F00244695A8
:10EA000037952795011CA395D2F3002069F0220FBA
:10EA1000331F441FB395DAF30DD086CD61307105F5
:10EA2000A0E88A07B94630F49B01AC016627772736
:10EA300088279078309621F0208331834283538356
:10EA400008950BD03FCF08DF28F00DDF18F0952395
:10EA500009F0D4CED9CE11247ACF56DFA0F3959FFA
:10EA6000D1F3950F50E0551F629FF001729FBB27B5
:10EA7000F00DB11D639FAA27F00DB11DAA1F649F61
:10EA80006627B00DA11D661F829F2227B00DA11D14
:10EA9000621F739FB00DA11D621F839FA00D611D9A
:10EAA000221F749F3327A00D611D231F849F600DBB
:10EAB000211D822F762F6A2F11249F5750408AF0F4
:10EAC000E1F088234AF0EE0FFF1FBB1F661F771F80
:10EAD000881F91505040A9F79E3F510570F08ECE8F
:10EAE00036CF5F3FECF3983EDCF3869577956795DC
:10EAF000B795F795E7959F5FC1F7FE2B880F911D9E
:10EB00009695879597F90895FA01EE0FFF1F3096B5
:10EB10002105310599F16115710561F48038BFE374
:10EB20009B0749F168949038810561F08038BFEF08
:10EB30009B0741F0992342F5FF3FE105310521058F
:10EB400011F1E8940894E795D901AA2329F4AB2F91
:10EB5000BE2FF85FD0F310C0FF5F70F4A695E0F70A
:10EB6000F73950F019F0FF3A38F49F779F930CD0A3
:10EB70000F9007FC905808953EF046CE60E070E09C
:10EB800080E89FE308954FE79F775F934F933F930C
:10EB90002F934ED02F913F914F915F9152DF99CD9E
:10EBA000990F0008550FAA0BE0E8FEEF161617069E
:10EBB000E807F907C0F012161306E407F50798F006
:10EBC000621B730B840B950B39F40A2661F0232B1F
:10EBD000242B252B21F408950A2609F4A140A6959B
:10EBE0008FEF811D811D08959F3F31F0915020F4DA
:10EBF000879577956795B795880F911D9695879519
:10EC000097F908959F938F937F936F93FF93EF935B
:10EC10009B01AC0116DFEF91FF91F9DD2F913F9140
:10EC20004F915F910ECF0EF0DFCFEECD6894E6CD21
:10EC300073DEC8F39923D1F3C6F3DF93CF931F9309
:10EC40000F93FF92C92FDD2788232AF02197660FA3
:10EC5000771F881FDAF720E030E040E85FEB9FE3A2
:10EC6000883920F0803E30F021968F775EDCE2EF2D
:10EC7000F0E003C05ADCEFE1F1E0C9DD8B01BE0139
:10EC8000EC01FB2E6F5771097595771F880B990B57
:10EC90007ADD28E132E741E35FE3DFDEAF2D980163
:10ECA000AE01FF900F911F91CF91DF914FDC0ACE03
:10ECB000FB01DC0104C08D910190801921F44150C9
:10ECC0005040C8F7881B990B0895FB01DC0102C076
:10ECD00001900D9241505040D8F708956817790778
:10ECE00068F4FB01DC01E40FF51FA40FB51F02C09F
:10ECF00002900E9241505040D8F70895E6CFDC01C3
:10ED000001C06D9341505040E0F70895FB01DC01D4
:10ED10000D900020E9F7119701900D920020E1F786
:10ED20000895FB01DC0101900D920020E1F70895A8
:10ED30008F929F92AF92BF92CF92DF92EF92FF920B
:10ED4000CF93DF93EC01688179818A819B81611582
:10ED500071058105910521F464E279ED8BE597E079
:10ED60002DE133EF41E050E08DD049015A019B0184
:10ED7000AC01A7EAB1E462D06B017C01ACEEB4EF68
:10ED8000A501940167D0C60ED71EE81EF91EF7FE36
:10ED900006C081E0C81AD108E10880E8F80AC882F4
:10EDA000D982EA82FB82E894F7F8B601C701DF91C5
:10EDB000CF91FF90EF90DF90CF90BF90AF909F905A
:10EDC0008F900895B5CF8CE991E0B2CF60939C010C
:10EDD00070939D0180939E0190939F010895FB0184
:10EDE0009F01E8944230BCF04532ACF44A3029F43B
:10EDF00097FB1EF4909581959F4F642F77272ED017
:10EE0000805D8A330CF0895D8193CB010097A9F76F
:10EE100016F45DE251931082C90100C0DC01FC01CF
:10EE2000672F71917723E1F7329704C07C916D933E
:10EE300070836291AE17BF07C8F308953ED0A59FB7
:10EE4000900DB49F900DA49F800D911D11240895E5
:10EE5000B7FFF4CFF3DF821B930B0895AA1BBB1BF4
:10EE600051E107C0AA1FBB1FA617B70710F0A61BCA
:10EE7000B70B881F991F5A95A9F780959095BC01EB
:10EE8000CD010895052E97FB16F4009406D057FD8A
:10EE90000CD01FD007FC09D07EF49095809570951A
:10EEA00061957F4F8F4F9F4F0895509540953095B6
:10EEB00021953F4F4F4F5F4F0895A29FB001B39FE1
:10EEC000C001A39F01D0B29F700D811D1124911D1F
:10EED0000895A1E21A2EAA1BBB1BFD010DC0AA1F9B
:10EEE000BB1FEE1FFF1FA217B307E407F50720F0B3
:10EEF000A21BB30BE40BF50B661F771F881F991F2E
:10EF00001A9469F760957095809590959B01AC0176
:0AEF1000BD01CF010895F894FFCF72
:10EF1A0000809001000C000000000000000000804A
:10EF2A0000000008000000000000000000000000CF
:10EF3A0000000000000000000000000000000000C7
:10EF4A00000000000000000000000000003022362F
:10EF5A006D247D20390F7646104010523F065B4FD4
:10EF6A00666D7D077F6F4848614843277B777F3905
:10EF7A003F79713D76060E763837373F733F776DA6
:10EF8A00783E3E7E76665B39640F230802777C58AA
:10EF9A005E79716F74040C743837545C7367506D02
:10EFAA00781C1C7E766E5B39300F01000100000070
:10EFBA0000006207640E3415D21B41228128942E68
:10EFCA007B34383ACB3F37457B4A994F925467593D
:10EFDA001A5EAB621A676A6B9B6FAD73A2777B7B13
:10EFEA00387FD9826186CF89258D629088939896D9
:10EFFA009199759C449FFFA1A6A43AA7BBA92AACE4
:10F00A0088AED5B011B33DB559B766B964BB54BD26
:10F01A0036BF0BC1D2C28CC43AC6DCC772C9FDCA9C
:10F02A007CCCF1CD5BCFBBD011D25ED3A1D4DBD5E2
:10F03A000CD734D854D96DDA7DDB85DC86DD80DEE9
:10F04A0073DF5FE044E123E2FCE2CEE39BE461E5A7
:10F05A0022E6DEE695E746E8F2E89AE93DEADBEAE7
:10F06A0074EB0AEC9BEC28EDB1ED36EEB8EE36EF18
:10F07A00B0EF27F09AF00BF178F1E2F149F2ADF234
:10F08A000EF36DF3C9F322F479F4CDF41FF56FF59D
:10F09A00BCF507F651F698F6DDF620F761F7A0F70A
:10F0AA00DEF71AF854F88DF8C4F8F9F82DF95FF973
:10F0BA0090F9C0F9EEF91BFA47FA71FA9BFAC3FA0A
:10F0CA00EAFA10FB35FB58FB7BFB9DFBBEFBDEFB24
:10F0DA00FDFB1BFC38FC55FC70FC8BFCA5FCBFFC43
:10F0EA00D8FCF0FC07FD1EFD34FD49FD5EFD72FDF6
:10F0FA0086FD99FDABFDBDFDCFFDE0FDF0FD01FEF6
:10F10A0010FE1FFE2EFE3CFE4AFE58FE65FE72FEF3
:10F11A007EFE8AFE96FEA2FEADFEB7FEC2FECCFEC3
:10F12A00D6FEE0FEE9FEF2FEFBFE04FF0CFF14FF32
:10F13A001CFF23FF2BFF32FF39FF40FF47FF4DFF24
:10F14A0053FF59FF5FFF65FF6BFF70FF75FF7BFF82
:10F15A0080FF84FF89FF8EFF92FF96FF9BFF9FFF30
:10F16A00A3FFA7FFAAFFAEFFB1FFB5FFB8FFBBFF22
:10F17A00BFFFC2FFC5FFC8FFCAFFCDFFD0FFD2FF46
:10F18A00D5FFD7FFDAFFDCFFDEFFE0FFE3FFE5FF95
:10F19A00E7FFE9FFEAFFECFFEEFFF0FFF1FFF3FF05
:10F1AA00F5FFF6FFF8FFF9FFFBFFFCFFFDFFFFFF8E
:10F1BA000000EE01DA03C305A9078C096C0B4A0D9E
:10F1CA00250FFD10D212A414741641180B1AD31B62
:10F1DA00981D5A1F1A21D72291244926FE27B129A0
:10F1EA00612B0E2DB92E62300832AB334D35EB361A
:10F1FA008738213AB93B4E3DE03E7140FE418A4391
:10F20A0013459A461F48A149224B9F4C1B4E944FC7
:10F21A000C518152F4536455D3563F58A959115B86
:10F22A00775CDB5D3D5F9C60FA615663AF6407669D
:10F23A005C67B068016A516B9E6CEA6D346F7B70D3
:10F24A00C171057347748775C57602783C79757AFA
:10F25A00AC7BE17C147E457F7580A381CF82F983E4
:10F26A00218548866D879188B289D28AF18B0D8D66
:10F27A00288E418F59906F9183929693A794B69551
:10F28A00C496D197DB98E599EC9AF29BF79CFA9D84
:10F29A00FB9EFB9FFAA0F7A1F2A2ECA3E5A4DCA5D2
:10F2AA00D2A6C6A7B9A8AAA99AAA88AB76AC61AD14
:10F2BA004CAE35AF1CB003B1E7B1CBB2ADB38EB42F
:10F2CA006EB54CB629B705B8DFB8B8B990BA67BBFE
:10F2DA003CBC10BDE3BDB4BE85BF54C022C1EEC163
:10F2EA00BAC284C34DC415C5DCC5A2C666C729C83F
:10F2FA00ECC8ADC96DCA2BCBE9CBA5CC61CD1BCE71
:10F30A00D4CE8DCF44D0FAD0AFD162D215D3C7D3E1
:10F31A0078D427D5D6D584D630D7DCD786D830D975
:10F32A00D9D980DA27DBCCDB71DC15DDB7DD59DE14
:10F33A00FADE9ADF39E0D7E074E110E2ACE246E3A4
:10F34A00DFE378E410E5A6E53CE6D1E665E7F9E710
:10F35A008BE81CE9ADE93DEACCEA5AEBE7EB74EC41
:10F36A0000ED8AED14EE9EEE26EFAEEF35F0BBF01F
:10F37A0040F1C4F148F2CBF24DF3CEF34FF4CFF49F
:10F38A004EF5CCF54AF6C7F643F7BEF739F8B3F8A7
:10F39A002CF9A5F91DFA94FA0AFB80FBF5FB6AFC25
:10F3AA00DDFC50FDC3FD34FEA5FE16FF85FFF4FF0C
:10F3BA00001D9307000000000000000002009907EA
:10F3CA00A307AD07B6070000001AC0070000000037
:10F3DA0000000000001BC807000000000000000039
:10F3EA000019D00700000000000000000202DA073E
:10F3FA00E407ED07F607FE0701140608ED080F08F3
:10F40A001308170800161B0800000000000000007F
:10F41A00001C210800000000000000000017280856
:10F42A000000000000000000001D9307000000001B
:10F43A00000000000201310839083C083A080000BF
:10F44A00010A3E0848084C0800000000020551085D
:10F45A005B0848084C085F08011764086C087008C4
:10F46A000000000002037408E407ED07F607FE0730
:10F47A0002047E0889088D089108950801129908E6
:10F48A009E0848084C0800000116A308A908AE08FF
:10F49A00B70800000018BE080000000000000000C5
:10F4AA001E00181D0C0D1F0102030405060708099A
:10F4BA000A0B191B1A1CFFFFFFFFFFFFFFFF80014A
:10F4CA00C000A800900080006000480030002400BE
:10F4DA00180012000C0009000600040003000200D4
:10F4EA00010000FFFFFFFFFF45094A094E095209C3
:10F4FA0056095A095E09620966096A096E09730999
:10F50A0078097D09820987098C097472616E7370A2
:10F51A00203D20000000000000000101010101015E
:10F52A0001010103020602010101000102040203B2
:10F53A0002010201080C080A080808080808080855
:10F54A00080A080C0C0000000000080C0A0A0A0A43
:10F55A000A0C0C0801020408102040800203020071
:10F56A000001000101010101000101003756656F28
:10F57A007C878B8F949AA4B0B9BFD2476C69476CC9
:10F58A006927732050363030207570677261646560
:10F59A0020616C7068612046656220203820323014
:10F5AA003135007370656564006C666F207368613D
:10F5BA0070650070756C73652D7472690072616E86
:10F5CA00642D73696E006E6F6973652D73617700C0
:10F5DA00566962207370640056696220616D740016
:10F5EA006D6F642064656C617900616D7020736869
:10F5FA0061706500666173742D6578700066617369
:10F60A00742D6C696E00736C6F2D65787000736C65
:10F61A006F2D6C696E0062656E64207467740056A3
:10F62A00636F0056636600566F6C00676C696465A9
:10F63A0000646574756E6500616D702056656C6F47
:10F64A00006C666F207467740061620061006C660A
:10F65A006F2072616E6765006C6F77006869676812
:10F66A00006D6F642072616E6765006D696E006679
:10F67A00756C6C006D6F6420746774006C666F0043
:10F68A005669620066696C2073686170650062651C
:10F69A006E642072616E676500326E640033726454
:10F6AA0000357468004F6374007072696F006C6192
:10F6BA0073740070697463680066726565007365C7
:10F6CA006D69746F6E65006F637461566500666973
:10F6DA006C2056656C6F0020726563760020736536
:10F6EA006E640062656E6465722063616C69627241
:10F6FA00617465640056632D0056632D206F66663B
:10F70A000056632D206F6E007072657365747320E6
:10F71A0064756D70656400496E742073796E630058
:10F72A004D6964692073796E630074617065207332
:10F73A00796E6300737072656164206F6E00737016
:10F74A0072656164206F6666006261736963207026
:10F75A0061746368006F6D6E690063683100636885
:10F76A003200636833006368340063683500636895
:10F77A003600636837006368380063683900636875
:10F78A0031300063683131006368313200636831B7
:10F79A003300636831340063683135006368313699
:10F7AA0000636C6561720072657374007469650048
:04F7BA00203D2000CE
:020000021000EC
:10E000002F923F924F925F926F927F928F929F9248
:10E01000AF92BF92CF92DF92EF92FF920F931F9336
:10E02000CF93DF93CDB7DEB72A970FB6F894DEBF54
:10E030000FBECDBF2FEF31EE44E0215030404040C5
:10E04000E1F700C00000F89414B817B81AB81DB86A
:10E0500010BA15B890EE98B91BB81EB883EE81BB04
:10E060002FEF24B997B947E04AB99DB980BB36EC88
:10E0700031BB469A97B94AB99DB915B880E888B9B5
:10E080001BB81EB8F7E4F1BB52E05A95F1F700C097
:10E0900086B189B18CB131BB479AE7EEE7B977EF2A
:10E0A0007AB962EE6DB931BB469AA1E0A5B982E4B6
:10E0B00088B91BB81EB887E881BB8DE08A95F1F757
:10E0C000000031BB469A97B94AB99DB9A5B920E479
:10E0D00028B91BB82EB9F1BBB2E0BA95F1F700C070
:10E0E00086B159B1BCB131BB479AE7B97AB96DB9BC
:10E0F000BDE0BA95F1F7000031BB469A97B94AB92D
:10E100009DB9A5B928B91BB82EB9F1BBF2E0FA95B3
:10E11000F1F700C026B199B14CB131BB479AE7B9CC
:10E120007AB96DB93DE03A95F1F70000422F469576
:10E13000437060E8269F90011124242B392F307101
:10E14000322B292F269526952870232B969590768D
:10E15000922B907C21E0903C09F020E0382F3695FE
:10E160003370A0E88A9FC0011124832B952F9071F2
:10E17000982B852F869586958870982B852F869568
:10E180008076982B907C81E0903C09F080E082239F
:10E1900009F4B4C286EC81BB469A21E025B990E42B
:10E1A00098B99BB91EB897E891BBBAE0BA95F1F758
:10E1B00000C081BB469A25B934E438B930E73BB991
:10E1C00032E23EB991BBEAE0EA95F1F700C081BBCB
:10E1D000469A25B922E428B920E52BB920EC2EB9BE
:10E1E00091BBFAE0FA95F1F700C081BB469A15B8E9
:10E1F00026E828B923E02BB91EB891BBAFE9BFE0F0
:10E200001197F1F700C0000081BB469A15B823E8CA
:10E2100028B923E12BB922E02EB991BBBAE0BA9517
:10E22000F1F700C081BB469A20EE27B997E09AB972
:10E230002DB915B870E878B99BB91EB867E461BB11
:10E24000E2E0EA95F1F700C036B139B13CB181BBEB
:10E25000479A57EE57B947EF4AB932EE3DB9F5E064
:10E26000FA95F1F7000081BB469A27B99AB92DB902
:10E2700015B878B99BB990E29EB961BB22E02A95A6
:10E28000F1F700C096B199B19CB181BB479A57B9DB
:10E290004AB93DB935E03A95F1F7000099249394D5
:10E2A000612C712C0F2EF4E84F2EF4E15F2EF02D2F
:10E2B0000F2EF4E82F2EF5E13F2EF02D88248394C5
:10E2C0009FD499230CF405C2803F9105C9F798D4D7
:10E2D000892B09F0FEC194D48136910509F0F9C16A
:10E2E0008FD4469709F0F5C18BD48B36910509F090
:10E2F000F0C186D499230CF4ECC1A3015827052E54
:10E300000294202D2F702527352F3025330F307E96
:10E310002327302D3527307F3695052E000C331FEF
:10E320005695569556955F7153275427422F7A017B
:10E330008F7799278C011695102F00271795079531
:10E340005FD499230CF4C5C1D701B8270B2E0294D2
:10E35000202D2F702B273B2F3025330F307E232786
:10E36000302D3B27307F36950B2E000C331FB69592
:10E37000B695B695BF71B327BA27A22F7D018F77C7
:10E380009927082B192B0115B1E01B0721F0012B50
:10E3900009F4A1C19EC134D46C0199230CF499C134
:10E3A00087011827012E0294802D8F708127912FCD
:10E3B0009025990F907E8927902D9127907F969593
:10E3C000012E000C991F1695169516951F71192789
:10E3D0001027082F15D45C0199230CF47AC1F80199
:10E3E000F8270F2E0294802D8F708F279F2F902556
:10E3F000990F907E8927902D9F27907F96950F2EBD
:10E40000000C991FF695F695F695FF71F927FE27F2
:10E41000E82FFA87E9878201F3D399230CF4F4C03B
:10E42000E984FA84A7015827052E0294202D2F7025
:10E430002527352F3025330F307E2327302D3527E4
:10E44000307F3695052E000C331F56955695569500
:10E450005F7153275427422F7A015A874987DC017D
:10E46000AF77BB27BA83A983CBD399230CF4CCC055
:10E47000F701F8270F2E0294202D2F702F273F2F02
:10E480003025330F307E2327302D3F27307F3695C0
:10E490000F2E000C331FF695F695F695FF71F327B6
:10E4A000FE27E22F7F01FA87E9879C012F77332728
:10E4B0003C832B83A5D399230CF4A6C0A70158272E
:10E4C000052E0294202D2F702527352F3025330F50
:10E4D000307E2327302D3527307F3695052E000CD2
:10E4E000331F5695569556955F7153275427422FE3
:10E4F0007A015A874987DC01AF77BB27BE83AD839A
:10E500007FD399230CF480C0F701F8270F2E0294D3
:10E51000202D2F702F273F2F3025330F307E2327BC
:10E52000302D3F27307F36950F2E000C331FF69588
:10E53000F695F695FF71F327FE27E22F7F01FA8704
:10E54000E9879C012F77332738872F8359D3992365
:10E550000CF45AC0A7015827052E0294202D2F70C5
:10E560002527352F3025330F307E2327302D3527B3
:10E57000307F3695052E000C331F569556955695CF
:10E580005F7153275427422F5A874987F8013397E1
:10E590009C013695322F2227379527955981252BB7
:10E5A0002083F80132979C0122703327002436958E
:10E5B00027950794369527950794322F202D6B8148
:10E5C000262B2083F80131979C0124703327220FDA
:10E5D000331F22953295307F3227207F3227AD813D
:10E5E0002A2B20838870992782959295907F98276F
:10E5F000807F9827BF818B2BF80180830C5F1F4F92
:10E600000215130509F008CFFBD299230CF461C061
:10E610008C01102F0027110FF3D299230CF459C04D
:10E620008F779927880F991F880F991F082B192B0F
:10E63000E7D299230CF44DC083709927082B192B2E
:10E6400029853A850217130709F043C0D9D2873FBD
:10E65000910509F03EC0990C3FE3391508F4982C58
:10E6600046EC41BB469A892D880F392D3695282FC7
:10E6700026702064992D991F9927991F292B992D70
:10E680009071482F440F4072942B807C982B832FDD
:10E690008270806285B828B99BB98EB957E851BBA2
:10E6A0006AE06A95F1F700C0B5016F777727C60178
:10E6B0008F7799279695982F882797958795682B18
:10E6C000792B762F662780E090E041E854E198D4DA
:10E6D000F7CD89E701C08DE696EC91BB469A982F5D
:10E6E0009071906E86958270806221E025B922E457
:10E6F00028B99BB98EB987E881BBFFCF2A960FB6A0
:10E70000F894DEBF0FBECDBFDF91CF911F910F9167
:10E71000FF90EF90DF90CF90BF90AF909F908F9041
:0EE720007F906F905F904F903F902F900895E4
:10EC000045E04A95F1F70000349B04C000C000C005
:10EC10003499FCCF86EC81BB469A20EE27B997E069
:10EC20009AB92DB915B820E828B99BB91EB897E450
:10EC300091BB52E05A95F1F700C096B129B13CB1B1
:10EC400081BB479A87EE87B987EF8AB982EE8DB983
:10EC500085E08A95F1F70000392F3695337040E84A
:10EC6000949FC0011124832B922F9071892B922F96
:10EC7000969596959870892B26952076282B217B42
:10EC8000213809F040C026EC21BB469A90EE97B996
:10EC900087E08AB99DB915B890E898B98BB980E238
:10ECA0008EB987E481BB52E05A95F1F700C036B1C6
:10ECB00099B14CB121BB479A87EE87B987EF8AB9E2
:10ECC00082EE8DB985E08A95F1F70000832F869555
:10ECD000837050E8359F90011124282B892F807173
:10ECE000282B892F869586958870282B9695907667
:10ECF000292B50E0CA01880F991F84709927822B15
:10ED0000282F30E002C02FEF3FEF822F932F08957E
:10F000008F929F92AF92BF92CF92EF92FF92CF9347
:10F01000DF93EA01CFB6F894F999FECF23E0FB0124
:10F0200080935B002093570010D707B600FCFDCFFC
:10F03000DE01B3954B015C0121E04881F980E12CB0
:10F04000F701E40FF11DAF0122960A01F401A0922D
:10F050005B0020935700F9D61124F2E08F0E911C2B
:10F06000A11CB11CAC17BD0741F725E0FB01809343
:10F070005B0020935700E9D607B600FCFDCF81E185
:10F0800080935700E2D6CFBEDF91CF91FF90EF90F3
:0CF09000CF90BF90AF909F908F9008959C
:00000001FF
